:020000040000FA
:10000000409401204D2F0000FF7700007D2F00005D
:100010007D2F00007D2F00007D2F00007D2F000030
:100020000000000000000000000000002D2D000076
:100030007D2F000000000000D52C00009775000007
:100040000D2F00000D2F00000D2F00000D2F0000C0
:100050000D2F00000D2F00000D2F00000D2F0000B0
:100060000D2F00000D2F00000D2F00000D2F0000A0
:100070000D2F00000D2F00000D2F00000D2F000090
:100080000D2F00000D2F00000D2F00000D2F000080
:100090000D2F00000D2F00000D2F00000D2F000070
:1000A0000D2F00000D2F00000D2F00000D2F000060
:1000B0000D2F00000D2F00000D2F00000D2F000050
:1000C0000D2F00000D2F00000D2F00000D2F000040
:1000D0000D2F00000D2F00000D2F00000D2F000030
:1000E0000D2F00000D2F00000D2F00000D2F000020
:1000F0000D2F00000D2F00000D2F00000D2F000010
:100100000D2F00000D2F00000D2F00000D2F0000FF
:100110000D2F00000D2F00000D2F00000D2F0000EF
:100120000D2F00000D2F00000D2F00000D2F0000DF
:100130000D2F00000D2F00000D2F00000D2F0000CF
:100140000D2F000053B94AB9002908BF00281CBF71
:100150004FF0FF314FF0FF3000F06CB9ADF1080CFB
:100160006DE904CE00F006F8DDF804E0DDE90223D5
:1001700004B070472DE9F047089D04468846002BDF
:100180007DD18A4217463FD9B2FA82F242B1C2F11A
:1001900020009140974024FA00F0944040EA010882
:1001A0004FEA174C230C1FFA87FEB8FBFCF60CFB3A
:1001B000168106FB0EF043EA0143984205D9FB186D
:1001C00002D2984200F22481013E191AA3B2B1FB77
:1001D000FCF00CFB101100FB0EFE43EA0144A645A7
:1001E00005D93C1902D2A64500F20F81013840EA38
:1001F0000640A4EB0E0400261DB1D4400023C5E93F
:1002000000433146BDE8F08702B9FFDEB2FA82F260
:10021000002A50D1CB1B4FEA174E1FFA87F8012650
:10022000210CB3FBFEFC0EFB1C300B4608FB0CF94B
:1002300041EA004189450AD979182CBF01230023DE
:10024000894502D9002B00F0D9800CF1FF3CA1EBCD
:100250000901A3B2B1FBFEF00EFB101108FB00F880
:1002600043EA0144A04505D93C1902D2A04500F259
:10027000C9800138A4EB080440EA0C40BCE78B427B
:1002800009D9002D00F0B1800026C5E900013046F3
:100290003146BDE8F087B3FA83F6002E46D18B4293
:1002A000C0F0A680824240F2A3803046002DA8D044
:1002B000C5E90048A5E79740C2F1200301FA02F022
:1002C0004FEA174ED94024FA03F31FFA87F89440F7
:1002D0000343B1FBFEF01E0C0EFB101100FB08FCEB
:1002E00046EA01418C4509D979182CBF0126002620
:1002F0008C4502D9002E00F093800138A1EB0C014F
:100300009BB2B1FBFEF60EFB161106FB08FC43EA9E
:1003100001418C4505D9791802D28C4500F28780BD
:10032000013EA1EB0C0346EA004679E7C6F120073F
:1003300003FA06F402FA06FC01FA06FEFA4020FA75
:1003400007F8F94000FA06F3224348EA0E044FEAA0
:1003500012484FEA144E1FFA82F9B1FBF8FA08FB73
:100360001A110AFB09F04EEA014E70450AD912EB48
:100370000E0E2CBF01210021704501D9002952D059
:100380000AF1FF3AAEEB000EA4B2BEFBF8F008FB98
:1003900010EE00FB09F944EA0E4EF14505D912EBC7
:1003A0000E0E01D2F14538D8013840EA0A40AEEBD2
:1003B000090EA0FB0C89CE4541464C4602D306D11E
:1003C000434504D20138B8EB0C0169EB020415B3C4
:1003D0005A1A6EEB040EF2400EFA07F72EFA06F3E5
:1003E00000261743C5E900730BE72E46284608E7A9
:1003F000841A61EB03010120884657E7ACF1020C37
:10040000394424E702383C4434E702383C44EEE601
:10041000023E3B44D9E62E46F3E602389644C4E752
:10042000023839446AE7AAF1020A9644AAE7023E72
:10043000394476E7704700BF7FB5404B404A41489A
:10044000C3F800264921C3F80426C3F80826C3F8D8
:100450000C26C3F81026C3F81426C3F81826C3F8D0
:100460001C2606F06BFD06F080F9374800F080F896
:1004700028B94521344A354806F060FDFEE7344886
:1004800004F05AF80446C56883684FF488721A214C
:100490001B68984718B92B6823F080632B60A3680A
:1004A00020465B6801A9984790B9019B5A010FD477
:1004B0004FF05023D3F800340BB1DB0708D54921A6
:1004C000244806F03BFD01F06FFF234802F0EAFAF2
:1004D00001A800F075FC214B1B68984204D045210F
:1004E0001F4806F02BFDFEE7039A49211D4806F040
:1004F00025FD49211C4806F021FD69469DF80800AC
:1005000000F042F8009B039C1C44019B1D89661966
:100510004FF02002EFF3118382F31188BFF36F8F46
:1005200007F03BF800F034FF635983F308887368E1
:10053000984745210D4806F001FDFEE70080015077
:100540003546526E18890000318900004489000048
:10055000638900006A890000788500005447012003
:100560008E890000B1890000E0890000058A000042
:1005700010B5044C236813B903F0DEFF2060206837
:1005800010BD00BF5047012008B540B1024600230E
:100590000448452106F0D2FC6FF0150008BD086044
:1005A000FCE700BF288A00001FB5074A03460C4637
:1005B0001068194601AA07F044FA18B9019B236094
:1005C000029B636004B010BD504701202DE9F04F3D
:1005D000DFF81C92DDB01546DDE968481E46DDF8FF
:1005E00098B1D9F8007000F0A1FE01227E4B3CA822
:1005F000C3F8002504F0EAFFCDF814903CB1B8F13F
:10060000000F04DD424621463CA806F031FC4FF0C5
:1006100000096B89B5F808809844EB689844C84590
:100620004ED80FA93CA805F043F800226E4BC3F842
:100630000025C3F800256A9B23B1202218460FA984
:1006400007F011F900233246009329464FF6FF7355
:1006500009A806F08BF80446002844D14FF0FF3576
:10066000DFF890A1DFF8808103900DF11E0307AA47
:1006700008A909A806F0C6F8041E34DB40F0A480DF
:10068000BDF81E90B9F1100F38D1BDF81C90B9F12A
:10069000200F40F0A3804B46304608993CAA06F054
:1006A00068FE0446F8B94A463CA90FA806F04EF980
:1006B00004464E4B1B68834215D101230393D4E7B4
:1006C000679AA8EB09039A4228BF1A46494613467F
:1006D000924630465A4606F04CFE044638B1002297
:1006E000414BC3F8002520465DB0BDE8F08F52466F
:1006F00059463CA806F0BCFBD14490E7B9F1010F84
:100700003FD1BDF81C30202B68D8304608993CAA50
:1007100006F02FFE04460028E5D19DF81C50202D40
:100720000AD8DAF80030DFF8D0B00493049B9C427A
:1007300005DB0023C8F800354FF0FF341DE000F062
:10074000F5FDC8F800951FA804F040FFDBF8042071
:100750001FA812685BF8081B06F08AFB17A91FA8E0
:1007600004F0A6FF00223CA9C8F8002517A82A46D5
:1007700007F069F818B9C8F80005254675E701348F
:10078000D4E7B9F1220F7FF470AF002D19DBDAF84E
:100790000030AB4215DDBDF81C30802B1ED8304632
:1007A00008993CAA06F0E5FD044600289BD1EDB26D
:1007B0002021BDF81C3000953CAA0FA800F01EF8BF
:1007C00007464FF0FF3550E7039B53B1074B1B68BB
:1007D000BB4201D0059B1F683C4684E74FF0FF34C5
:1007E00081E701247FE700BF0000845054470120C7
:1007F0000045012080850000848500002DE9F0433C
:1008000097B090461E469DF87820364B0F4653F819
:10081000321003EBC2035B688146186801913023F4
:10082000014402AA01A806F0B0FA10B14FF0FF305F
:1008300055E0DDE901531D44294606AB03AA01A892
:1008400006F0CBFA0028F1D1049A072AEED1264906
:10085000059806F0F8FF0028E8D1079A082AE5D1A4
:100860002249089806F0EFFF0028DFD1294602AAA6
:1008700001A806F09EFA0028D8D1DDE90143E2186C
:100880009542D3D1412BD1D12378042BCED14644EC
:1008900001343023314603AA02A80194CDF8088020
:1008A00006F073FA0028C1D1DDE9023213449E42FA
:1008B000BCD3324602A906A805F0EFFF0028B5D147
:1008C000324602A90EA805F0E8FF0028AED1202F7D
:1008D000ACD13B464846019906AA00F03FFD17B04F
:1008E000BDE8F083848500004E8A0000568A00002F
:1008F0002DE9F041022386B00D466F460026DFF851
:100900006C80ADF8003017F8010B01A901F022F955
:100910000446D8B901981023816802AA103906F05C
:1009200028FD044628B1019806F022FD0EE00126BC
:10093000E9E71022414602A806F085FF50B1019870
:1009400006F016FD002EF2D04FF0FF34204606B020
:10095000BDE8F081019807F02BFA0423A0F108010B
:100960002A46019806F005FD0446DCE7688700008A
:100970002DE9F041384B88B0064600200D461C6832
:1009800005F0EAFE06A9C0B201F0E4F8002857D14C
:10099000294605F0E1FE2C2407A9C0B204FB05643A
:1009A00001F0D8F8002836D04FF02C0808FB05F8E5
:1009B00006EB0807396911F0100137D14FF4807345
:1009C0000193264B224600930846CDE90311069B6E
:1009D0000291FFF7FBFD0446214B56F808200698CC
:1009E0009A420CD13A89FB68D1438B4207D8134411
:1009F0008268934203D21B4B1B68A3421DD045B3B0
:100A00008268002106F0FBFC174A4521174806F0D2
:100A100095FA012411E0079806F020FD0746079893
:100A200006F0A6FC631EE21C93420DD1002DF0D00F
:100A30003046069906F08CF82C46069806F098FC8D
:100A4000204608B0BDE8F08113F8011FB942EBD091
:100A5000AAE7074AD9E700BF004501207A660120CE
:100A60003DB8F396544701205F8A0000718A000068
:100A7000698A000073B50D46002104462846CDE979
:100A8000001106F024F830B3164E2268B24203D1AA
:100A9000204601AA05F091FFE36AB34204D16A46F9
:100AA0000121204605F089FFDDE90032934288BF2D
:100AB0000193019BAB60019A2946204600F026FB7A
:100AC000094B1A68002A03DD5721084806F036FA58
:100AD000002002B070BD05F10801FFF709FFAB6807
:100AE0000193E8E73DB8F396B8570120998A0000D2
:100AF0002DE9F84F8A46904699460026DFF870B0F7
:100B0000194C1A4D0B9B9E4201D300200FE00B9B0A
:100B100050469F1BB7F5806F28BF4FF48067144A7B
:100B20003B4606EB090106F024FC10B10120BDE8AC
:100B3000F88F0A993B465A464046711806F036FC33
:100B40000028F3D1C4F800563E44C4F80456C4F853
:100B50000856C4F80C56C4F81056C4F81456C4F815
:100B60001856C4F81C56CDE7008001503546526E29
:100B70007A6201202DE9F043894B0446602285B05A
:100B80000F4600211E6806F099FE0021854B08469D
:100B90006362854B236505F0DFFD04F12001C0B2DF
:100BA00000F0D8FF0121002005F0D6FD04F14C0132
:100BB000C0B200F0CFFF0546204605F05FFF0246B9
:100BC00038B14FF480725721784806F0B7F9012305
:100BD0008DE00146204605F038FF804618B100221E
:100BE00057217348F1E7204600F0A6F90028EED01F
:100BF000684605F063FF6946204605F0FDFF18B121
:100C0000424657216B48E0E7684605F060FF80F0F8
:100C100001006A46C1B2204605F017FF02460028CF
:100C2000DDD1684605F053FF804660BB694620462B
:100C3000FFF720FF9DF8073084F85830033B012B65
:100C400006D8404606F025F810B1FF2384F8583046
:100C50009DF80730023B022B0BD8002006F007F866
:100C600038B1FF2384F858304521534806F066F91F
:100C7000FEE794F85830FF2BF6D06A460021204654
:100C800005F0E3FEA3E79DF80790B9F1010F23D12A
:100C9000104603F081F9831E022B80460DD8494689
:100CA0002046FFF765FE454B1B68984205D001289A
:100CB0000CBF4FF001084FF0050884F8588094F8F5
:100CC0005830042B8DF8073014D8012B18D82FD0AA
:100CD000FF2384F858302BE001212046FFF748FE1F
:100CE000364B1B68984214BF05239DF8073084F8E3
:100CF0005830E4E7052BEBD1002005F0CAFF12E0E5
:100D000069462046FFF7B6FE94F858300546DA1ECD
:100D1000012A0BD8002005F0BCFF05460028D7D1DA
:100D2000002005F0A4FF054610B1D1E7022BF7D053
:100D300094F85830FF2B04D145211F4806F0FEF8E7
:100D4000FEE7012B06D06A460021204605F07DFE15
:100D50000546B8B900212046FFF70AFE0646DFF82F
:100D60005C80D8F8003083420CD110220021684604
:100D700006F0A4FD236AD8F800605A783A715B68DF
:100D80003C60BB60E06C06F0F3FA206A06F0F0FA13
:100D9000002D14BF2846304605B0BDE8F08300BFE3
:100DA00000450120B8470120B84F0120C88A000043
:100DB0000A8B0000368B0000608B00005447012036
:100DC00008B501460148FFF7D5FE08BD5847012088
:100DD00073B516461C4633B3436A5D686379012BCD
:100DE00015D101BB1F4B22681B689A4298BF002592
:100DF000002005F0B1FC01A9C0B200F0ABFEF0B1DB
:100E00000125019806F0B4FA284602B070BD022B05
:100E100009D12368012B08D9124A1268934202D8DB
:100E2000B1FA81F149090025E2E7FCD10029DFD0C0
:100E30000129F8D12179023918BF0121F3E72946A8
:100E400020233246019806F094FA05460028D7D1AF
:100E5000002CD6D0356804482D1A18BF4FF0FF3546
:100E6000CFE700BF044501203DB8F3962DE9F04FD0
:100E700007460C4685B001460020164605F06DFD7C
:100E8000051E52DB3846E46D05F071FD5FFA84F90A
:100E90004FF0000A4FF0010B4FF0FF3405F1FF381F
:100EA00009FB08089DB9BAF1010F03DD452121486E
:100EB00006F044F8631C06D0FF2C2ADC40F2011334
:100EC00001343460B380284605B0BDE8F08F6B1E56
:100ED00000934146012338460DF10F0206F049FA0E
:100EE000031E019323DB012238460DF10F0106F0AA
:100EF00070FF019B40B19B4501D00AF1010A9B465E
:100F0000009DA8EB0908CDE7B4F1FF3F08BF2C46D0
:100F1000F5E70223A4F580747371631004F00104F3
:100F20000133013433603471CDE70725CBE7012568
:100F3000C9E700BF6C8B000038B5826A446DA242DD
:100F400008D0631C934205D05721144805F0F6FFE2
:100F5000002038BDB2F5807F1CD957211048F5E735
:100F6000416A056D01EBC30105EBC30549686D6876
:100F70008D4202D057210B48E8E70133A342EFD15D
:100F80009A4205D9426A02EBC3035B689942F1D1E8
:100F90000120DEE700231946F0E700BF8F8B000039
:100FA000C78B0000F68B000000B589B0022004A9B1
:100FB00006F042FF9DF81020012A41D0254B26491A
:100FC000032A18BF0B469DF81320492102929DF871
:100FD0001220224801929DF811200092204A05F02B
:100FE000ADFF062006A906F027FF9DF81820012A6C
:100FF00028D0184B1849032A18BF0B469DF81B2010
:10100000492102929DF81A20144801929DF8192056
:101010000092144A05F092FF9DF81030012B13D175
:101020009DF81230032B0FD19DF81830012B0BD0F7
:101030000D48492105F082FF022009B05DF804FB4C
:101040000A4BC0E7094BD9E70948492105F076FF6B
:101050000020F2E7278C00002D8C00003F8C000060
:10106000318C0000808C0000908C0000228C0000ED
:10107000AF8C000070B5064618464B6814461D4AF2
:1010800003F0FF2393420D4686B02ED10B68012B4F
:101090002BD104A906F0D0FE9DF81020012A26D0FD
:1010A000154B1649032A18BF0B469DF813204921FA
:1010B00002929DF81220124801929DF81120009290
:1010C000104A05F03BFF9DF81030032B0DD121464F
:1010D000304605F03DFD204606F09EFE2046A968FC
:1010E00005F05CFC204602F0F9FE06B070BD064B30
:1010F000DBE700BF00010004278C00002D8C0000FE
:101100003F8C0000808C0000228C00002DE9F04F05
:10111000436A2DED028B0C465E68054601210023D3
:101120008BB033449342084601F10101F9D3784F63
:101130003860204605F0CBFCBB46C8B1E86D05F031
:1011400007FC0022AB6A013B3244904201D9013BCB
:10115000FAE7DBF800209A420AD357216D4805F0E0
:10116000EDFE0123E3710BB0BDEC028BBDE8F08F07
:1011700008A9022000F0EEFC09A9062000F0EAFC14
:10118000062321462846099AFFF774FF6379012B4D
:1011900008D1DBF80070DFF880A1DBF80030A7B9D8
:1011A0000123236002230127DFF86C81637105931B
:1011B000DBF80030DDF820909F424DD9484606F01C
:1011C000D7F8099806F0D4F8CDE7226801339B1AC6
:1011D0009F423FD86B6A012A196853F8370003EB26
:1011E000C70353F8083CDDF82080A3EB010308EEA9
:1011F000103AA0EB010912D1E268099B022A0AD039
:1012000041462846039305F0A3FC22464146284662
:1012100005F0D3FC039B1946284605F099FC32469D
:101220004946404605F092FC18EE103A42464146C7
:101230002846CDE90096FFF75BFC2146284605F0DD
:1012400053FC23680133236020B1DAF80030013306
:10125000CAF80030013FA0E723689F4256D3696A6D
:10126000286D51F83730FA0004930B68083A50F8AB
:1012700002C0039303682079DDF824A00128ACEBB9
:10128000030341D189580793039B3246C91A484644
:10129000069105F05BFC0699079B4A46009128469B
:1012A000514601960693FFF723FC2146284605F098
:1012B0001BFC059B2371069B20B1D8F8002001324E
:1012C000C8F80020194632465046069305F03EFC09
:1012D000069B494600932846DDE9032301969B1AA5
:1012E0005246FFF705FC2146284605F0FDFB236822
:1012F000013323604FF00103237138B1D8F8003077
:101300000133C8F8003001E00228DBD001374FE795
:1013100004450120C68C0000B8570120024B0A4644
:101320001B680021184700BF0845012070B5094D12
:101330002B7853B90126084CC4F8006504F0E8F98D
:1013400028B92E70C4F8000570BD0020FCE74FF0EE
:10135000FF30F9E77A6701200000845070B5AEB025
:101360001D460446CDE90221FFF7E0FFDDE9022139
:101370000123064E05A8C6F800352346009506F061
:1013800051FF0023C6F800352EB070BD0000845018
:101390000122124B12491A604FF0FF33C1F8483353
:1013A000C1F8083301F580514A60043100210D4A2B
:1013B000C2F84833C2F80833A2F55042C2F800150B
:1013C000C2F8083302F58052C2F80015C2F808339B
:1013D0004FF05022C2F80833704700BF044001505C
:1013E00000400150005001502DE9F043079C1CB90A
:1013F00020461460BDE8F0830325B4FBF5F505EB4A
:101400004507BC4218BF0135B5F1804F05D34FF0F9
:10141000FF3313606FF00B00ECE7AD0001358D4238
:1014200000D808B91560F5E706460025DFF8B4E0F6
:10143000BD4231469C4606F1040603F1030329D35D
:10144000A54222D20135A54228BF00239CF80060A6
:10145000244F38BF9CF801304FEAA60C17F80CC097
:10146000A54281F800C007EB131C2FBF3D239B0052
:1014700003F03C03FB5C36018B703D2306F0300625
:101480001CF80660CB704E700431081A1060002002
:101490000870AFE713F803CC13F8021C4FEAAC094D
:1014A0001EF809904FEA0C1C13F8018C0CF0300C5C
:1014B00006F8049C0EEB111919F80CC0890006F807
:1014C00003CC01F03C010EEB981C1CF8011008F055
:1014D0003F0806F8021C1EF80810033506F8011C28
:1014E000A6E700BFD08D00002DE9F04300273C4661
:1014F0003D46079EDFF82881B5420AD32E4604E018
:101500000135AE420EF1010E05D1CCBB14600020B6
:1015100056E04FF0000E13F805C0BCF1200FEFD0DD
:10152000AE42F2D0A6EB0509B9F1010F15D9BCF115
:101530000D0F12D103EB050999F80190B9F10A0FCB
:101540001CD0BEF1000F05D1BCF13D0F08D1013711
:10155000022F08D96FF0150032E0BCF10A0FEFE757
:101560001CF0800FF6D118F80CC0BCF17F0FF1D041
:10157000BCF13F0F01D8002FECD101340135BBE79E
:10158000062504F0070CE40805FB0CFC6C430CF189
:10159000070CE41B04EBDC0478B18C420DD8002767
:1015A000014603253C46DFF878E0DFF878801E44EA
:1015B0009E4207D1091A1160A9E76FF00B00146071
:1015C000BDE8F08313F8019BA9F10A0C5FFA8CFCCB
:1015D000BCF1160F04D828FA0CFC1CF0010FE7D15F
:1015E0001EF809C00134BCF1400F08BF013D0CF0EA
:1015F0003F0C042C4CEA8717DAD17DB13C0C012D4D
:101600000C7002D101310024D2E7022D4FEA1724D9
:101610004C7016BF8F7002310331F4E72C46C7E7D8
:10162000508D0000090040000B6801330B60014B36
:101630001B6818470C45012007B50B4600210246E0
:101640000191034801A900F0EDF803B05DF804FB37
:10165000291600002DE9F74FB0F81890044619F04C
:10166000080893460ED001290CBF49F0100949F033
:101670002009A0F818908BF31188BFF36F8F03B087
:10168000BDE8F08FDFF898A109F00709022907D11A
:10169000204605F060FC0028EDD00128238B4DD1B9
:1016A0006769218B002F15DA256821F00701C4E94D
:1016B000008841F0010121830026218B01F00702FF
:1016C0004A4502D0A368002B59D10DB9002E71D024
:1016D000002355E001F007035A1F012A1FD821F00B
:1016E0000701062B256889B2C4E900880CD1002DBA
:1016F0002B4638BF00232BB1628B1B6801326283FB
:10170000002BF8D141F002012046218305F023FC93
:101710000028D1D0238B43F020032383CCE7042B74
:101720000AD121F0070189B22046218305F013FC7C
:1017300010B141F0200121830025BDE7032809D124
:10174000226923F00703166843F00603002523836C
:101750002F46B2E7042806D1226923F00703566812
:1017600043F00403F2E7052806D1226923F00703BA
:10177000966843F00503E9E700252E46E8E70123D4
:1017800041F0080121838BF31188BFF36F8F03BBF6
:10179000002D34D116B151462046B0474FF02003FA
:1017A000EFF3118B83F31188BFF36F8F238B23F03B
:1017B00008032383238BDA062AD5012123F01003A3
:1017C0002383B4F8189009F0070900297FF45EAF6D
:1017D00051E7A1680029DBD00B68002B38BF00233C
:1017E000994620463B46D1F804B00192D847019A69
:1017F000B9F1000FCCD04946D9F80030EDE72946C1
:101800003B46204601922D6805F0C1FB019ABFE7D7
:1018100013F020011EBF23F0200302212383D0E711
:10182000BB6F00002DE9F04F002406468B469A4618
:101830004FF0FF3527468DB00B9402F1FF394FF082
:1018400000080AE0B8F1000F0FD1252800F03A8116
:101850005946B0470B9A01320B9219F8010F002834
:10186000F0D10B980DB0BDE8F08F7A280AD8622825
:1018700012D8302853D047D8252800F01D812D28B4
:1018800000F0278159462520B0470B9A594601326E
:1018900099F800000B9210E1A0F16302172AF1D829
:1018A00001A353F822F000BFA91A00005B19000041
:1018B0008518000085180000851800003D190000FB
:1018C0005B19000085180000851800003D19000014
:1018D000851800008518000085180000E519000033
:1018E0008518000085180000831A00008518000084
:1018F0005B1900008518000085180000E51900003C
:10190000851800003D19000039280DD95828B9D193
:101910006C2C40F0AA8000235AF8042B91E0002D93
:1019200002DA002F00F0D7800A2225EAE57502FBD3
:101930000505002F08BF0227303D8EE7682803D138
:10194000682C06D1482488E76C2802D16C2C00F062
:10195000C480002C96D104467FE77A2C06D1D0466D
:1019600058F8042BD317752828D111E06C2CF6D029
:101970004C2C06D10AF1070323F00708F8E80223EC
:10198000F1E77528DAF800200AF1040815D10023E0
:10199000F81E18BF0120012F0CBF30212021CDE9F6
:1019A00001010A200DF12C0E009059463046CDE978
:1019B000035E05F058FCC24641E7D317002A73F1D5
:1019C0000001E5DA59462D20CDE90623B047DDE9CF
:1019D00006230B98524200F101000B9063EB430386
:1019E000013DD5E7702893D15AF8048B3C4B3D4A12
:1019F000B8F1000F18BF134613F8010B59460693B0
:101A00000993B0470B98069B01300B90187800287B
:101A1000F2D1B8F1000F11D16A1F032F7FF40FAF7D
:101A20009046B8F1000F7FF70AAF59462020B04723
:101A30000B9A08F1FF3801320B92F2E74246034657
:101A4000023DF81E18BF0120012F0CBF30212021BC
:101A5000CDE9010110200DF12C0E009059463046C1
:101A6000CDE9035E05F0FFFBE9E64C2C7FF453AFB4
:101A70000AF1070323F007039A465B685AF8082B1C
:101A8000DFE75AF8048B43469C4613F8010B18B95C
:101A9000ACEB0802AA1AC0E759460693B0470B9868
:101AA000069B01300B90EFE759465AF8040BB047FC
:101AB0000B9B01330B93C2E65946B0470B9A013298
:101AC0000B92BCE6444647464FF0FF354FF0010805
:101AD000C3E60327C1E60127BFE64C24BDE600BFED
:101AE000108E0000168E00004FF02002EFF31183DD
:101AF00082F31188BFF36F8F0121044AC2F84015A9
:101B000083F31188BFF36F8F00207047009003505C
:101B100020B1034B800143F001031847704700BF19
:101B200070850000094B30B51D68094B1C68002307
:101B30009D4202DC0021084630BD1A01A25C04EB84
:101B400003118242F7D00133F2E700BF2086000084
:101B500010450120084B10B51B680C462BB1FFF750
:101B6000E1FF28B12060002010BD6FF00C00FBE702
:101B70006FF00100F8E700BF1045012030B589B0D3
:101B80000C4615460190FFF7CDFFB8B143682268B7
:101B900002938368C068CDE903350023CDE90623AD
:101BA000059305F0C5FB60B1074901AA05F04DFF9B
:101BB000079808B9059B236009B030BD6FF0150088
:101BC000FAE76FF01200F7E73573000007B50190F0
:101BD0004FF02002EFF3118382F31188BFF36F8F70
:101BE00005F0DBFC019801F097FB034805F0A6F92E
:101BF00001F00CF9FCE700BF238E000070B504462D
:101C00000C250D480E46231A9A100C4B40215343C5
:101C1000DBB25D4305F14003184405F031FC011EC1
:101C200004DB074B2B445B68984700212046334672
:101C3000BDE87040184700BFCC570120B76DDBB638
:101C4000388600002DE9F0410F4C104D031B9B100E
:101C50005D43EBB20C255D43074605F140000E469F
:101C60002044402105F025FC011E08DB084B2C44D4
:101C7000C4E90E36074B5B59BDE8F04118473846BA
:101C80003346BDE8F0411847CC570120B76DDBB6AD
:101C90001B7500003886000070B500220121044643
:101CA000052001F071F8052001F050F80F4802F00E
:101CB0009BFA0F4B984215D106F0E3F8E6680D4900
:101CC000304605F098F900280BDB01253564E468FF
:101CD000084904F11C0005F08EF9002801DB002002
:101CE000E56470BD6FF00400FBE700BF351D000028
:101CF0000000AD0B5086000073B50C230146002692
:101D00004B430A48C4184033D4E90E521844A66322
:101D1000019205F0ECFB35B12B46019A044802B064
:101D2000BDE87040184702B070BD00BFCC5701201D
:101D30000446012010B1012804D07047034B1B6CEE
:101D40005B0701D1FFF7D8BF704700BFCC57012018
:101D500008B54FF02003EFF3118183F31188BFF32F
:101D60006F8F124A136843F0020013F001031060F2
:101D70000CD04FF05022D2F80C34D2F80C2413F0CF
:101D8000010303D00A4805F0B2FB012381F3118857
:101D9000BFF36F8F23B1BDE808400020FFF7ACBF51
:101DA0000120BDE8084002F02FBA00BF1C580120F6
:101DB0000C580120074BD3E8EF2F22F00201C3E8B3
:101DC000E01F0028F7D1D30702D4012002F04EBA59
:101DD000704700BF1C5801202DE9F8430122064638
:101DE0003949D1E8EF3FC1E8E02F0028F9D133B9F4
:101DF000364937484B60CB608A6005F00FF9731E97
:101E0000012B32D8012E07D14FF05023D3F81C34C8
:101E100003F00303022B28D006F0D7F9044618B9C3
:101E20002C4B1B78002B47D14FF02003EFF311858B
:101E300083F31188BFF36F8F0124274FDFF89C8055
:101E4000DFF89C904FF05022D2F81834D2F81824C2
:101E5000D2030CD503F00303022B01D0012E06D1CF
:101E600024B385F31188BFF36F8FBDE8F883C4B145
:101E7000284600F0D9FF4FF05022D2F81835DBB2D7
:101E8000012BDFD139680029DCD0002139603968A5
:101E90000221C2F818152022C8F88021C9F80030A4
:101EA000D0E70021212002F00BFFE4E74FF05023A0
:101EB0000222C3F80423D8E74FF05023022205463C
:101EC000C3F80823B9E700BF20580120BC57012000
:101ED000E85701203F6C01200451005000E100E070
:101EE00008500050044A1368C91A21F07F40034487
:101EF000136002F0FBBF00BF305801202DE9F0470E
:101F00004FF480374FF00009860000F1500406F1CD
:101F10005026A40006F58036A4B204F15024D6F869
:101F20004035DFF86C8021F07F4504F58034874030
:101F3000D8F804A5A3EB0A0323F07F432AF07F42DD
:101F4000012BC6F8402502D1132006F044F90AF10E
:101F50000202AB1A23F07F43B3F5000F88BF15468A
:101F6000C4F80090236825F07F43C8F84473C6F88E
:101F70004035D8F804359A4506D0EB1A023B23F0D9
:101F80007F43B3F5000F01D8BDE8F0872B46CFE7BC
:101F900000500150F8B5002427460F4E0F4B104A51
:101FA00018461D6804B1F8BDD2F80413C903FAD568
:101FB00031680029F7D0346031684FF48031C2F8BD
:101FC00048130124D2F8401525B100205A681F603B
:101FD000A847E3E70560E6E7405101502458012097
:101FE0000050015038B500244FF480334FF40012F4
:101FF0000D4D0121C5F80845C5F804330B4B1520DC
:10200000C3F88021224600F0BFFE152000F09EFE9E
:102010000123074A02201360064A2B601360FFF772
:10202000DBFE204638BD00BF0050015000E100E05B
:10203000085001502C580120134BB0F1FF3F08BF4E
:102040001846013800281CDD9842A8BF18460F4BDF
:10205000D3F804250E4B1968521A12F4000F18BF5A
:10206000002022F07F4301330A4A03440A481060EB
:1020700000205060044A934294BFC9188918FFF7A2
:102080003DBF0020E3E700BFFFFF7F00005001508D
:102090003058012024580120E51E00004FF0200296
:1020A000EFF3118382F31188BFF36F8F064AD2F8E2
:1020B0000405064A1268801A20F07F4083F31188D5
:1020C000BFF36F8F704700BF0050015030580120A0
:1020D000014802F0CDBF00BF5C86000008B5B0B17A
:1020E0004368042B0DD100220368D3E8EF1F0129B8
:1020F00003D1C3E8E02F0028F7D1074808BF1046F6
:1021000008BD3BB1006802F0D5FB0020F8E76FF492
:10211000E040F5E70148F3E7E98FFFFFEA8FFFFFB3
:1021200010B5044618B90D4B0D485B6898476168B7
:1021300008290DD031F004030AD011F0020108D0B3
:102140002146084802F014FB00232360002363604B
:1021500010BD1422206805F0B1FBF7E7A44501206B
:10216000768E00003458012010B5044618B9164B7D
:1021700016485B6898476368042B23D0082B21D04E
:10218000CBB92368BBB94FF0FF324FF0FF33214684
:102190000F4802F0BBFA08B923681BB90A4B0D4877
:1021A0005B68984714220021206805F087FB63686C
:1021B00043F002036360206805F053FF636843F057
:1021C0000103636010BD00BFA4450120768E0000AE
:1021D000345801209C8E000008B5E8B14368042BF8
:1021E0000CD101220368D3E8EF1F002903D1C3E813
:1021F000E02F0028F7D10BD1002008BD53B10068B3
:102200004FF0FF324FF0FF3302F0DCFA0028F3D03A
:102210000348F2E70348F0E76FF4E040EDE700BF62
:10222000E98FFFFFEA8FFFFF08B50649402314221C
:10223000054805F0FBFEBDE808400449044802F0EB
:1022400069BF00BF50580120345801207486000037
:1022500064860000F7B5254D286883685B6C03B180
:102260009847286883685B6BABB1984798B1204C5E
:10227000204E286883689B696BB101220DF107012C
:102280009847012807D1236873B933682BB94521D2
:10229000194804F053FE03B0F0BD71681A688B4210
:1022A000326000D17260236014499DF807700A887B
:1022B0000846B2F5007F06D2236802F1010C1344F0
:1022C000A1F800C01F720A2FD3D1236802880C49DD
:1022D0005A6000221A604E6826B9C1E900330280B4
:1022E0002260C5E733604B60F9E700BF78610120E9
:1022F000585D0120505D0120C98E000078620120E8
:1023000070610120044B10B5044618688368E1B27F
:102310005B689847204610BD78610120F8B50646F5
:102320000B4615464FF02002EFF3118C82F3118813
:10233000BFF36F8F194C216849B1194A5068884220
:1023400005D000200860506898B9C2E90011154A0C
:10235000116829B157680868B942106008BF506019
:102360008CF31188BFF36F8F216029B9002028609A
:10237000F8BD01605160EAE748680831F6D05C1E9C
:102380008442A8BF04463046224605F06CFA00237A
:10239000335501232B60E018EAE700BF5C5D0120A4
:1023A000505D01207061012037B500251D4B1E4A8C
:1023B000C3E900551D4B03F502711360C3F80852C1
:1023C000196051601A4802F0B7F81A4C206028B31F
:1023D000836823B19B6C13B12A461749984720683C
:1023E00083685B6B53B1984740B1206883689B69F1
:1023F00023B101220DF107019847F5E700230F4AA9
:102400002068138082681C46926A02B1904784F368
:102410001188BFF36F8F002003B030BD4FF0FF3045
:10242000FAE700BF70610120505D0120605D01206E
:10243000F88E0000786101205522000078620120AA
:1024400038B54368044698188028154608D80648C9
:10245000184405F008FA002062682A44626038BD1A
:102460004FF00040FBE700BF7B67012040F60613FA
:102470002DE9F041DFF81481D2B0D8F80000ADF8B2
:102480000C303D4B81885C680378C4F3072201332C
:102490000370002342EA042242800A0242EA112227
:1024A000437082800821009341F2210204F0FBFC7A
:1024B0000123324F41F221022146ADF81000009372
:1024C0000346384604F0EFFC02252D4E40BA33682F
:1024D000ADF81000022103A85B68984704F10A03D5
:1024E0005BBA0DF11201022206A8ADF8123005F018
:1024F000BAF9D8F8001008220DF11A00ADF8125000
:1025000005F0B1F9BDF8120006AB083080B22246E2
:102510003946ADF81200184405F0A5F9BDF81200CF
:1025200006AB204480B22A46ADF8120004A9184434
:1025300005F099F9BDF8123005AA2B449BB2ADF80D
:1025400012300093AD2106AB26A8FEF74DFF05998A
:102550003368ADF8121026A85B6889B298473368D3
:1025600029465B68074898474921074804F0E6FC7C
:1025700052B0BDE8F08100BF344501207B670120E7
:102580007C6101200E8F0000118F0000806101200E
:1025900038B50C4C0C4D4FF0FF322146284605F063
:1025A0001EFD0A49204605F02CF800230022204693
:1025B00005F0F2FC2146284605F022FDBDE8384032
:1025C000FFF754BF9461012084610120198F00003E
:1025D0002DE9FF410C681B4F02380D46C4F5007110
:1025E0000090194B381903AA0131FEF77DFF04460C
:1025F00028BB2B68039A1344022B2B601BD9398804
:10260000023B0E0246EA1126B6B29E4213D14FF0AB
:102610000108034641F221023146CDF80080B81C82
:1026200004F041FC38B9022E05D92B68023B1F4447
:102630002B60BC704446204604B0BDE8F0814FF0EA
:10264000FF34F8E7FB670120FE6901202DE9F04F18
:1026500007290446B5B060D9057815F0FD055CD1B1
:102660004288A1F10806130243EA12239BB2B34247
:1026700053D38288B64BB7491860130243EA12233A
:1026800083802A46B4484D6005F079FCA388012B6D
:1026900040F0EC81E3792BB1012B00F09C80FFF737
:1026A00077FF3AE04FF0FF32AC49AB4805F097FCBA
:1026B000AB49AA4804F0A5FF4FF0FF32A7480AA98A
:1026C00005F08AFC00260027A64DDFF8C082DFF85F
:1026D000C0923146002004F03FF809A9C0B2FFF7CC
:1026E00039FA044658B92023014612AA099804F081
:1026F00040FE129BAB4216D0099804F039FE002F21
:1027000008BF012E0CD10AA9944805F079FC934921
:10271000914805F075FCFFF7A9FE35B0BDE8F08FD4
:1027200001260027D5E740230DF1680A01932146D1
:102730002046CDE90344099B0294CDF800A012AADB
:10274000FDF744FF0028D7D1099804F011FE4FF09F
:10275000FF320EA90AA805F042FC41460EA804F07B
:1027600050FF32463B460EA805F016FC49460EA81F
:1027700004F047FF9DF85C10504604F020FF4FF036
:102780002E0B34AB441C18449DF85D1000F868BC57
:102790000AEB040004F013FF34AB2044441C18443B
:1027A000BDF85E1000F868BC0AEB040004F007FFF7
:1027B00034AB204403440130189903F868BC5044FA
:1027C00004F0FDFE51460EA804F01BFF0EA90AA856
:1027D00005F016FC93E731461AAA04F108000A95A1
:1027E00000F03AFA08B9032638E04FF0FF384FF00E
:1027F00000092A4628462C4646464F46AB46DDF899
:10280000CCC01AAB624552D1002F08BFB6F1FF3FD2
:10281000E9D0BBF1000FE6D0002103F09DFF0AA92B
:10282000C0B2FFF797F90028DDD156EA0703DFF8B9
:1028300048A10BD10A9BCAF800009A6800234245C0
:1028400073EB0903CFDB484BC3F800800023DAF8B1
:102850000010BB4208BFB1423FD00026324649219A
:10286000424804F06BFB4FF0FF323C493A4805F018
:10287000B6FB3F49394804F0C4FE32463748F317E7
:1028800005F08AFB4EB93B49344804F0BAFE3A4B96
:1028900032481A68334605F077FB30492E4805F078
:1028A000AFFBFFF7E3FD0A9804F062FD35E7197C02
:1028B000032904D8DFE801F00206090E9868013206
:1028C00014339FE7D3E902B4F9E7996888464FEAE1
:1028D000E179F4E79E68F717F1E7234B21441A6882
:1028E000984691423FF67FAF0A9804F0AEFDB4FBE4
:1028F000F0F303FB1043DAF80000D8F800200119C8
:10290000914238BFE41A0EA9204428BFDDB2FDF77A
:102910004BFE064620B14521184804F00FFB9DE709
:10292000174B0E9A19681F468A4233D04921154821
:102930001A6004F003FBDDE90E120A9804F05FFD53
:10294000064638B3324645210F4804F0F7FA85E7CA
:1029500080610120344501208461012094610120BF
:102960001C8F00003DB8F396A8610120FB8F00008A
:10297000198F000009900000A4610120308F000031
:102980003C4501205B8F00007E8F0000238F0000FC
:10299000288F0000DAF8002049213F48A31804F0EE
:1029A000CDFA002D49D0661B30D033465A46DAF8AE
:1029B00000100A9804F0FAFC00287FF414AF2C46AB
:1029C000DAF80030B3443344CAF800302A46594696
:1029D00012A804F048FF0A9804F040FD12ABC5F1BC
:1029E00008020146581904F069FF0A9DDAF8001040
:1029F0002846079104F029FD03462846079912AAA4
:102A000004F0D4FC00287FF4EEAE01E0002CDDD110
:102A1000DAF800301C44D8F80030CAF800409C4274
:102A20007FF41BAF0A9803F0A2FF0EA9FDF7BCFDCF
:102A3000064640B1452119486FE723465A46DAF861
:102A400000100A98DCE70E9A3B689A427FF705AFC0
:102A50004921134804F072FADDE90E120A9804F0D5
:102A6000CEFC064600283FF4F9AE6BE7002B7FF45E
:102A700054AEE379012B3FF412AE052B7FF44DAE3B
:102A8000FFF786FD00214FF4005002F019F90120F4
:102A9000FFF79CF841E600BFA18F0000C18F000046
:102AA0005B8F00002DE9F3411B4F002405463E4695
:102AB0001A4BDFF86C8000941860C4F500712B6825
:102AC00001AA0131381998470028019B01DC002B2D
:102AD000F3D004442BB940F201239C42EDD10024F1
:102AE000EBE73378062B09D17378092B0BD1002340
:102AF00000936946A01EFFF76BFD04E0042B02D192
:102B00007378142BF5D00128E9D100994046023999
:102B1000FFF79CFDE3E700BFFC6901207C61012019
:102B2000FD6701202DE9F041076805460C4617B9FD
:102B30000020BDE8F08100231A46D0F8088004F098
:102B400000FE88B1D4E900123E4804F07CFE06463F
:102B500050B90346024604F10801284604F0B7FDC7
:102B600010B126740120E4E7002321461A462846C6
:102B70002F60C5F8088004F0E4FD80B1D4E90012AC
:102B8000314804F060FE034648B9024604F10801EA
:102B9000284604F0D6FD10B101202074C9E70023B7
:102BA00021461A4628462F60C5F8088004F0C9FD62
:102BB00080B1D4E90012254804F045FE034648B927
:102BC000024604F10801284604F081FD10B10223F9
:102BD0002374C7E7002321461A4628462F60C5F80C
:102BE000088004F0AEFD78B1D4E90012184804F072
:102BF0002AFE034640B9024604F10801284604F0C3
:102C000066FD08B10323E3E7002321461A46284660
:102C10002F60C5F8088004F094FD002888D0D4E91E
:102C200000120C4804F00FFE0346002880D1024633
:102C300004F10801284604F084FD00283FF478AF31
:102C40000423C5E78A8C00000D900000129000005C
:102C5000099000001690000070B501258CB0014469
:102C600009AE052309900A91144630462A4607A961
:102C70000B9504F071FD002360B11422CDE90143EE
:102C8000CDE9033205212846044B009604F1640285
:102C900004F080FD00F001000CB070BD252B000099
:102CA000094A0A49936809689867D96708494B68CF
:102CB00043F080534B60002383F31188BFF36F8F81
:102CC0009368D86F704700BF2C6201208C8700008A
:102CD00000ED00E013498A684FF038001044EFF32C
:102CE000098C80E8F01F202080F31188BFF36F8FDC
:102CF0000D4F4FF000664A6A8A603E60906F002375
:102D0000936780F3118802F1380090E8F01F8CF38C
:102D1000098802F1000004B504F069FDBDE8044033
:102D2000704700002C62012004ED00E01EF0040F4B
:102D30000CBFEFF30880EFF30980816911F8021CE2
:102D40000229FFD001B504F056FD01BD43B2002BAE
:102D500008DB012200F01F0002FA00F0024A5B09C2
:102D600042F82300704700BF00E100E0054B420934
:102D700053F82220012300F01F0003FA00F0104056
:102D8000704700BF00E100E043B2002B01F10101F8
:102D9000ACBF03F16043064B4FEA4111C9B2ABBF70
:102DA00003F5614300F00F0083F8001319547047D6
:102DB00014ED00E01FB50025044603910292019333
:102DC000E1EE105A00F0E8FA85F30B88DDE9021015
:102DD0000A4B019AA3F52056202586F30B8883F32E
:102DE000098863B64FF0000383F31188BFF36F8F38
:102DF000A04785F31188BFF36F8FFEE74094012051
:102E0000014910220A60704710ED00E072B64040A0
:102E100080F31188BFF36F8FBFF34F8F30BF62B65F
:102E2000BFF36F8F704700BF72B6494081F31188BE
:102E300020BF80F3118862B6704700BF37B50546E2
:102E40000C46C9B18B6810480093D1E90023452195
:102E500004F074F8636945210093D4E903230B4817
:102E600004F06CF84521E269094804F067F845214F
:102E7000A269084804F062F82146284603B0BDE87C
:102E8000304001F081BB00BF1A9000004E9000005E
:102E9000829000009690000030BFFFF7FDBF00BF9A
:102EA000174A08B5174B22F07F029A60BFF34F8F85
:102EB000BFF36F8FD3F8882022F47002C3F8882004
:102EC000D3F8882042F4A002C3F888200E4A536841
:102ED00023F040435360BFF34F8FBFF36F8F002346
:102EE000E1EE103AEFF3148323F0040383F3148824
:102EF00001F098FB01F010FF00F020FA01F0B4FBA4
:102F00000000000000ED00E030EF00E001B572B617
:102F10000B4A106A00281EBF0021116205F084F8D8
:102F200062B6EFF30580A0F110004FEAC00005493A
:102F3000014409C99847BDE801400349084700001A
:102F40002C620120DC8200001533000004F0EBF954
:102F5000202080F3118808484FF40061401880F366
:102F60000988EFF314800221084380F31488BFF32B
:102F70006F8FFFF795FF000040940120EFF308806A
:102F8000EFF3098101B5724600F008F901BD00BFF9
:102F900070B5224C06460D462148452103F0CEFF70
:102FA000A26AD00603D545211E4803F0C7FFA36AD5
:102FB000190703D545211C4803F0C0FF174CA36A2D
:102FC0009A0710D54521194803F0B8FF626BA36A30
:102FD0001B0608D54521164803F0B0FF1EB1A36AB1
:102FE00023F08003A3620D4CA26AD00703D54521CC
:102FF000104803F0A3FFA36A990603D545210E48A4
:1030000003F09CFF0020054B9A6AD20658BF9A6ACB
:103010009A6A42F0FF029A62287070BD00ED00E0EB
:10302000C9900000E49000001C9100003491000061
:10303000519100006C9100009091000070B5234CFC
:1030400006460D462248452103F078FFA26AD104C6
:1030500003D545211F4803F071FFA36A1A0503D564
:1030600045211D4803F06AFF184CA36A9B0510D543
:103070001A48452103F062FFA26BA36A180408D521
:103080004521174803F05AFF1EB1A36A23F40043F9
:10309000A3620E4CA36A590503D54521114803F0DC
:1030A0004DFFA36ADA050BD545210F4803F046FF13
:1030B0000020064A936A43F47F439362287070BDF0
:1030C000A36A9B04F4D545210848EFE700ED00E032
:1030D000C4910000DF9100001C910000F5910000F8
:1030E000139200002D9200004D920000909100007C
:1030F00038B5214C4521214803F020FFA26A9501F3
:1031000003D545211E4803F019FFA36ADC0103D54E
:1031100045211C4803F012FF174DAC6A14F48014CB
:1031200004D04521184803F009FF0224AB6A1803B4
:1031300003D54521154803F001FF0F4DAA6A51033D
:1031400003D54521124803F0F9FEAB6A9A0303D573
:103150004521104803F0F2FE074DAB6ADB0303D5AF
:1031600045210D4803F0EAFEAB6A20466FEA0343AF
:103170006FEA1343AB6238BD00ED00E06A920000D5
:10318000879200009F920000BE920000ED92000026
:10319000109300003A930000599300002DE9F0438A
:1031A0004A4B0025D3F804908BB0C9F3080885F387
:1031B0001188BFF36F8F02F07F43B3F17F4F07D1C8
:1031C00002F00C03082B05D14521414803F0B6FE5F
:1031D0002F4604E012074EBF0F4607460125002286
:1031E000A8F1030614468DF80720092E5BD8DFE806
:1031F00006F0054F53335A5A5A5A5A574521354803
:1032000003F09CFE314B8DF80740DC6A14F0020499
:1032100005D04521304803F091FE00241FE0DB6A11
:103220005B001CD545212D4803F088FE2C4B1B78F4
:103230002BB101200DF10701FFF7AAFE0EE0294B8B
:103240001B782BB101200DF10701FFF7F7FE05E018
:10325000254B1B889BB213B1FFF74AFF04469DF82C
:10326000073093B92022394602A804F0FCFA099BE2
:1032700035B3C3F3080222B96FEA53236FEA43233D
:103280000993204602A9FFF7D9FD0BB0BDE8F083F2
:1032900000200DF10701CFE700200DF10701D4E771
:1032A00045211248B7E7124919F4F87F114A12482C
:1032B00008BF0A46A8F11003452103F03FFEACE722
:1032C00023F4FF7323F00103DAE700BF00ED00E011
:1032D000B7930000E79300000394000029940000D6
:1032E00028ED00E029ED00E02AED00E04D9400001B
:1032F000899300009E93000088940000044B5A6953
:1033000042F010025A615A6942F480625A61704771
:1033100000ED00E0704700BFBFF34F8F0549064B3B
:10332000CA6802F4E0621343CB60BFF34F8F00BF63
:10333000FDE700BF00ED00E00400FA0500232021B6
:103340000348C2180133412B82F80013F9D17047AA
:1033500000E100E008B50E4B9B68834207D1EFF314
:10336000058393B10B4A536843F08053536001F0D7
:103370009BFB4FF02003EFF3118083F31188BFF321
:103380006F8FBDE8084004F073BE01F0B1FC00BFD0
:103390002C62012000ED00E00121024B024A0348AB
:1033A00000F032B9000004200045012088860000AA
:1033B00010B50B680C7A23F01F0204F01F031A43A8
:1033C000CB68640923F01F03044943EA440343F034
:1033D00001038860CA600B6110BD00BF90ED00E082
:1033E00030B54B680C6885B00A898D7A0094013B32
:1033F00024F01F04234402F01F0242EA451223F086
:103400001F030F2804468DF80820039309D90246AC
:103410004521064803F092FD6FF01504204605B0E3
:1034200030BD6946FFF7C4FFF8E700BFA494000071
:103430002DE9F04F8946144606464FF00008524DDC
:1034400085B0C84523DA7768002F42D01F2F17D9DF
:10345000FB0615D1D6F800A01AF01F0F10D1504668
:1034600004F0D4F9834607EB0A00013804F0CEF9E2
:10347000834510D06FF0150B5A464521434802E0B2
:1034800042464521424803F059FD6FF0150420469D
:1034900005B0BDE8F08F1BF1160FEDD0631E5B4544
:1034A000EADBC5F808B0E968C5F808B02F6921F073
:1034B0001F01D6E900321A44994247F01F0702F172
:1034C000FF3A1CD1574508D131465FFA8BF0FFF720
:1034D00087FF08F101080C36B3E73146C5F808B09C
:1034E000EB6822F01F0203F01F031A43EA60E0B208
:1034F000FFF776FF10F1160FC7D0441CE9E7013B38
:103500005745E0B223F01F03C5F808B006D12A6979
:10351000314602F01F0213432B61E9E7296901F0EC
:103520001F010B432B613146FFF75AFF10F1160FB5
:10353000ABD0C5F808B0EA689DF80830013F62F3E7
:1035400004038DF808302B699DF808205B0863F3AD
:1035500047128DF80820D6E900321344009323F077
:103560001F033B44441CA3EB0A0AE0B22AF01F03EA
:103570000F28039303D902464521064883E769468D
:10358000FFF716FFB9E700BF90ED00E0F7940000E9
:10359000CF940000A49400000522034B5A60BFF3AF
:1035A0004F8FBFF36F8F704790ED00E0BFF35F8FD9
:1035B0000022014B5A60704790ED00E038B50E4C88
:1035C0002568102D14D8FFF7F1FF00200B4B0C4A93
:1035D0001A63854205D10B4B1D70FFF7DDFF0020FC
:1035E00038BD616801EB0011FFF7E2FE0130F0E742
:1035F0004FF0FF30F4E700BF9486000090ED00E04C
:10360000AAFF4400FD6B012010B5034C2278FFF7A0
:103610000FFF207010BD00BFFD6B0120064A00F0B7
:103620001F0002EB8000D0F8003223F4403343EA5D
:103630000141C0F8001270470025845008B5094BBD
:103640001A786AB901210D2019700521FFF79CFB3A
:103650000D20FFF77BFB4FF00042034BC3F8042320
:10366000002008BDFE6B012000D00050F7B50E46CB
:10367000416806F01F05097AB2F5A03FC76845EA20
:1036800041150AD15C4805F01F01803150F8211026
:10369000C80707D56FF0220093E0B2F5005FF96824
:1036A00000F091800121F868B1400143F9600121E7
:1036B0007869B140B2F5A03F0CBF084388437861F8
:1036C0000020BA69B3F5C02F0CBF0A438A43BA6120
:1036D0003A69B3F5802F0CBF114322EA0101474A32
:1036E0003961D2F80433DBB200F5A27152F821102F
:1036F000C1F304218D426BD123FA00F1C90767D5CC
:10370000830003F1A04303F55043D3F8101521F0D3
:103710000101C3F8101501238340C2F80833C0B279
:1037200000F038FE28460021FFF778FFF868F040E7
:1037300010F0010045D07869F04010F001044ED03F
:10374000BB690DF10700F340DB0757BF396903265A
:1037500021FA06F606F001065CBFC6F10206F6B2D3
:1037600000F03AFE264B984236D100209DF8071013
:103770002D028B0003F1A04303F55043D3F810252D
:1037800005F4F85522F4473222F44072C3F81025AC
:10379000D3F8102515438A0002F1A04202F55142E8
:1037A00045EA0646C3F8106510601268D3F8102584
:1037B00042F00102C3F810250123104A8B40C2F8E1
:1037C000043303B0F0BD0120B04021EA00016DE7F1
:1037D0000130082888D1A5E76FF01200F1E73969B8
:1037E0002846F14001F00101C1F10301C9B2FFF720
:1037F00015FF2046E5E700BF0025845000D00050AB
:103800000000AD0B284B70B5466828481340834232
:103810003BD00DD8062B15D005D89BB1022B36D046
:103820006FF0150030E0B3F5801FF9D1012309E0F6
:103830001F4883422DD0B3F5A00F2CD0B3F5800FD5
:10384000EED10223D0064CBF0325C2F3401582F40B
:10385000807412F4007FC2F34020C4F3002406D029
:1038600012F4006F766818D001228A40B26040EAF4
:103870004402002042EA032301F01F010D4A43EAFB
:103880008503803142F8213070BD0723DAE7042335
:10389000D8E70523D6E70323D4E7520542BF012228
:1038A0008A40F260E3E700BF0600F0000600100067
:1038B00002004000002584502DE9F8433F4F3E6848
:1038C000002E4FD04FF001084FF000093C4BDD684F
:1038D000D3E905210A4325EA02053A4A1B6914691E
:1038E0005C4025EA040475BB3D603B68002301256C
:1038F0001F463548D0F8042305FA03F1114211D0D0
:103900009A0002F1A04202F55142116851B103F54B
:10391000A27150F821101760C1F3042105FA01F1DA
:1039200012680C430133082BE4D1ECB94EB10126E7
:103930000027234DEC68D5E905210A4324EA020457
:1039400054BBBDE8F88315EA080F06D0002109F042
:103950001F00FFF763FE25EA080509F101094FEA98
:103960004808C0E73446C1E7154B59680029DDD047
:103970000D68164F002D38BF00258A68224002D0FE
:1039800038464B689847002DD0D02B682946002B2D
:1039900038BF00231D46F0E726420CD0296907F006
:1039A0001F00F94001F00101C1F10301C9B2FFF7A5
:1039B00035FE24EA060401377600C1E77CD10050C9
:1039C000AC6101200025845000D000504446012005
:1039D000024B0B6001231360704700BFC8610120D8
:1039E000004870470487000010B504F05BFA034CF0
:1039F000206004F054FA6060002010BDC86101200E
:103A0000F8B50E46144604F04AFA214605463046FB
:103A100003F0C4FF3746F8B1B6FBF5F305FB1363BB
:103A200023B9B4FBF5F305FB134040B123463246FE
:103A300045210C4803F082FA6FF015000BE0A54217
:103A400009D804F02CFA0546384600F007FD641B3F
:103A50002F44F9D12046F8BD23463246452102487D
:103A6000E8E700BF2E9500005295000037B50C46E0
:103A7000194620460193154603F090FF019B40B97B
:103A800009482246452103F059FA6FF0150003B0AA
:103A900030BD33B11A462146284603F0E4FE00202B
:103AA000F5E71846F3E700BF52950000F8B50E465B
:103AB0001946304617461C4603F070FF40B92346AE
:103AC00032464521124803F039FA6FF01500F8BD6F
:103AD00044EA060515F0030504D023463246452185
:103AE0000C48F0E78CB12B19032BA6EB050006D888
:103AF000094AD2F80034DB07FBD50020E7E77B1B3F
:103B0000196800F0C9FC043DEDE72046DFE700BF7F
:103B1000529500007495000000900350F0B54B7969
:103B2000012B29D0032B24D110268B79032B20D1F4
:103B3000CC7924B1012C1CD143681B79CBB10A7913
:103B400012B1022A15D10E220B684568B3F5164F43
:103B50002D6865D02DD8B3F5165F64D016D8B3F5AF
:103B6000966F62D00AD8B3F5967F61D0B3F5167F11
:103B700061D06FF0220052E00026D6E7B3F5166F51
:103B80005CD0B3F5965FF4D1374B3CE0B3F5E14F31
:103B900057D007D8B3F5615F55D0B3F5964FE8D14C
:103BA000324B30E047F61227BB42E2D14FF400031C
:103BB00029E0B3F5613F48D013D8B3F5963F47D01D
:103BC00009D84DF6C027BB4244D0B3F5614FD0D1E0
:103BD0004FF46B0317E0B3F5E13FCAD14FF0EB733D
:103BE00011E0B3F5612F38D008D8214FBB4237D050
:103BF000B3F5E12FBDD14FF0E86304E01D4FBB42A8
:103C0000B7D14FF08053C5F82435C36834432243FD
:103C1000043303C9C5F86C2583E803000020F0BD18
:103C20004FF41D03EFE7144BEDE74FF49E23EAE753
:103C30004FF4A033E7E74FF41C33E4E74FF41D23C0
:103C4000E1E70E4BDFE70E4BDDE74FF06C73DAE791
:103C50000C4BD8E74FF46503D5E74FF07063D2E71C
:103C60004FF08063CFE700BF00B0130000A04E000C
:103C700090D0030040420F000050270000C07500A4
:103C800000F03A0000903A012DE9F04106468846DE
:103C9000C76804F09AFAB8B9284B1B7883F001037F
:103CA0007268156893B14FF02003EFF3118483F32A
:103CB0001188BFF36F8F304603F043FF38BB84F3A6
:103CC0001188BFF36F8FEEE70123E9E764243046E4
:103CD00003F037FF70B9012004F0D1F8013CF6D1B0
:103CE0000021212000F0ECFFF0E784F31188BFF3FE
:103CF0006F8FF5E74FF02003EFF3118483F3118802
:103D0000BFF36F8F304603F01CFF0028EDD0012376
:103D1000002207F8148FC5F84475C5F84835C5F872
:103D20002021D5F82011C5F85821D5F85821AB60CD
:103D300084F31188BFF36F8FBDE8F0813F6C0120E1
:103D40004FF0000C43682DE9F041C6681C680F462F
:103D5000C4F800C505463060086801213E4B00F0FC
:103D60001F02914099600321803243F822107A6843
:103D7000511C1EBF02F01F01803143F821C0B968F9
:103D8000C4F80C05481C18BF0020C4F814251EBF39
:103D900001F01F02803243F82200F868421C0CD068
:103DA0004FF0010C00F01F020CFA02FCC3F808C02F
:103DB0004FF0030C803243F822C0C4F80805C4F861
:103DC0001015E96828460431FFF7A8FE804678B947
:103DD0006B689B79E3B106F1160000F0BDFA1F4B4A
:103DE000984208D045211E4803F0A8F86FF0040857
:103DF0004046BDE8F081B37D43F00043C4F8A031F4
:103E0000C4F88C300123B27D9340164AC2F80435C1
:103E10000823C4F800357B6801330CD00023C4F8B4
:103E20001031D4F8103106F11503C4F834350123EC
:103E3000C4F8383523606B689B791BB94FF48073E5
:103E4000C4F8043300231436C4F84465C4F8483574
:103E50000123A360E360CBE7002584500000AD0B95
:103E6000A19500000070015030B585B06C46054644
:103E7000084B0FCB84E80F00002201210820FEF739
:103E800083FF0820FEF762FF21462846FFF758FF10
:103E900005B030BD4085000030B585B06C460546A4
:103EA000084B0FCB84E80F00002201210920FEF708
:103EB0006BFF0920FEF74AFF21462846FFF740FF27
:103EC00005B030BD508500000348452108B503F01A
:103ED00035F80020FFF720FADC950000816808B56E
:103EE000044A1023103903F061FA003818BF01208A
:103EF00008BD00BF6887000030B50C46816887B0F8
:103F0000102302AA1039054603F033FA002811DB0A
:103F10001022284602A903F00EFF68B10323237084
:103F2000A968012328460DF10702283903F021FA78
:103F300000280BDA01202AE01022164902A803F01B
:103F400082FC002814BF02230123E8E79DF8073014
:103F5000284603F00F021B096270237101220DF144
:103F6000070103F0E8FE10B96378042B03D901239D
:103F7000637000232371AA682846203AA11C03F02D
:103F80002EFF0028D6D12846E11C03F051FF07B0D0
:103F900030BD00BF688700002DE9F04385B0694659
:103FA000022003F049FF18B1FF2005B0BDE8F083FF
:103FB000062002A903F040FF0028F5D102469DF833
:103FC00000509DF808609DF803709DF80B809DF8E7
:103FD00002901E4C2946207803F0EDFE00B33146D6
:103FE000607803F0E8FED8B1A378042B01D0BB427F
:103FF00016D1E378042B01D0434511D12379042B4A
:104000000CD16379022B16D1114A1248492102F0D2
:1040100095FF6079831E022BC7D9C5E74B45F0D0C9
:104020000132032A04F10604D4D10B48492102F0DD
:1040300085FF0120B9E7032B05D0084A0849042B66
:1040400018BF0A46E1E7074ADFE700BF54960000C1
:10405000109600002C9600003F9600000996000084
:104060001A96000015960000054B1868043B1B6863
:10407000092B03D1431E5842584170470020704716
:104080003401FF0008B54C4B1B68092B01BF4FF0F2
:1040900050230022C3F81421C3F81821FFF7E4FFCE
:1040A00030B10123454A1360A2F63822C2F87835B0
:1040B000414B1B68092B07D1414B1B68012B1EBFCD
:1040C0000122404BC3F87825FFF7CEFF10B10E2236
:1040D0003D4B1A60384B1B68092B04D100223B4B27
:1040E0001A6001225A600022D30003F57F03D3F83F
:1040F0000013013108D0D3F800130132D3F8043390
:10410000B2F5807F0B60EFD1314BDA69D1073BD537
:10411000304B1946D3F80024012AFBD1C3F80425FB
:10412000D1F80034012BFBD1294BDA69D20708D52D
:10413000DA69284922F00102DA61D1F80024012A63
:10414000FBD11A6A01320AD11A6A22F0FF0242F048
:1041500020021A621F4AD2F80034012BFBD1002240
:104160001C4BC3F80425D3F80024012AFBD1BFF36C
:104170004F8F1949194BCA6802F4E0621343CB60B0
:10418000BFF34F8F00BFFDE71B6A0133C0D0124B56
:10419000D3F88C2042F44062C3F88C20D3F88820F6
:1041A00042F47002C3F88820BFF34F8FBFF36F8FC4
:1041B0000B4B0C4A1A6008BD3001FF00384A005012
:1041C0003401FF0000400050E4AE03500C470050A3
:1041D0000080FF000090035000ED00E00400FA05AD
:1041E000984501200090D003044B1A7922B901228E
:1041F00018601A710248704702487047D061012068
:104200000000AD0B0C00AD0B10B1012820D07047A1
:104210004FF05022D2F81834D2F81814C90311D52F
:1042200003F00303022B0DD1C2F8183500220D4B09
:104230001A601B6802224FF05023C3F804230122A6
:104240009A6070474FF050230122C3F81825EDE71C
:104250000022054B1A601B684FF05023C3F804037B
:1042600018607047045100500051005038B510B12B
:10427000012818D038BD4FF050230222012142F20C
:1042800010751C46C3F80823154A10601268154AB9
:104290001160D4F81834DB03ECD5012003F0EFFDF6
:1042A000013DF6D1E6E74FF05024002242F21075AE
:1042B0000D4BC4F808031A601B680C4B1860D4F847
:1042C0000C34D4F80C2403F00103D203D2D5002B14
:1042D000D0D0012003F0D3FD013DF0D1CAE700BFEB
:1042E000045100500C500050005100500450005038
:1042F000164B10B51A6852B1002018601B680122D5
:104300004FF05023C3F80823114B1B689847114BFB
:104310001A688AB100221A601B684FF05023D3F844
:104320001824D3F8181402F00302012A4FF00201F6
:1043300003D1C3F818159A6010BDC3F80813044BD5
:104340000120BDE810401B68184700BF0051005015
:10435000D0610120045100500B4A70B51668F1433A
:1043600089B271B10025ECB221FA04F3DB0705F143
:104370000105F8D50123A3403343047003481360BB
:1043800070BD0348FCE700BFD86101200000AD0B01
:104390000200AD0B012303FA00F010F0FF0F12D062
:1043A0004FF02003EFF3118183F31188BFF36F8F78
:1043B000064AD36C23EA0000D06481F31188BFF36E
:1043C0006F8F034870470348704700BFDC610120CE
:1043D0000000AD0B0400AD0B2DE9F041FF220024DD
:1043E00001260546DFF858E01448DFF85880E3B2AC
:1043F0004FF02001EFF3118C81F31188BFF36F8F21
:1044000022FA03F1C9070AD5DEF84C1006FA03F7C1
:10441000394201BF40463943CEF84C102B708CF323
:104420001188BFF36F8F404505D006FA03F39A4316
:1044300004F10104DBD1BDE8F08100BF0200AD0B47
:10444000DC6101200000AD0B0022034BC3F8842582
:10445000C3F80425704700BF0090035008B5C0F3AF
:104460000B0383B90222094BC3F88425C3F8042542
:104470004FF0FF320260D3F80024D207FBD5FFF7DC
:10448000E3FF034808BD0348FCE700BF009003506A
:104490000000AD0B0A00AD0B0122074BC3F88425C9
:1044A000C3F80425D3F80824D207FBD50160BFF375
:1044B0005F8FFFF7C9BF00BF00900350F8B5104BE6
:1044C000104F53F82050013053F82060AE4200D80E
:1044D000F8BDD5E900342046984770B16CB101238E
:1044E000E41B094A2411610952F8210004F01F0459
:1044F00003FA04F4044342F821400835E6E700BF1C
:10450000788700000446012074460120084BC01A39
:104510000011084B420953F82220012300F01F002C
:1045200003FA00F010420CBF18460020704700BF8D
:104530000446012074460120114970B505460E4617
:10454000104C8C4204D10F4CB4420AD1002414E028
:104550002046FFF7DBFF10B12368AB420DD01034CB
:10456000EFE72046FFF7D2FF08B91034ECE7284602
:10457000216803F05CF90028F7D1204670BD00BF28
:104580007446012004460120F7B505460E464FF05B
:104590002003EFF3118783F31188BFF36F8F00F0CF
:1045A000A1FB0022042D98BF184B044694BF53F87A
:1045B0002530174B009245212A46164802F0BEFCD2
:1045C0003EB1F369C3F308031BB14521124802F061
:1045D000B5FC2CB1204603F002FE08B1037803B904
:1045E0000E480346224645210D4802F0A7FC3146FD
:1045F0002846FFF769FC87F31188BFF36F8F2046C9
:1046000003B0BDE8F040FEF7A5BE00BF90870000F4
:10461000669600007C960000A99600007496000043
:10462000CF9600000248034A0021121A03F046B94F
:10463000C8460120406C0120012208B5084B022029
:104640001A70FFF73BFF03F0CCFD0320FFF736FFA6
:10465000FBF7F2FE034A137B23F00103137308BD3B
:104660003F6C0120C846012008B5144B03F50062D9
:1046700082F3088883F30A880025E023104C84F82D
:104680002230E57725766576A576636A43F4E023E4
:104690006362FEF733FEFEF7B3FB4FF0FF332846AD
:1046A000A362E362FFF70AFF0120FFF707FF2B4633
:1046B0002A4629460348FEF77DFB00BF40940120AF
:1046C00000ED00E03946000070B50E4B0E4CA342E1
:1046D00001D3002070BDD3E9030141EA000212F0CA
:1046E00003020BD19D685A61AA4201D11C33EEE747
:1046F0005E6901320E6059610144F5E76FF0150003
:10470000E8E700BF7846012078460120D3B50C4683
:1047100016461F464FF02003EFF3118183F31188F3
:10472000BFF36F8F43695BB123601B68436183698B
:1047300001338361002081F31188BFF36F8F11E093
:1047400056EA070203D16FF00B002360F3E702463D
:10475000CDE90067044800F05FFA18B9034B9B6885
:104760005B69236002B0D0BD406C01202C62012047
:10477000F8B504460D464FF02003EFF3118683F39E
:104780001188BFF36F8F47696FB903F0F9FC50B11F
:104790002A68C767426103F098FC3146BDE8F840DB
:1047A000074800F0CBB82B6862691A602B68636118
:1047B000A369013BA36186F31188BFF36F8FF8BD36
:1047C000406C01202DE9F341044616461F464FF088
:1047D0002003EFF3118883F31188BFF36F8FC36851
:1047E000324A6BB180689168884219D056EA070353
:1047F00018D188F31188BFF36F8F6FF00F000CE0B2
:10480000916891F90E100133E36093682161A36010
:1048100088F31188BFF36F8F002002B0BDE8F081EC
:104820002169F0E790F90E3091F90E109942A8BF76
:10483000194621EAE1718B422CDD00F0FDF90546B5
:1048400022464146CDE90067194800F0E5F9002805
:10485000E3D04FF02003EFF3118683F31188BFF309
:104860006F8F23682169A34207D033B193F90E30CB
:104870009942A8BF194621EAE171A06890F90E306B
:10488000994209D16DB13146094800F057F86FF0EF
:104890000A00C2E70025D3E700F0CEF90028F2D1E4
:1048A000F0E786F31188BFF36F8FF0E72C620120E9
:1048B000406C012038B583680446002B33D01D4A74
:1048C0009268934232D1C368012B05D0013BC3608B
:1048D00003F0E4FB002038BD4FF02003EFF3118517
:1048E00083F31188BFF36F8F0169806890F90E30F0
:1048F000994201D000F0A0F9204603F041FCA060ED
:1049000058B190F90E2022610022C26703F0DDFB4E
:104910002946094800F012F8DAE7E06085F31188CB
:10492000BFF36F8FD4E76FF01500D4E74FF0FF307F
:10493000D1E700BF2C620120406C012049B9EFF3A0
:10494000058030B9054B5A6A9B689A4201D0FEF740
:10495000A7B981F31188BFF36F8F70472C620120D4
:10496000094B03F12802824205D19B688B4202D198
:104970004B7BDB0606D1D1E9003213605A6000237D
:10498000C1E90033704700BF2C6201200F4A014685
:10499000136910B50BB1D0680DE002F1280003F0E7
:1049A0008AFB9468637B13F0200F1CBF43F008035D
:1049B00063730028EFD039B99368597BC90603D1D6
:1049C0008169002908BF1846506210BD2C62012081
:1049D00070B490F90D20437B002A2CDBDB062AD132
:1049E000836943BB154A114651F8284F8C4218BFC2
:1049F0002346002B38BF0023D46AB3B190F90E6070
:104A000093F90E50AE4203DBA3420ED01B68F4E7CD
:104A10005A68C0E9003210605860437B63F07F033E
:104A2000437370BC0020FFF7B1BFC0E90014D36A24
:104A30001860D062F1E770BC704700BF2C620120A3
:104A400070B50446183003F0CDFB4FF02003EFF3B0
:104A5000118683F31188BFF36F8F94F90D30002B0B
:104A600007DA21460E48FFF77BFF637B03F07F03E5
:104A700063730C4D637BA86843F010036373031BDF
:104A800058425841FFF782FF86F31188BFF36F8FBA
:104A9000AB68A34203D1BDE8704003F0F5BA70BD26
:104AA000546201202C6201202DE9F04104464FF0B0
:104AB0002003EFF3118283F31188BFF36F8F437BE1
:104AC00013F0280F05D082F31188BFF36F8FBDE874
:104AD000F08143F02003437382F31188BFF36F8F9B
:104AE000183003F07FFB4FF02003EFF3118683F3C0
:104AF0001188BFF36F8F637BD80616D1A269A2B964
:104B0000190607D521462248FFF72AFF637B03F0E9
:104B10007F0363731F4B9868021B50425041FFF79D
:104B200035FF002704F130081DE09B07F9D5214629
:104B3000A068FFF715FF637B23F002036373002374
:104B4000A360EEE705F1180003F04CFBA8682946C6
:104B5000FFF706FF6B7B284623F002036B73AF6001
:104B6000EF67FFF735FF256B454501D0002DE9D1F3
:104B7000637B43F008036373236E86F31188BFF3EE
:104B80006F8F002BA3D02046BDE8F041184700BF2F
:104B9000546201202C62012008B590F90D300146C5
:104BA000002B06DA0748FFF7DBFE4B7B03F07F03A1
:104BB0004B73054B9868431A58425841BDE808406A
:104BC000FFF7E4BE546201202C6201202DE9F04180
:104BD000064614461D464FF02003EFF3118783F37A
:104BE0001188BFF36F8F03F0A0FA87F31188BFF32A
:104BF0006F8F6B1C08BFB4F1FF3F08D022462B46D5
:104C000006F118000349BDE8F04100F0E7B8BDE83F
:104C1000F08100BFEB80000010B50C46054811463E
:104C2000DDE902238068FFF7D1FF2046BDE8104090
:104C3000FEF736B82C6201202DE9F04104464FF012
:104C40002003EFF3118883F31188BFF36F8F437B49
:104C50004EB2DB062ED1856965BB184F214607F1A0
:104C60002800FFF77DFEBB6AFA6A834218BF1D4623
:104C7000002D38BF0025A673B5B195F90E10B142CD
:104C800003DCAA4210D02D68F6E76A68C4E9005236
:104C900014606C600120FFF779FE012088F3118811
:104CA000BFF36F8FBDE8F081C4E90002FB6A1C60AE
:104CB000FC62EFE70020A673F0E700BF2C62012042
:104CC000013108BFB0F1FF3F08B506D1044B986829
:104CD000FFF7B6FE4FF0FF3008BD0020FCE700BF35
:104CE0002C620120014B9868704700BF2C620120A4
:104CF00008B54FF02003EFF3118483F31188BFF35D
:104D00006F8F044B98681861FFF79AFE2046FDF7F5
:104D1000C7FF00BF2C62012008B50648064A0749B4
:104D2000121A02F0A0FDBDE80840054A05490648F0
:104D300002F099BD00450120C846012054970000AB
:104D4000000000003C97000000450120034B1B6859
:104D50000BB9FDF7A3B90020704700BF5C620120CA
:104D600030B5036868B10A4A5268904209D043B12D
:104D7000D3E90421D0E90445121945EB0101C3E947
:104D80000421426813605A600023C0E9003330BD3B
:104D90009C450120104B10B51C689C4208BF0024A4
:104DA000FFF7D4FF9CB1D4E90423121A63EBE0733C
:104DB000012A73F100010DDB10466FF00042194625
:104DC0000023824273EB010400DA104610BD6FF03D
:104DD0000040FBE70020F9E79C4501202DE9F74F53
:104DE000019119464B1C08BFB2F1FF3F82466BD0C0
:104DF0006FF001034FF0FF3B541C41F10005B3EB92
:104E000004086BEB0509B8F1000F79F100030FDB23
:104E1000FFF79CFF6FF00103324AD2E9001C5B1AD6
:104E20006BEB0C021E1B62EB0507341A67EBE07597
:104E3000019BCAF808304FF02003EFF3118683F38B
:104E40001188BFF36F8FFFF781FF012C75F100030D
:104E5000BCBF01240025244B24181A6845EBE075DB
:104E60009A42CAE9044501D05F6852B95A68CAF843
:104E70000030CAF804205A68C2F800A0C3F804A0A1
:104E800014E0D2E90489DAE90445444575EB0901E7
:104E90001DDAB8EB040069EB0501C2E904015168B1
:104EA000CAE90021C1F800A0C2F804A01A689A4219
:104EB00006D0924504D1FFF76DFF0021FDF7BCF845
:104EC00086F31188BFF36F8F03B0BDE8F08FB4EBAA
:104ED000080065EB0901BA42CAE90401C6D01268AC
:104EE000C3E700BF484701209C4501202DE9F74F4B
:104EF0004FF02003EFF3118483F31188BFF36F8F1A
:104F0000DFF8ACA0294D5146DFF8A8B02860D5F8ED
:104F100000C0DBF800006246DAE90089D317584583
:104F2000CDE900230DD060B1D0E90467B445BB41A1
:104F30001DDA009BB6EB030C019B67EB0306C0E98F
:104F400004C60026009B2E6013EB0802019B43EB76
:104F50000903C1E90023FFF71DFF3146FDF76CF897
:104F600084F31188BFF36F8F03B0BDE8F08F002288
:104F7000002318EB060849EBE679C0E90423ACEB03
:104F80000606CAE900892E60FFF7EAFE84F311885D
:104F9000BFF36F8F836898474FF02003EFF31184BE
:104FA00083F31188BFF36F8F0149B0E75C62012082
:104FB000484701209C45012038B5064C064DAC42BF
:104FC00001D3002038BD2046D4E9011203F020F9B6
:104FD0001434F4E7784601207846012010B50A4CD5
:104FE00023681BB101230020236010BD00F0AEF840
:104FF0000028F7D00138062803D8044B53F82000C6
:1050000010BD034810BD00BF60620120A4870000EE
:10501000FE8FFFFFBFF34F8F0549064BCA6802F4AE
:10502000E0621343CB60BFF34F8F00BFFDE700BFCB
:1050300000ED00E00400FA054FF0FE33002130B42B
:10504000064A074D074C2B6013602360064A074C45
:10505000EB606368C2F8001530BC18470414845034
:10506000001484500814845000008450A44501208A
:10507000024BD0E90012C3E900127047A445012099
:1050800048B143682BB1BFF35F8F0023036018461C
:105090007047024870476FF4E0407047EA8FFFFFA7
:1050A00010B5044628B1636813B100232360636020
:1050B00010BD024B02485B689847F4E7A445012005
:1050C000C087000010B5044630B10022636822603A
:1050D00043F00103636010BD0148FFF7ADFFF4E743
:1050E000E887000080B1436863B10122D0E8EF3F58
:1050F000C0E8E12F0029F9D1012BF7D0BFF35F8F72
:1051000000207047024870476FF4E040704700BFCE
:10511000EA8FFFFF70B40B4B0668C268D0E90154F8
:10512000C3E90242C3E90065D1E903020E68064BF8
:10513000D1E90154C3E90065C3E902401A6170BCBA
:10514000704700BFB4450120C445012010B500F0F0
:1051500033F820B1032400F067F8204610BD00F0BA
:1051600035F890B900F0B0F890B90F4B1B681B0EE2
:10517000F02B08D10D4A0E4B12689A420AD0072430
:1051800000F01CF8E7E70624FAE70424204610BDE7
:105190000024F5E7012000F097F804460028F7D135
:1051A000044B1860D9E700BF28198450241A845092
:1051B0000000E0200C1A8450002070470020704747
:1051C000014B1860704700BF041A845010B5114895
:1051D00000F048F800B110BD0F4800F043F8002877
:1051E000F9D10E4C204600F03DF80028F3D10C4BCD
:1051F0000C481C6000F036F801460028EBD100F0A6
:105200002DF8044608B1204610BD00F03FF82046B6
:10521000FAE700BFFC450120F0450120F8450120D8
:1052200000460120F445012008B5084800F024F8A4
:10523000074800F021F8074800F01EF8064800F083
:105240001BF8BDE8084000F00BB800BFFC4501208A
:10525000F0450120F8450120F44501200020704769
:10526000704700BF08B5034B02681B681068984779
:10527000002008BDB445012008B5034B02685B68F7
:1052800010689847002008BDB445012070B5094C4E
:10529000094D2069AB68984718B1084B08485B680E
:1052A00098470021074AEB6811602069BDE870400B
:1052B000184700BFC4450120B4450120A445012082
:1052C0000C8800007462012070B51A4D1A4E044615
:1052D000B26828699047F0B95CB1184C2368ABB14B
:1052E000012B1AD0013B23602869F36898470020FE
:1052F00070BD124C216839B90120114B114AC3F815
:1053000000051368002BFCD101312160F368286986
:105310009847002070BD0C4870BD0A4A1368002BE6
:10532000FCD1074A6FF07E40C2F80035FFF748FF16
:105330002368D7E7C4450120B445012074620120E9
:105340000000845010198450E98FFFFF30B10268CB
:10535000034B04489A4208BF002070470248704738
:10536000DD55AABB8208F0007108F00038B50D4683
:105370000446B0B1A0220021043002F06CFF95B1C8
:105380000822294604F1640002F06BFF082205F1AF
:10539000200104F1840002F064FF0020034B23602D
:1053A00038BD0348FCE70348FAE700BFDD55AABB58
:1053B0007108F0008308F0002DE9F74305460E461A
:1053C00099461146FFF7C2FF0446002840F084804A
:1053D000002E00F08580002900F08480B9F1200FB4
:1053E00040F0828005F14404082205F104082046BB
:1053F00002F037FF05F1240708223146404602F04B
:1054000030FF06F120010822384602F02AFF02A9E7
:1054100041F8049D4FF4807002F017FF002865D119
:105420004FF48073324A0121136093600823314A9C
:1054300000F034FB0121052308462F4A00F02EFB23
:105440000823424601211C2000F028FB08233A468D
:105450000121032000F022FB224608230121022023
:1054600000F01CFB0823254A01211A2000F016FB3E
:105470000523234A01211B2000F010FB0823214AA9
:105480000121142000F00AFB08231F4A01211520E6
:1054900000F004FB082305F164020121162000F04E
:1054A000FDFA082305F184020121172000F0F6FA25
:1054B0000823164A01210B2000F0F0FA00F04AFB05
:1054C0000446019800F0D8FA114B002C18BF1C4676
:1054D000A421284602F0C1FE204603B0BDE8F083B7
:1054E0000C4CF9E70C4CF7E70C4CF5E7084CEFE7F0
:1054F000901084506C880000E48800002C88000024
:10550000D088000090880000B08800004C8800001F
:105510008408F0007608F0008008F0008108F000B0
:10552000C2690C4B1A60826943F8042C426943F843
:10553000082C026943F80C2CC26843F8102C8268CE
:1055400043F8142C426843F8182C026843F81C2CCA
:10555000704700BF5C1684500C4B1B68C3610C4B3A
:105560001B6883610B4B1B6843610B4B1B6803611A
:105570000A4B1B68C3600A4B1B688360094B1B689E
:105580004360094B1B680360704700BF5C16845082
:105590005816845054168450501684504C1684501B
:1055A00048168450441684504016845030B1026826
:1055B000034B04489A4208BF0020704702487047D6
:1055C000DD55AABB0202F0000002F00038B5044627
:1055D00068B1051D7021284602F03FFE28462022B2
:1055E000044902F036FE0020034B236038BD034817
:1055F000FCE700BFF8880000DD55AABB0002F00000
:105600002DE9F04385B015466F46274B04460E46FC
:105610000FCB87E80F002DB94FF00009484605B0C1
:10562000BDE8F0832046FFF7C1FF81460028F5D191
:10563000231D0193636AA3BB236F8BB1C3F14008A1
:10564000A84528BFA84604F1300031461844424618
:1056500002F0FFFD236F464443442367A5EB080592
:10566000226F402A06D104F13001384600F0B4FB25
:105670000023236705F03F0835F03F0505D031468C
:105680002A46384600F0A8FB2E44B8F1000FC3D0DC
:105690004246314604F1300002F0DBFDC4F8708070
:1056A000BCE7DFF80890B9E7608500000C02F00065
:1056B0002DE9FF4104466F46134B0E460FCB87E89A
:1056C0000F002046FFF772FF8046B0B9CEB1636A83
:1056D000251D01953BB90123226F636204F130015E
:1056E000384600F079FB2B46043E243453F8042B53
:1056F00012BAA34246F8042FF8D1404604B0BDE8E0
:10570000F081DFF80880F8E7608500000502F0000E
:10571000084B1B681B0EF02B08D1074B1A68074B70
:105720009A4205D10020064B18607047052070474B
:105730000620704728198450241A84500000E02065
:105740000C1A8450002230B5134640F6FC7549000F
:10575000023802F1A15404F5823490424FEA8404E5
:1057600002F10102CABF236025605B181E2AF0D136
:10577000034A13600B445360024B034A1A6030BD66
:10578000781084508410845020F80F001E4B30B5E0
:105790001A4685B0196800910099CC07FAD500F136
:1057A000A15000F582308000016813680193019BCD
:1057B000D807FAD5154B164C186820231F3090FBDC
:1057C000F3F0144D0138002810DA002301304001B5
:1057D00053B14FF00042A0F12001134204D101382F
:1057E00088424FEA5202F8D105B030BD13680393E6
:1057F000039BDB07FAD5431823602B680293029BB7
:10580000002BE3D10138DEE7B4108450AC10845093
:10581000E4108450DC108450F0B51D6885B001F0B0
:105820001F040DB91F2C28D1174D2E462F68019744
:10583000019FFF07FAD500F1A15000F582308000EA
:10584000006835680395039DED07FAD51F2C00EB22
:10585000611018BFC9430D4D18BF01F01F0128602A
:105860000B480068029002981CBF00FA01F1116019
:105870004FF0000108BF1060196010684300C00FAE
:10588000136005B0F0BD00BFB4108450E410845024
:10589000DC1084500C4B890118603F3020F03F0031
:1058A0004030586099600948D9601961596199611F
:1058B0001C3382B0196002680192019AD207FAD5AE
:1058C000196002B0704700BF90108450B41084502B
:1058D00038B5A0F12003B3F5426F05462CD88F28C8
:1058E00026D800F1470300F16604DB064FEA5414A2
:1058F00000D0013464013F34A409013411B1A14244
:105900001AD30C464FF48050E300B0FBF3F020288C
:1059100028BF202002B110600122084B21461A60E6
:10592000FFF710FF28462146FFF7B4FF002038BDDF
:1059300000F11F046409DDE70148F8E71C188450F2
:105940002221F000464BF0B51D4689B01C68019439
:10595000019CE407FAD5434B002413449B001A68CA
:105960000B181E2B88BFC0F11E011F320B185209E5
:105970005343B3F5806F84BF4FF48061B1FBF2F104
:10598000274688BF091ADFF8E4E000F1A150DFF8EC
:10599000E0C000F58230A14233DC2B680493049B05
:1059A000DB07FAD5304B1B68296805910599CF07AD
:1059B000FAD52E4C2E49236000231E46934203F154
:1059C000010040D11946002620F0010228488A42F1
:1059D0003CD8296806910699CE07FAD52549096869
:1059E000286807900798C007FAD5216000210C4667
:1059F0001F488B422DD100201D499A422CD809B056
:105A0000F0BD2B680293029BDB07FAD503199B00BC
:105A10001B682E680396039EF607FAD5CEF8003071
:105A20000023934203F1010306D1164623F001033C
:105A3000B34204D80134AEE7CCF80070F1E7CCF8FB
:105A400000700136F4E70E600346B7E706600131E7
:105A5000BDE704600131CCE708600133CDE700BF4A
:105A6000B4108450240421147C108450D410845029
:105A7000D81084507810845008B540B120280146D1
:105A80004FF0070228BF20210020FFF75BFF002214
:105A9000014B1A6008BD00BF1C188450F0B5294D99
:105AA00085B02C462E680096009EF607FAD500F1C8
:105AB000A15000F5823080000568206801900198AF
:105AC000C707FAD52048214F056002EB8306B24292
:105AD00029D100275A1C1D4E22F001029A4227D8D4
:105AE00023680293029BDE07FAD5194B0B449B00F7
:105AF0001B681F335B099A4213D2216803910399F3
:105B0000C907FAD500211544056008469B1A0F4ABB
:105B10008B4210D800205A1C0C4922F001029A42F4
:105B20000CD805B0F0BD52F804CBC7F800C0CEE7E2
:105B300037600133D2E710600131E9E708600133D3
:105B4000EDE700BFB4108450D4108450D8108450B6
:105B5000240421142DE9F041814BA0B01D68986800
:105B600020331E461A680192019AD707FAD57D4B59
:105B70007D4A1A6032680292029AD407FAD57B4AAB
:105B80001A607B4A1446116803910399C907FAD534
:105B9000784A1168C1F3402137680497049FFF07D2
:105BA000FAD5754F1F6027680597059FFF07FAD53F
:105BB0001768002900F0CF80B90540F1CC8031682A
:105BC00006910699CF07FAD56C49196021680791AB
:105BD0000799C907FAD51168C1F3402137680897BA
:105BE000089FFF07FAD5664F1F6027680997099F2E
:105BF000FF07FAD51268002900F0AF80910540F147
:105C0000AC8032680A920A9AD207FAD5564A1A60CC
:105C100032680B920B9AD707FAD55A4A1A60316844
:105C20000C910C99CC07FAD55749196031680D9140
:105C30000D99C907FAD55549196031680E910E9929
:105C4000CF07FAD55249196031680F910F99CC07E7
:105C5000FAD550491960504B1E4619681091109999
:105C6000C907FAD53F4C4D4B236033681193119B04
:105C7000DB07FAD54A4B236033681293129BDF0788
:105C8000FAD5484B23603A4B9846196813911399FB
:105C9000C907FAD5324F386033681493149BDB0779
:105CA000FAD5226033681593159BD807FAD53E4B79
:105CB000236033681693169BD907FAD53B4B2360B4
:105CC00033681793179BDA07FAD5394B236033688B
:105CD0001893189BDB07FAD5364B2360336819936A
:105CE000199BD807FAD5344B236033681A931A9B53
:105CF000D907FAD5314B236033681B931B9BDA0716
:105D0000FAD52F4B236000F01DFC08BBD8F80030FB
:105D10001C931C9BDB07F9D53D6033681D931D9BCD
:105D2000D907FAD5274B236033681E931E9BDA07E9
:105D3000FAD5254B2360D8F800301F931F9BDB0753
:105D4000F9D50C4B1B6813F4805F204B08BF184635
:105D500020B0BDE8F0811E48FAE71E48F8E700BF12
:105D6000901084508010845000100251C01F72297E
:105D7000B410845088108450C0CF0129C01F0E2950
:105D8000C03F002940010249003184A800001649A3
:105D9000400108A180440888B0108450C044708835
:105DA00080077A41C0077E4100006A498006164993
:105DB00040006E4900020021008220214082202103
:105DC0008082242140A161A100C861510308F10033
:105DD0000108F1000208F100324B2DE9F74F80462F
:105DE0009246994644681A68002AFCD12E4B9B467D
:105DF0001A68002AFCD14FF0FF30019100F094FCAA
:105E0000802000F097FC01230720284A284DA2F5A6
:105E10009E722B60C2F83C011360636A254F264EC8
:105E20003B60A36A20463360D8F8003042F8043C57
:105E3000D8F8083098470199D9F80030002BFBD1E9
:105E4000BAF1000F20D104221C4B1A60D9F800309F
:105E5000002BFBD1DBF800A0BAF1000FFAD1D8F883
:105E60000C30204698473B6863623368A362144B4A
:105E7000C3F800A0C3F844A1D9F80030002BFBD12F
:105E80002B6003B0BDE8F08F236A4020012B04BFD4
:105E90000B4A13600B4B1960C3F804A000F050FCD0
:105EA000D4E700BF10198450201C8450001984507E
:105EB00018188450CC178450D0178450C8178450B9
:105EC00084168450281C8450544B10B5194698B041
:105ED0001A680192019AD207FAD5514B514A1A60B9
:105EE0000A680292029AD407FAD54F4A1A600A68E1
:105EF0000392039AD007FAD54C4818600A680492B6
:105F0000049AD207FAD54A4A1A600A680592059A95
:105F1000D407FAD5474A1A600A680692069AD20749
:105F2000FAD5454A1A600A680792079AD407FAD543
:105F3000424A1A600A680892089AD207FAD5404A7B
:105F40001A600A680992099AD407FAD53D4A1A607C
:105F50000A680A920A9AD207FAD53B4A1A600A6876
:105F60000B920B9AD407FAD5384A1A600A680C9239
:105F70000C9AD207FAD5364A1A600A680D920D9A21
:105F8000D407FAD5334A1A600A680E920E9AD207DD
:105F9000FAD5314A1A600A680F920F9AD407FAD5D7
:105FA0002E4A1A600A681092109AD207FAD52C4A23
:105FB0001A601A4B19461C681194119CE407FAD513
:105FC000174B1860086812901298C407FAD51A6027
:105FD0000A681392139AD007FAD5124A1A600A680F
:105FE0001492149AD207FAD51E4A1A600A681592BA
:105FF000159AD407FAD51C4A1A600A681692169A9E
:10600000D007FAD5194A1A600A681792179AD20768
:10601000FAD5174A1A6018B010BD00BFB0108450EE
:106020008010845000936521000431904096659063
:106030000083612100C3302100C36490008161901E
:1060400000461021008111210041442100C3202974
:106050000C4610C80086312100C3602140C12829A8
:10606000409665210013319040962529594614C861
:1060700040043249494B10B5194694B01A68009251
:10608000009AD207FAD5464B464A1A600A6801922E
:10609000019AD407FAD5444A1A600A680292029A11
:1060A000D007FAD5414818600A680392039AD207CC
:1060B000FAD53F4A1A600A680492049AD407FAD5BE
:1060C0003C4A1A600A680592059AD207FAD53A4AFC
:1060D0001A600A680692069AD407FAD5374A1A60F7
:1060E0000A680792079AD207FAD5354A1A600A68F1
:1060F0000892089AD407FAD5324A1A600A680992B7
:10610000099AD207FAD5304A1A600A680A920A9A9E
:10611000D407FAD52D4A1A600A680B920B9AD20757
:10612000FAD52B4A1A600A680C920C9AD407FAD551
:10613000284A1A600A680D920D9AD207FAD5264AA3
:106140001A600A680E920E9AD407FAD5234A1A608A
:106150000A680F920F9AD207FAD5214A1A600F4B9C
:1061600019461C681094109CE407FAD50C4B186073
:10617000086811901198C407FAD51A600A6812923B
:10618000129AD007FAD5174A1A600A681392139A1E
:10619000D207FAD5144A1A6014B010BDB01084505A
:1061A000801084508090652100040990409665908D
:1061B000808061218020082180206490008161908E
:1061C0000046102100811121004144218020202916
:1061D000024610C80086092180206021402128291C
:1061E0004096652140962529594614C8504B10B554
:1061F0001C4696B01A680192019AD207FAD54D4B07
:106200004D4A1A6022680292029AD207FAD54B4A86
:106210001A604B4A42EA804022680392039AD207EE
:10622000FAD5186022680492049AD007FAD5454A34
:106230001A60A2F5800242EA814122680592059A1D
:10624000D207FAD5196022680692069AD007FAD5C5
:106250003D4A1A6022680792079AD107FAD53B4A4D
:106260001A6022680892089AD207FAD5384A1A604A
:1062700022680992099AD007FAD5364A1A6022682C
:106280000A920A9AD107FAD5334A1A6022680B9209
:106290000B9AD207FAD5314A1A6022680C920C9AEE
:1062A000D007FAD52E4A1A6022680D920D9AD107AE
:1062B000FAD52C4A1A6022680E920E9AD207FAD5A5
:1062C000294A1A6022680F920F9AD007FAD5274AF6
:1062D0001A60216810911099C907FAD51A60144BF9
:1062E0001A46196811911199C807FAD5114B20491E
:1062F0001960116812911299C907FAD51D491960E0
:10630000116813911399CC07FAD50B4919601168DC
:1063100014911499C807FAD5174919601168159195
:106320001599C907FAD5154A1A6016B010BD00BFF5
:10633000B010845080108450400441900086292978
:10634000D81001C8401441904014212940146521FF
:106350000034409000310C90C0400C90C030202997
:1063600040960D9000416090031645C800861121AB
:1063700000416021594644C84014459040142D9076
:10638000264870B5054688B004680094009CE6076E
:10639000FAD5234C23480460234C44EA83432C68F9
:1063A0000194019CE407FAD50360930143EA824219
:1063B00042F0104444F4C0442B680293029BDE0771
:1063C000FAD504602B680393039BDB07FAD5174BC0
:1063D00003608B0143EA814141F0104343F4C04321
:1063E0002E680496049EF607FAD503602B68059381
:1063F000059BDE07FAD5046041F058412B680693EF
:10640000069BDC07FAD5016042F058422B680793DF
:10641000079BDB07FAD5026008B070BDB01084504E
:10642000C0210229801084508071009880611890EA
:10643000354B8EB019461A680092009AD207FAD5E9
:10644000324B334A1A600A680192019AD007FAD592
:10645000304A1A600A680292029AD207FAD52E4A86
:106460001A600A680392039AD007FAD52B4A1A6079
:106470000A680492049AD207FAD5294A1A600A686F
:106480000592059AD007FAD5264A1A600A6806923C
:10649000069AD207FAD5244A1A600A680792079A20
:1064A000D007FAD5214A1A600A680892089AD207DA
:1064B000FAD51F4A1A600A680992099AD007FAD5D4
:1064C0001C4A1A600A680A920A9AD207FAD51A4A2E
:1064D0001A6008680B900B98C007FAD51A600A6812
:1064E0000C920C9AD007FAD5144A1A600A680D92D9
:1064F0000D9AD207FAD5124A0E211A6000200D23F8
:106500000F220EB0FFF73CBFB010845080108450B3
:106510008043012940633921807001298020542162
:1065200000D13490C0403490C0302029C0530D9029
:1065300000413890832308C880E3102100413821AE
:10654000CF4308C801232DE9F04192B0CDE90333D0
:10655000624B1D461A680592059AD207FAD5604B20
:10656000604C2360604B19461A680692069AD7075A
:10657000FAD55E4B1A68D60400F1A8802A68079203
:10658000079AD007FAD55A4A22600A680892089AF0
:10659000D207FAD51E68C6F30036002E40F0988068
:1065A0001220FFF7F3F807461320FFF7EFF88742B2
:1065B0008CBF12201320FFF7E9F8471EFFF738FFC2
:1065C00003AB01AA39461220FFF726F904AB804637
:1065D00002AA39461320FFF71FF900EB48000228F2
:1065E00032D003283ED0012874D12B680993099B2F
:1065F000DB07FAD53F4B23602B680A930A9BD80729
:10660000FAD53D4B23602B680F930F9BD907FAD522
:106610003A4B23602B681093109BDA07FAD5384B5E
:1066200023602B681193119BDB07FAD5354B236050
:10663000013F25D51023192218210020FFF7A0FEC5
:10664000304612B0BDE8F0812B680B930B9BD90745
:10665000FAD52D4B23602B680C930C9BDA07FAD5E7
:106660002A4BCFE72B680D930D9BDB07FAD5284B00
:1066700023602B680E930E9BD807FAD5254BC1E7F4
:1066800003AB01AA39461220FFF7C6F804AB044653
:1066900002AA39461320FFF7BFF810EB440402D1D9
:1066A000FFF712FCC4E7FFF7E5FC022C08D0032C2F
:1066B00009D0012C10D117211620FFF797FDB7E75D
:1066C00015211420F9E70F210E20F6E7124EB7E747
:1066D000124EB5E7124EB3E7124EB1E7B010845038
:1066E00000084A5180108450B4108450881084509F
:1066F00000084E5100065A4940065E4900044241D6
:106700000014424940042E490006524940065649A9
:1067100000063A4940063E490608F1000708F10024
:106720000408F1000508F100014B1860704700BF34
:10673000081A8450014B1860704700BF041A845037
:10674000034A13681842FCD0024A1060184670478A
:10675000001A8450081A845029B1012914BF6FF01F
:106760001500062070470220704770472DE9F74357
:106770000E4617469946044628B94FF0FF38404662
:1067800003B0BDE8F0830029F7D0002AF5D0CB682C
:106790000D8938461D44042329460DEB030200F001
:1067A000E8FD80460028E8D146F60812BDF804103E
:1067B0007389914223D1BDF806109942DDD104239B
:1067C00038460DEB0302294400F0D3FD0028D4D154
:1067D00046F60713BDF804209A42CED19DF8283022
:1067E000BDF80620A3727389C4E900672B44E360F7
:1067F00004351344A4F8089063612561BFE7002BBA
:10680000E6D0BAE72DE9F7430F4690461E46044608
:1068100020B94FF0FF3003B0BDE8F0830368002BD0
:10682000F7D04368002BF4D04FF6FF79D4E9042366
:106830009A4216D223685B8923B1E368934204BF6E
:10684000043323610423216960680DEB030200F027
:1068500090FD0028DDD1A37A256923B1E368AB421E
:1068600001D80120D7E72189BDF80630494503F159
:10687000040203D0BDF804C08C450BD116B1BDF89D
:106880000410318004353D60A8F8003023691344BA
:106890002361C0E715442561C8E773B50C46064679
:1068A00011460223204601AA00F06FFA0546E8B916
:1068B000019A1F2A0ED9A2F1200130462022236816
:1068C000194400F0D0FF2368019A1344236028463E
:1068D00002B070BD0146C2F12002304600F0EEFF6A
:1068E000019A2168C2F120003044EAE76FF0020506
:1068F000EDE72DE9F74306460F4691461D4600F0A9
:10690000A4FD082804461ED8304600F0A7FDAC427E
:1069100038BF2C4680462A464946E4B2684600F015
:10692000A2FF4146621B0DEB050000F0C7FF2346A6
:106930006A463946304600F039FD003818BF01205C
:1069400003B0BDE8F0834FF0FF30F9E700F07BBF04
:106950004FF440735843303070470B7803F0FB031B
:10696000022B14BF4FF0FF304FF44070704710B54A
:10697000044600F06AFD4FF44072A368303B02FB0E
:10698000103010BD012307B5816801AA20398DF8A8
:106990000430FFF7AEFF03B05DF804FB13B5044607
:1069A000019101F005FA0423A0F108010DEB0302A7
:1069B0002046FFF79EFF02B010BDF7B50546002048
:1069C0000C461746FFF7C8FE6946C0B2FBF7C2F88F
:1069D00030B10125009800F0CBFC284603B0F0BD93
:1069E0002C2101FB04542189E3680098CE1804236C
:1069F00031460DEB030200F0BCFC05460028E8D14F
:106A000046F60813BDF8042064899A421AD1BDF8ED
:106A100006309C4201D00325DCE7042300980DEBEF
:106A20000302A11900F0A5FC0028D2D146F60713F5
:106A3000BDF804209A42EED1BDF80610214431443D
:106A40003960C7E7002CF1D0E5E773B51346019232
:106A50000E46024600210546FAF7BAF9044650B937
:106A600001212846019B05F12C02FAF7B1F910B17A
:106A7000002E18BF0446204602B070BD37B54FF453
:106A800080750446426A01A902200195FBF776F859
:106A900048B9019B0620226DA36201A90195FBF76D
:106AA0006DF8054608B1012505E0019B206A636584
:106AB00000F0CBFCE065284603B030BD0123036045
:106AC00003F1012343600023C0E902337047437997
:106AD000012B07D10368012B04D10079431E5842D2
:106AE000584170470020704770B586B006460D4685
:106AF000022003A9FBF72EF830BB0398FFF737FFFE
:106B0000F16D0446284600F0E2F80444039800F0D2
:106B10009CFC0190039800F0A1FC0822014604A807
:106B200000F0CCFE2A7921468DF81020019B0398B5
:106B300004AA00F03BFC041E18BF0124039800F0D7
:106B400017FC204606B070BD0124F7E700F057BCE3
:106B50002DE9F8430E46002107460846FFF7FCFDE5
:106B6000044601210020FFF7F7FD33789C4220D036
:106B7000984220D101242C2303FB0474F86DA56AEC
:106B8000FFF7E6FE00278046013D636A304603EBCF
:106B9000C50253F83510D2F804901B684A46C91A4A
:106BA0004F44FFF7D3FFB84505F1FF35EDD8BDE8F9
:106BB000F8830024DFE70120F9E737B515460C46D6
:106BC0000620694601F038F9E979012903D000224D
:106BD000204601F045F99DF80330012B02D12046F3
:106BE00001F01AF9A9682046FFF7D8FE2046FDF704
:106BF00075F9002003B030BD73B50D460646FAF7AF
:106C0000D3F90446E86030B102282ED101A9FAF781
:106C1000A1FF18B10124204602B070BD2A463146BA
:106C20000198FAF723F90446D8B9019801F0C0F8A1
:106C3000012301460DF10302019800F09AFB04467E
:106C40000028E7D1012201980DF1030101F0C1F8FC
:106C500010B101238DF803309DF8033003F00F03CA
:106C6000EB71019800F084FBD5E70724D3E713B557
:106C7000022001A9FAF76EFF48B90198FFF782FEDA
:106C80000446019800F074FB204602B010BD0124B8
:106C9000FAE71FB5022001A9FAF75CFFA8B901982D
:106CA00002A9FDF729F9044668B99DF80B30032BBA
:106CB00003D1019801F0B0F80446019800F058FBA8
:106CC000204604B010BD0124F7E70124F8E730B5F1
:106CD00043790468012B0ABF01220222002501FB2F
:106CE00002F204F1FF3402FB04F2037918BF0D0233
:106CF000013B01FB0321481930BD036870B5CD1A73
:106D0000002D0DDD93F900601C78002E0BDB5C1C60
:106D100004601B7813600368C91A13688B4232D968
:106D20006FF05F0070BD04F07F04013C032C27D896
:106D3000DFE804F00209121E012DF1D05C78023365
:106D400014600360E7E7022DEADDB3F80140033386
:106D500064BAA4B21460F4E7032DE1DD9C785D7899
:106D6000240244EA0544DD7804332C431460E8E748
:106D7000042DD5DDD3F80140053324BA1460E0E7D3
:106D80006FF06300CEE70020CCE770B404680E1B00
:106D9000002E07DD26789E4208D10134046070BCC5
:106DA000FFF7ABBF6FF05F0070BC70476FF0610022
:106DB000FAE738B5032304461546FFF7E6FF58B94E
:106DC00013685A1E012B2A6004D923685A1C2260BA
:106DD0001B780BB16FF0670038BD2DE9F743904683
:106DE0001F4601AA302305468946FFF7CEFF044619
:106DF000F8B92E68A9EB0609B9F1000F35DD424656
:106E0000019933780E4442F8043B31460623284664
:106E1000FFF7BBFF044660B92A68D8F80410C8F829
:106E200008205318B3422B6007D10C213846FAF7DB
:106E300075FA204603B0BDE8F083515C3A46013351
:106E400042F8041B284631462B60FFF756FF0446E4
:106E50000028EED12B687A68BB601344B3420CBFA4
:106E600004466FF065042B60E3E76FF05F04E0E732
:106E7000F8B5B1F1005F0546144600AF10D26E467A
:106E8000D31D23F00703ADEB030D684600F0EBFCC8
:106E9000694622462846FEF7B3FBB546BD46F8BD17
:106EA000FEF7AEFBFAE72DE9F0419DF8184000250A
:106EB000002C14BF022400244FF0800C6718AF424E
:106EC0001BD81846BDE8F08123465C008D42A4B271
:106ED00008D290F800802CFA06FE18EA0E0F18BFB0
:106EE00044F001041B0406F1010648BF5440082E7B
:106EF000EAD1234601350130E1E70026E5E760B13C
:106F0000436803F00303012B03D0032B05D103686F
:106F10001BB100238360184670476FF0150070475F
:106F200000224368816003F00303032B14BF134660
:106F30000368426018467047002070470FB407B5D9
:106F400004A951F8040B0191FAF776FB03B05DF840
:106F500004EB04B07047038B13F0070305D10368FB
:106F6000002B0CBF002003207047022B05D1438B60
:106F7000002B14BF002004207047012B05D10368AB
:106F8000002B0CBF0020052070470020704773B510
:106F90000D4606461946281D01920093FFF7C0FFD3
:106FA000044640B1DDE9003229463046A44602B02D
:106FB000BDE87040604702B070BD10B44FF02004CF
:106FC000EFF3118284F31188BFF36F8F41615DF895
:106FD000044B0121FAF73EBB10B50C4640B139B164
:106FE000081DFFF78CFF28B9A36833F0030301D015
:106FF0006FF0150010BD38B50C46054658B151B1BB
:107000000B6843B14B6833B11C22002100F056FCE1
:1070100000202C6138BD6FF01500FBE770B5044609
:107020000E46FFF7D9FF051E31DB4FF02003EFF3CB
:10703000118183F31188BFF36F8F4FF6FF75638B58
:10704000208BAB4200F007022ED0022A0ED1013372
:1070500063831546012381F31188BFF36F8FB3B1AA
:10706000002331462046FFF792FF10E0830701D04E
:10707000062A0ED100233360636893B9C4E9006621
:10708000154662B90A4620460221FAF7E3FA284675
:1070900070BD052A0CBF6FF022056FF004050023B8
:1070A000D9E71E606660EBE76FF00A05F7E78368D3
:1070B00000EBC101B3F5004F2CBF51F8220031F8AD
:1070C0001200704700EBC1018068B0F5004F2CBF83
:1070D00041F8223021F812307047012208B5FFF73D
:1070E000E6FF400808BD836800EBC101B3F5004F1F
:1070F00008D34B681AB143F001034B60704723F08B
:107100000103FAE74B881AB143F001034B80704743
:1071100023F00103FAE753000122FFF7D3BF806891
:107120000131B0F5004F2CBF02200120081AB0FA3F
:1071300080F0C0F11F0070472DE9F04104460D4674
:10714000FFF7CBFFA3680146B3F5004F01D3012839
:1071500035D02046FFF7E3FF04EB800216699EB9A5
:10716000012303FA00F0E36829460343E360204665
:1071700015612B460222FFF7A5FF03222946204670
:10718000BDE8F041FFF79EBF022231462046FFF7DF
:107190008EFF07460346022229462046FFF792FF4C
:1071A0003346032229462046FFF78CFF0322394647
:1071B0002B462046FFF786FF02223146DFE7BDE877
:1071C000F081B2F5802FF8B52CBF082504250023E7
:1071D000551B0022CC1D24F007040460C4E90023E1
:1071E00000230D4425F007052D1BED0829462046F8
:1071F000A560E360FFF793FF8600411C18461B362D
:10720000F60804F110028B4229DB324620460021A9
:10721000FFF781FFAF1B204601220021FFF763FF2C
:107220003A463146FFF777FF334631462046002283
:10723000FFF748FF294620460022FFF76CFF3B4638
:10724000294620460022FFF73DFF2946204601221D
:10725000FFF749FF3146BDE8F840FFF76DBF42F840
:10726000040B0133CFE72DE9F04F8BB09B469DF81F
:1072700054300E460393149B92461946002205464D
:107280000024CDE900129DF85880189F0DF11009D7
:107290005046DDE900235946F8F754FFD3B2092BD5
:1072A00084BF2732D3B203F1300209F8012BDDE9A4
:1072B00000239B4508BF924504F1010423D2179B8C
:1072C000A3EB040A2AEAEA7AD346AAEB0B09BBF13C
:1072D000000F01D0039BCBB9A2460AF1FF3A04ABE1
:1072E000314613F80A00A847BAF1000FF5D1DA4683
:1072F000BAF1000F10D13B681C444C445C443C6024
:107300000BB0BDE8F08F82468B46C1E73146404660
:10731000A8470BF1FF3BD8E731464046A8470AF1A2
:10732000FF3AE5E77047FCF7ADBE8368DB681847B6
:10733000FDF702B970B502684C68A24216D38B689B
:1073400023449A4206D2D1E90435AB4204D36FF00C
:107350000B038B6100200AE0CD68121B45F8332037
:10736000426805EBC306013372600B61012070BDFA
:10737000704773B51E46836805468B420C460192E2
:1073800010D371188B420DD3C068FFF7D1FF696825
:1073900021448368019A1C683346A44602B0BDE8C4
:1073A000704060476FF0150002B070BD2DE9F341E9
:1073B0009846836807468B420D4601921CD3414490
:1073C0008B4219D3C068FFF7B3FF06460021FFF7D1
:1073D000ACFF044660B979682944B36830465C68FC
:1073E000019A4346A047044601213046FFF79DFF1E
:1073F000204602B0BDE8F0816FF01504F8E783681D
:107400002DE9F0418B4207460D4690461AD30A44B7
:10741000934217D3C068FFF78BFF06460021FFF7A2
:1074200084FF044658B979682944B3684246304617
:107430009B689847044601213046FFF776FF2046B7
:10744000BDE8F0816FF01504F9E708B5C068FFF7F3
:107450006FFF83681B699847007808BD08B5C0684E
:10746000FFF766FF83681B699847007908BDCBB2B8
:107470000C21C26803FB0121086C00F00700704773
:107480004FF02003EFF3118283F31188BFF36F8F66
:10749000036813F0C00301D08B4207D101230360BE
:1074A000002082F31188BFF36F8F70474FF0FF30D9
:1074B000F7E710B54FF02003EFF3118283F3118843
:1074C000BFF36F8F036803F00704012C06D101603E
:1074D000002082F31188BFF36F8F10BD03F0C0034B
:1074E0008B4214BF4FF0FF306FF04400F1E74FF0D4
:1074F0002003EFF3118283F31188BFF36F8F0368CA
:1075000003F0C00343F00203036082F31188BFF36A
:107510006F8F70476FF02200704710B41C24C06852
:10752000CBB203FB040000215DF8044B10470020A0
:10753000FCF76ABE0020FCF799BE38B50C24C9B22E
:107540004C430546C06804F1400380211844FFF70E
:1075500097FF002804DB69680C44636898470020A3
:1075600038BD2DE9F0410C24C9B24C43C56806462C
:1075700004F140008021284490461F46FFF799FF00
:10758000002806DB2544C5E90E8773681B59984718
:107590000020BDE8F0817047704770470020FAF77F
:1075A00015BB70B506460D460024AC4200DB70BD2D
:1075B000305DFAF7A7FE0130F9D00134F5E7F0B5F8
:1075C00001230A24B1FBF3F2092A06D8024600255A
:1075D0000A2623B91370101AF0BD6343F2E7B1FB1A
:1075E000F3F4B3FBF6FC03FB14171DB9994201D267
:1075F000092B03D8303402F8014B01356346394674
:10760000E7E713B504460846019100F009F9024680
:107610002046019902B0BDE8104000F0CBBCF8B59F
:107620000446036880680D46174610B9013B236085
:10763000F8BD6168994203D8013B23600020F7E759
:1076400013F8016B0021284606F01F06236000F0A6
:1076500035F9172E05D82E70A3680120013BA360D1
:10766000E6E7183EF3B2032B226807D8012303FA9A
:1076700006F6B74203D2013A2260DFE700266168CE
:1076800093199942F7D3721E013D511C236802D110
:107690001E442660E0E79B5C013A05F8013FF4E7F1
:1076A00070B5164604220D461C46FFF7B8FF58B1C8
:1076B0001EB12A6833689A4207D32CB12868236820
:1076C00098428CBF0020012070BD0020FCE7F8B577
:1076D0001D4603680C461B7816463F2B4FEA53178E
:1076E00001D90020F8BD0422FFF799FF0028F8D047
:1076F0002368002BF5DB012F04BFC3F101032360D6
:107700001EB1226833689A42EBDB002DEAD0206874
:107710002B689842CCBF00200120E3E770B50D46EE
:10772000016806460C786409023C012C01D900204E
:1077300070BD291DFFF7B4FF0028F8D033682B6017
:10774000F6E738B504460D46FFF7E8FF18B12368A1
:107750006A681344236038BD73B5CDE9003203680D
:1077600004461E78836876090B60331F012B0D4693
:1077700002D9002002B070BD6B4601AAFFF790FF4E
:107780000028F6D02B68A268052E08BF5B002A608F
:10779000A360EFE72DE9F74F80461646994600248F
:1077A0000F46DDE90C51BC4202D10120346015E0E6
:1077B000DDE90E2328460191D5F800B0D5F808A0E0
:1077C000C847109B0199194458B9444534BF00205B
:1077D00001203460C5F800B0C5F808A003B0BDE8CA
:1077E000F08F0134DFE700210120FBF727BB836E18
:1077F00083F30B88704701460068FBF71FBB08B591
:10780000FBF74AFBBDE80840FBF784BD40E800F009
:10781000C3B210F4803F14BF18466FF015007047D4
:10782000034600201A5C02B970470130FAE70138BC
:10783000013910F8013F11F8012F934201D1002BBB
:10784000F7D1981A704710B55AB10139841810F859
:10785000012B11F8013FA04201D09A42F7D0D01A73
:1078600010BD1046FCE7F0B581EA0004A507034609
:107870000BD0013B0A4491421BD1F0BD002AFCD041
:1078800011F8014B013A03F8014B9C07F6D122F0A5
:1078900003041D1F96080F19B94205D16FF00305A7
:1078A000234405FB0622E4E751F804CB45F804CF56
:1078B000F2E711F8014B03F8014FDCE7034670B51E
:1078C000C9B29C0711D141EA012422F0030644EA1F
:1078D00004451E449408B3420DD16FF0030505FB27
:1078E00004221A44934209D170BD002AFCD003F847
:1078F000011B013AE5E743F8045BECE703F8011BE1
:10790000F0E7436800205B681B690B6070474368C1
:107910005B68586842400A4042405A600020704705
:10792000436800205B6899607047436800205B688B
:10793000D9607047436800205A68536859405160C5
:107940007047C36830B5586858B10024814213D1DC
:1079500008685CB99C685860A14200D1986000201A
:10796000086072B9002030BD2846EFE720609868B3
:10797000814208BF9C60F2E705680446002DF3D100
:107980003AB15A680A60986859600028EAD199604B
:10799000E9E76FF01500E6E70020704738B50446C8
:1079A0000D4600F079FA844209D2002C07DBA84288
:1079B00005D3611981428CBF0020012038BD002011
:1079C000FCE72DE9F3411E4683680C465B69694676
:1079D000174601AA9847DDE9001000231D469E4680
:1079E0009C4600F1FF38B8F1FF3F02D16FF015005F
:1079F00018E00A68CFB1486800FB0255A54208F1BB
:107A0000FF3817DD03B10091009B5B68736077B1AD
:107A1000A4EB0E04B4FBF3F4002004FB03E3644482
:107A20003360B46002B0BDE8F0811544E6E7A4EB32
:107A30000C04F1E74B68944403FB02EE0831012388
:107A4000D1E713460122FFF7BCBF2DE9F047002420
:107A5000836886B0884691465B6902AA01A9984767
:107A6000A2462546029BAB4202D806B0BDE8F0878D
:107A70000026019F07EBC5077B6804933A680AEB71
:107A80000603B24202D89A460135EBE7494603A8FD
:107A900003940593C0470028E7D0049B01361C449B
:107AA000ECE7436810B41B68D3F80423D20518D55B
:107AB000D3F82021AAB14FF02001EFF3118281F316
:107AC0001188BFF36F8FD3F8201131B10021C3F8B3
:107AD0002011D3F820110121D96082F31188BFF35E
:107AE0006F8FC268D2685AB1D3F8581159B10021CA
:107AF000947B11613CB14FF48000C3F8080391738B
:107B00005DF8044B7047D3F8241121B10021C3F86C
:107B10002411D3F824311368002BF1D051685DF89B
:107B2000044B18470B46C268D2E9010183E8030001
:107B30000020704743681B68D3F88004C3F88004B2
:107B4000704742681368D3F8580138B9927932B94E
:107B5000D3F82001003818BF01207047012070477A
:107B60004368C2681B68D3F8100148B10020527DF9
:107B70000A70C3F81001D3F8102101221A6070476F
:107B80004FF0FF307047F8B54368C6681D68F3686A
:107B90009C8910339442A8BF14460122D3E8EF7F9A
:107BA000002F04D1C3E8EC2FBCF1000FF6D10CBFBD
:107BB000134600231CD01C462046F8BDF268CF5C5B
:107BC0009268D7540133A342F8DB4FF02003EFF360
:107BD000118183F31188BFF36F8FFFF7B2FFF36852
:107BE00040B90446186181F31188BFF36F8FE3E752
:107BF0000023E8E79B68C5F844350023C5F84845ED
:107C0000C5F82031D5F82021C5F85831D5F85831BC
:107C10000123AB60E7E743681A68D2F8103153B12B
:107C2000C3680020C2F81001D2F8100101205B7D6A
:107C30000B7010607047184670474368C1681A6837
:107C40004FF02000EFF3118380F31188BFF36F8FA3
:107C50000020C96888734FF48001C2F8041383F3CD
:107C60001188BFF36F8F70470122C368DB689A7376
:107C70007047C368DB689A7B02F0FF0162B9426813
:107C80001268D2F8580140B1D2F8040310F4800011
:107C900003D00120196170470020704743681B68BA
:107CA000D3F81001003818BF012070471022436834
:107CB0001B68C3F804237047102243681B68C3F88D
:107CC000082370474FF4007243681B68C3F804230D
:107CD00070474FF4007243681B68C3F8082370476D
:107CE00001207047C368DB68C3E90012704738B5EC
:107CF000436804461D68D5F804335B0205D4D5F803
:107D0000040310F0100006D138BDFFF7B2FF0028C1
:107D1000F5D00120F8E72046FFF7C0FF003818BF74
:107D20000120F1E708B5FAF7D3F9FAF77DFABDE8D3
:107D30000840FDF753B938B50C461546FFF78EFBE2
:107D400021462544A94201D1012038BD11F8013B4B
:107D50009842F7D00020F8E72DE9F34105460E469A
:107D60009046FFF772FB082804461ED82846FFF706
:107D700075FB012C38BF0124074601224146E4B2BD
:107D80006846FFF770FD3946621E0DF10100FFF7EE
:107D900095FD23466A4631462846FFF707FB003823
:107DA00018BF012002B0BDE8F0814FF0FF30F9E7C5
:107DB000806828387047042809D0052803D1481E58
:107DC00018BF01207047431A58425841704701209C
:107DD000704711B10AB1FFF7AEBF0020704738B548
:107DE0000C460123114622460546FFF7C2FA002839
:107DF00010DB012221462846FFF7EBFF18B10323D1
:107E00000020237038BD2378012B0CBF01230223EF
:107E10002370F7E70120F5E7012307B5816801AA80
:107E200018398DF80430FFF797FF03B05DF804FBB5
:107E30008268183AFFF7D3BF13B50C46C0B201A948
:107E4000F9F788FE50B921460198FCF755F8044629
:107E50000198FFF78DFA204602B010BD0124FAE721
:107E600007B541EA021281688DF8072028390DF123
:107E70000702FFF771FF03B05DF804FB004700F055
:107E8000AAB908B50520FAF771FF20B9BDE8084086
:107E90000520FAF75BBF08BD4FF4801070474FF420
:107EA000805070474FF48070704703681847F0B5F2
:107EB0001D46144687B013BA2ABA6946CDE9002395
:107EC0000646082204A89DF83070FFF7CCFC002D70
:107ED00008BF182C0DF117010BD29DF817303B4449
:107EE0008DF8173006AB30685A1AFFF7DEFF07B07F
:107EF000F0BD002D08BFB4F5807F2CBF0123002307
:107F00000122002D08BFB4F5803F28BF0133012DA9
:107F100008BF002C24BF0133DBB29A403B44891ACE
:107F200018330B70DEE730B484689DF808500134D4
:107F30008460029530BCFFF7BABF7FB50025846826
:107F4000066801340E60846003F02004501C8D60CC
:107F5000CC600ED144F00404CC601F3301223046C3
:107F60000DF10F018DF80F30FFF79FFF002004B0D7
:107F700070BD009308462B46FFF799FFF6E70023F4
:107F80000160C0E90232704707B500210091FFF798
:107F9000CAFF03B05DF804FB07B5D91701F0200153
:107FA00082EAE372009183EAE373FFF7BCFF03B058
:107FB0005DF804FB602330B5154685B00446009398
:107FC00000230391FFF7AFFF2A460399206805B00D
:107FD000BDE83040FFF769BF8023FFF7AEBF10B4A4
:107FE0006FF0004402F10043A34204D3A0235DF8E4
:107FF000044BFFF7A2BF4FF480605DF8044B70475D
:10800000CB6813B50C6813F0040304600AD0FF2397
:10801000012220460DF107018DF80730FFF745FFDB
:1080200002B010BD1846FBE7FFF7B6BA30B5002422
:10803000846141EA020414F00304C0E902320161E0
:108040000CD14461A34203D1C0E90000002030BD3F
:10805000456901340D6041611144F3E76FF015008B
:10806000F5E70023C0E90000C0E902331846704775
:10807000034620B9EFF305820AB9FAF711BE83F37C
:108080001188BFF36F8F70474FF02003EFF311801B
:1080900083F31188BFF36F8FFFF7EABF7047014684
:1080A00008B58068FCF75CFC4B7B23F002034B7344
:1080B00000238B6008BD0368984204D0002B38BFB2
:1080C0000023184670470020704710B54FF020037A
:1080D000EFF3118483F31188BFF36F8FFCF778FC03
:1080E00084F31188BFF36F8F10BD37B504464FF08E
:1080F0002003EFF3118583F31188BFF36F8F54F8DA
:10810000103C18381BB10190FFF7C9FF019814F813
:108110000B3C23F0140304F80B3CFCF759FC85F3EB
:108120001188BFF36F8F03B030BD38B504460D46DC
:10813000FCF732FD637B43F002036373C5B12B6828
:10814000A5609D4208BF0023002B38BF002383B1E8
:1081500094F90E1093F90E20914204DB6A689A425A
:1081600007D01B68F3E75A68C4E9003214605C600A
:1081700038BD6B68256063606B681C606C60F7E7F6
:1081800038B54FF02003EFF3118283F31188BFF36A
:108190006F8FFFF790FF044682F31188BFF36F8F54
:1081A00088B14FF02003EFF3118583F31188BFF3FB
:1081B0006F8FFFF774FF85F31188BFF36F8F04F1A2
:1081C000180000F00FF8204638BDEFF305800038A6
:1081D00018BF0120704708B1F9F79ABC704700201A
:1081E0007047704710B54FF02002EFF3118482F30F
:1081F0001188BFF36F8F03683BB1FCF7B1FD00201E
:1082000084F31188BFF36F8F10BD6FF01500F7E78F
:1082100010B400F10C04C0E903445DF8044BFEF710
:10822000D0BF70472DE9F041069F044615461E4613
:10823000FDF79CF838B93B46324629462046BDE852
:10824000F041FDF7B9B8BDE8F0810A460021FDF71D
:108250003FBBFFF708BBFFF731BB0A460021FFF722
:108260002DBB01EB820204388A4201D10020704705
:1082700052F8043D1BBA40F8043FF5E7F87EFF7F53
:1082800001000000E91A000000000000C9460000DB
:1082900000000000B94F000000000000BD350000E4
:1082A00000000000991C000004460120993E0000D7
:1082B00014460120693E000024460120E51F00000D
:1082C000344601203D36000044460120257D000053
:1082D00054460120E93900006446012000000000F6
:1082E000E777000000000000E777000000000000D2
:1082F000E777000000000000E777000000000000C2
:10830000E7770000F14200007D7E000000000000E1
:10831000E777000000000000E77700002446012016
:10832000A37A000014460120A37A00000000000098
:10833000E777000000000000E77700000000000081
:10834000E777000000000000B938000000000000DE
:10835000E777000000000000E77700000000000061
:10836000E777000000000000E77700000000000051
:10837000E777000000000000E77700000000000041
:10838000E777000000000000951F000000000000DB
:10839000E777000000000000E77700000000000021
:1083A000E777000000000000E77700000000000011
:1083B000E777000000000000E77700000000000001
:1083C000E777000000000000E777000000000000F1
:1083D000E777000000000000E777000000000000E1
:1083E000E777000000000000E777000000000000D1
:1083F000E777000000000000E777000000000000C1
:10840000E777000000000000E777000000000000B0
:10841000E777000000000000E777000000000000A0
:10842000E777000000000000E77700000000000090
:10843000E777000000000000E77700000000000080
:10844000E777000000000000E77700000000000070
:10845000E777000000000000E77700000000000060
:10846000E777000000000000E77700000000000050
:10847000E777000000000000E77700000000000040
:10848000E777000000000000E77700000000000030
:10849000E777000000000000E77700000000000020
:1084A000E777000000000000E77700000000000010
:1084B000E777000000000000E77700000000000000
:1084C000E777000000000000E777000000000000F0
:1084D000E777000000000000E777000000000000E0
:1084E000E77700005E8E000003000000F2950000B8
:1084F000030000009795000003000000208A0000A0
:1085000003000000A0940000030000003697000064
:10851000030000001D8E000003000000FF8E00001D
:1085200003000000198E000003000000CC9500003D
:1085300001000000FFFFFFFFFFFFFFFFFFFFFFFF46
:1085400012000000130000001500000014000000DD
:1085500016000000170000001900000018000000BD
:1085600002000000000000002155000059550000E5
:108570000338FDD8704700001D230000A3750000DC
:1085800001000000F58C00008C8500005B000000FD
:10859000000000000000000000C000003189000061
:1085A0000100000000C0000000020000318900004E
:1085B0000200000000C000000040070031890000F8
:1085C0000300000000C20000003E070031890000E7
:1085D0000400000000C2000000C00000318900005B
:1085E0000500000000820100007E060031890000C5
:1085F000060000000000080000400700318900006C
:108600000700000000400F0000A0000031890000BA
:108610000800000000E00F00002000003189000089
:1086200009000000157500003B750000637500002F
:10863000000000006F740000511D0000B51D000017
:10864000528E00002F75000035750000588E000016
:10865000451C0000FD1B00000000000000000000A1
:108660009D7500006921000021210000D921000032
:10867000DD2000002C450120144501202445012067
:10868000000000001C450120004501200000000002
:1086900006000100020000009C86000000000000AF
:1086A0001F95000002000000E0FF0F00E8440120D9
:1086B0002795000021000000E0FF0320053800009E
:1086C000037900000F790000217900002B79000068
:1086D000357900006D36000043790000000000008D
:1086E000FFFFFFFF00258450000000006D3A0000EE
:1086F000AD3A0000013A000099790000E13900002C
:10870000D139000004000000FF000000617B000080
:10871000893C0000357B00001D3B0000257B0000EC
:10872000877B0000177C00003B7C0000697C000018
:10873000737C0000AD7C0000B97C0000737C0000FD
:108740009D7C0000C57C0000D37C0000EF7C000015
:10875000E17C0000E57C0000008000500600010084
:10876000009000500600010077C295F360D2EF7FC1
:108770003552500F2CB6798084820000BC820000F4
:10878000C4820000DC820000DC820000F5FFFFFFF5
:10879000EC960000FA9600000E9700001D9700006E
:1087A00029970000FF8FFFFFFF8FFFFFFE8FFFFF66
:1087B000FE8FFFFFFD8FFFFFFC8FFFFFFC8FFFFF92
:1087C0006D757465785F667265652063616C6C6554
:1087D000642077697468204E554C4C20706172613A
:1087E0006D6574657200000043616E277420696EC8
:1087F000697469616C697A65206D757465782C207F
:10880000776173204E554C4C0D0A0000436F756C18
:1088100064206E6F74206C6F636B20706F7765726D
:108820002073617665206D7574657800FFFFFFFF2A
:10883000FFFFFFFFFFFFFFFF000000000000000040
:108840000000000001000000FFFFFFFFFCFFFFFF32
:10885000FFFFFFFFFFFFFFFF000000000000000020
:108860000000000001000000FFFFFFFF512563FC36
:10887000C2CAB9F3849E17A7ADFAE6BCFFFFFFFF9B
:10888000FFFFFFFF00000000FFFFFFFF00000000F0
:1088900096C298D84539A1F4A033EB2D817D03779A
:1088A000F240A463E5E6BCF847422CE1F2D1176B35
:1088B000F551BF376840B6CBCE5E316B5733CE2B08
:1088C000169E0F7C4AEBE78E9B7F1AFEE242E34F37
:1088D000FFFFFFFF7F00000080000000000000009D
:1088E00000000000FFFFFFFF7F000000800000008D
:1088F000000000000000000067E6096A85AE67BB63
:1089000072F36E3C3AF54FA57F520E518C68059B71
:10891000ABD9831F19CDE05B25633A205374617294
:1089200074696E6720626F6F746C6F616465720A40
:10893000004E52465F464C4153485F4452565F4E8C
:10894000414D450025633A20466C6173682064659B
:1089500076696365202573206E6F7420666F756E6F
:10896000640A004750494F5F300025633A20456E46
:10897000746572207468652073657269616C207219
:1089800065636F76657279206D6F64650A00256393
:108990003A20556E61626C6520746F2066696E6462
:1089A00020626F6F7461626C6520696D6167650A32
:1089B0000025633A20426F6F746C6F6164657220AA
:1089C000636861696E6C6F61642061646472657371
:1089D00073206F66667365743A20307825780A00D4
:1089E00025633A204A756D70696E6720746F207434
:1089F000686520666972737420696D6167652073AC
:108A00006C6F740A0025633A204E65766572207398
:108A1000686F756C642067657420686572650A000C
:108A20006D6375626F6F740025633A20696E7661BD
:108A30006C696420666C6173682049442025643B3E
:108A40002065787065637465642025640A002A8651
:108A500048CE3D0201002A8648CE3D03010700733F
:108A600065636F6E64617279007072696D617279AD
:108A70000025633A20496D61676520696E2074683E
:108A80006520257320736C6F74206973206E6F747A
:108A90002076616C6964210A0025633A20256420F0
:108AA0007374617475732077726974652066616987
:108AB0006C7320706572666F726D696E6720746882
:108AC0006520737761700A0025633A204661696CFE
:108AD00065642072656164696E6720736563746F95
:108AE00072733B20424F4F545F4D41585F494D4791
:108AF0005F534543544F52533D2564202D20746FDE
:108B00006F20736D616C6C3F0A0025633A204661EB
:108B1000696C65642072656164696E6720696D6166
:108B2000676520686561646572733B20496D6167A4
:108B3000653D25750A0025633A204661696C6564C8
:108B40002072656164696E6720626F6F7420737450
:108B5000617475733B20496D6167653D25750A0039
:108B600025633A2070616E6963210A0025633A200B
:108B7000446574656374656420696E636F6E7369C0
:108B80007374656E7420737461747573210A0025A3
:108B9000633A2043616E6E6F742075706772616412
:108BA000653A206E6F74206120636F6D7061746927
:108BB000626C6520616D6F756E74206F66207365E1
:108BC00063746F72730A0025633A2043616E6E6F9F
:108BD0007420757067726164653A206D6F726520EC
:108BE000736563746F7273207468616E20616C6C5E
:108BF0006F7765640A0025633A2043616E6E6F7477
:108C000020757067726164653A206E6F74207361BD
:108C10006D6520736563746F72206C61796F757414
:108C20000A00676F6F6400756E736574006261643B
:108C3000005072696D61727920696D616765002508
:108C4000633A2025733A206D616769633D25732C73
:108C500020737761705F747970653D307825782C6A
:108C600020636F70795F646F6E653D307825782C76
:108C700020696D6167655F6F6B3D307825780A000C
:108C80005365636F6E6461727920696D6167650019
:108C900025633A20426F6F7420736F757263653A73
:108CA000207072696D61727920736C6F740A00258F
:108CB000633A20426F6F7420736F757263653A2058
:108CC0006E6F6E650A0025633A204E6F7420656EE4
:108CD0006F756768206672656520737061636520D3
:108CE000746F2072756E2073776170207570677273
:108CF0006164650A003059301306072A8648CE3D64
:108D0000020106082A8648CE3D03010703420004FB
:108D10002ACB403CE8FEED5BA44995A1A91DAEE835
:108D2000DBBE1937CD14FB2F245737E5953988D989
:108D300094B9D65AEBD7CDD5308AD6FE48B24A6A16
:108D4000810EE5F07D8B6834CC3A6AFC538EFAC113
:108D50007F7F7F7F7F7F7F7F7F7F7F7F7F7F7F7F23
:108D60007F7F7F7F7F7F7F7F7F7F7F7F7F7F7F7F13
:108D70007F7F7F7F7F7F7F7F7F7F7F3E7F7F7F3F84
:108D80003435363738393A3B3C3D7F7F7F407F7FF3
:108D90007F000102030405060708090A0B0C0D0EEB
:108DA0000F101112131415161718197F7F7F7F7F6C
:108DB0007F1A1B1C1D1E1F20212223242526272845
:108DC000292A2B2C2D2E2F303132337F7F7F7F7F2E
:108DD0004142434445464748494A4B4C4D4E4F500B
:108DE0005152535455565758595A616263646566D7
:108DF0006768696A6B6C6D6E6F707172737475768B
:108E00007778797A303132333435363738392B2F19
:108E1000286E696C2900307800736F6300706F777B
:108E20006572004661696C656420746F20726562CA
:108E30006F6F743A207370696E6E696E6720656E2D
:108E4000646C6573736C792E2E2E0A00434C4F436D
:108E50004B006866636C6B006C66636C6B00636CE4
:108E60006F636B5F636F6E74726F6C007379735FA7
:108E7000636C6F636B006D757465785F696E6974A0
:108E80002063616C6C65642077697468204E554C72
:108E90004C20706172616D6574657200436F756C12
:108EA00064206E6F7420616C6C6F63617465206DFB
:108EB00075746578206265666F726520696E697485
:108EC00069616C697A696E670025633A204E6F7438
:108ED00020656E6F756768206D656D6F727920749F
:108EE0006F2073746F726520696E636F6D696E6752
:108EF0002064617461210A00554152545F3000734F
:108F0000657269616C5F61646170746572000A0DFD
:108F10000025633A2054580A00726300696D616746
:108F2000657300736C6F740076657273696F6E00A1
:108F300025633A20556E61626C6520746F2064650C
:108F40007465726D696E6520666C61736820736507
:108F500063746F722073697A650A0025633A20454D
:108F6000726173696E6720736563746F72206174D8
:108F7000206F666673657420307825780A00256353
:108F80003A204572726F72202564207768696C659B
:108F90002065726173696E6720736563746F720A0E
:108FA0000025633A2057726974696E6720617420E6
:108FB0003078257820756E74696C20307825780AB1
:108FC0000025633A20556E61626C6520746F2064E1
:108FD000657465726D696E6520666C617368207377
:108FE0006563746F72206F6674686520696D616770
:108FF0006520747261696C65720A0025633A2052BB
:10900000583A20307825780A006F666600646174EB
:1090100061006C656E007368610025633A207230F0
:109020002F61313A20203078253038782020723175
:109030002F61323A20203078253038782020723263
:109040002F61333A20203078253038780A002563A4
:109050003A2072332F61343A202030782530387826
:10906000207231322F69703A2020307825303878DC
:10907000207231342F6C723A2020307825303878C5
:109080000A0025633A2020787073723A20203078E5
:10909000253038780A0025633A204661756C74697A
:1090A0006E6720696E737472756374696F6E206188
:1090B00064647265737320287231352F7063293AA6
:1090C000203078253038780A0025633A202A2A2A69
:1090D0002A2A204D5055204641554C54202A2A2AF0
:1090E0002A2A0A0025633A202020537461636B69A1
:1090F0006E67206572726F722028636F6E74657878
:10910000742061726561206D6967687420626520F2
:109110006E6F742076616C6964290A0025633A20B9
:109120002020556E737461636B696E67206572727F
:109130006F720A0025633A20202044617461204147
:1091400063636573732056696F6C6174696F6E0A2F
:109150000025633A2020204D4D4641522041646451
:10916000726573733A20307825780A0025633A20B7
:109170002020496E737472756374696F6E20416349
:10918000636573732056696F6C6174696F6E0A0052
:1091900025633A202020466C6F6174696E672D70DC
:1091A0006F696E74206C617A7920737461746520C4
:1091B000707265736572766174696F6E2065727224
:1091C0006F720A0025633A202A2A2A2A2A20425549
:1091D00053204641554C54202A2A2A2A2A0A00257F
:1091E000633A202020537461636B696E6720657257
:1091F000726F720A0025633A2020205072656369FD
:109200007365206461746120627573206572726F8A
:10921000720A0025633A20202042464152204164D0
:1092200064726573733A20307825780A0025633AB2
:10923000202020496D7072656369736520646174D4
:109240006120627573206572726F720A0025633A3D
:10925000202020496E737472756374696F6E20628A
:109260007573206572726F720A0025633A202A2A8C
:109270002A2A2A205553414745204641554C54201F
:109280002A2A2A2A2A0A0025633A202020446976BD
:109290006973696F6E206279207A65726F0A0025A2
:1092A000633A202020556E616C69676E6564206D9D
:1092B000656D6F7279206163636573730A0025635E
:1092C0003A202020537461636B206F766572666C60
:1092D0006F772028636F6E746578742061726561A2
:1092E000206E6F742076616C6964290A0025633AE8
:1092F0002020204E6F20636F70726F636573736FF1
:109300007220696E737472756374696F6E730A008C
:1093100025633A202020496C6C6567616C206C6F76
:109320006164206F66204558435F52455455524E44
:1093300020696E746F2050430A0025633A20202074
:10934000496C6C6567616C20757365206F6620746D
:10935000686520455053520A0025633A2020204179
:109360007474656D707420746F20657865637574AE
:109370006520756E646566696E656420696E7374D8
:1093800072756374696F6E0A0052657365727665F3
:109390006420457863657074696F6E20280053708F
:1093A0007572696F757320696E7465727275707409
:1093B0002028495251200025633A20535053454CF0
:1093C00020696E20746872656164206D6F64652029
:1093D000646F6573206E6F7420696E646963617475
:1093E00065205053500A0025633A202A2A2A2A2A47
:1093F0002048415244204641554C54202A2A2A2ACA
:109400002A0A0025633A2020204275732066617580
:109410006C74206F6E20766563746F722074616265
:109420006C6520726561640A0025633A202020463D
:1094300061756C7420657363616C6174696F6E2013
:10944000287365652062656C6F77290A0025633A89
:10945000202A2A2A2A2A204465627567206D6F6EA9
:1094600069746F7220657863657074696F6E202807
:109470006E6F7420696D706C656D656E74656429BE
:10948000202A2A2A2A2A0A0025633A202A2A2A2A56
:109490002A20257320256429202A2A2A2A2A0A001C
:1094A0006D70750025633A204661696C65642074AF
:1094B0006F20616C6C6F63617465206E6577204D01
:1094C000505520726567696F6E2025750A0A002560
:1094D000633A20506172746974696F6E2025753A21
:1094E0002073616E69747920636865636B206661BF
:1094F000696C65642E0A0025633A20496E76616CBA
:10950000696420756E6465726C79696E6720726536
:1095100067696F6E20696E6465782025750A00465C
:109520004C4153485F30005352414D5F300025633A
:109530003A20756E616C69676E656420616464725F
:109540006573733A2030782530386C783A257A750F
:109550000A0025633A20696E76616C696420616453
:1095600064726573733A2030782530386C783A2508
:109570007A750A0025633A206E6F7420776F7264E3
:109580002D616C69676E65643A2030782530386CDF
:10959000783A257A750A00666C6173685F6E726648
:1095A0000025633A204661696C656420746F206110
:1095B0006C6C6F6361746520505049204368616E24
:1095C0006E656C0A00554152545F310075617274CA
:1095D0005F6E7266785F75617274650025633A200C
:1095E000526573657474696E672073797374656D01
:1095F0000A00666174616C5F6572726F7200485731
:109600005F43433358585F3000726576657274006B
:1096100074657374007065726D004255473B20633A
:10962000616E27742068617070656E0025633A2052
:109630005377617020747970653A2025730A00258C
:10964000633A205377617020747970653A206E6FA9
:109650006E650A000401040304020401040104030A
:10966000010303040104556E6B6E6F776E20657203
:10967000726F7200756E6B6E6F776E0025633A20A5
:109680003E3E3E205A455048595220464154414C96
:10969000204552524F522025643A202573206F6E88
:1096A000204350552025640A0025633A2046617501
:1096B0006C7420647572696E6720696E746572726D
:1096C0007570742068616E646C696E670A0A0025A3
:1096D000633A2043757272656E74207468726561B6
:1096E000643A20257020282573290A00435055200C
:1096F000657863657074696F6E00556E68616E643D
:109700006C656420696E7465727275707400537450
:1097100061636B206F766572666C6F77004B657264
:109720006E656C206F6F7073004B65726E656C2098
:1097300070616E6963006F7300000000FFFFFFFF40
:10974000FFFFFFFFFFFFFFFFFFFFFFFFFFFFFFFF29
:10975000FFFFFFFFFFFFFFFFFFFFFFFFBD780000E0
:10976000396F00009085000078460120010000005C
:109770008C46012001000000A046012001000000ED
:10978000B446012001000000412400000000000058
:10979000FFFFFFFF0000000000000000FF6B012042
:1097A0002000000000000000000000000000000099
:1097B0001F6C0120200000000000000000000000DD
:1097C00000C201000001030040450120000000002C
:1097D000000000000000000040420F0000010300F4
:1097E0005445012000000000000000000090D0035C
:1097F0009C4501209C450120000000001550000000
:109800006462012001000000C5500000A15000006A
:10981000E550000081500000E8450120AC450120E2
:10982000E045012000000000D845012068620120C9
:10983000010000006C620120010000007062012044
:1098400001000000C8450120D4450120CC4501207D
:10985000C4450120F84501204C8E000038860000E8
:1098600024860000CC570120C595000060870000C9
:109870000C87000080450120F88E0000588700000A
:109880000C870000684501206C8E0000000000007D
:10989000000000000000000063890000E086000076
:1098A000BC860000AC610120FE95000000000000B5
:1098B00000000000000000003189000000000000EE
:1098C000EC86000000000000000000007846012047
:1098D000784601200000000000000000FFFFFFFFAD
:1098E0008C4601208C460120000000000000000092
:1098F000FFFFFFFFA0460120A0460120000000005E
:1099000000000000FFFFFFFFB4460120B446012025
:0C9910000000000000000000FFFFFFFF4F
:10C000003DB8F396000000000002000048EB03007A
:10C010000000000000000000000000000000000020
:10C02000FFFFFFFFFFFFFFFFFFFFFFFFFFFFFFFF20
:10C03000FFFFFFFFFFFFFFFFFFFFFFFFFFFFFFFF10
:10C04000FFFFFFFFFFFFFFFFFFFFFFFFFFFFFFFF00
:10C05000FFFFFFFFFFFFFFFFFFFFFFFFFFFFFFFFF0
:10C06000FFFFFFFFFFFFFFFFFFFFFFFFFFFFFFFFE0
:10C07000FFFFFFFFFFFFFFFFFFFFFFFFFFFFFFFFD0
:10C08000FFFFFFFFFFFFFFFFFFFFFFFFFFFFFFFFC0
:10C09000FFFFFFFFFFFFFFFFFFFFFFFFFFFFFFFFB0
:10C0A000FFFFFFFFFFFFFFFFFFFFFFFFFFFFFFFFA0
:10C0B000FFFFFFFFFFFFFFFFFFFFFFFFFFFFFFFF90
:10C0C000FFFFFFFFFFFFFFFFFFFFFFFFFFFFFFFF80
:10C0D000FFFFFFFFFFFFFFFFFFFFFFFFFFFFFFFF70
:10C0E000FFFFFFFFFFFFFFFFFFFFFFFFFFFFFFFF60
:10C0F000FFFFFFFFFFFFFFFFFFFFFFFFFFFFFFFF50
:10C10000FFFFFFFFFFFFFFFFFFFFFFFFFFFFFFFF3F
:10C11000FFFFFFFFFFFFFFFFFFFFFFFFFFFFFFFF2F
:10C12000FFFFFFFFFFFFFFFFFFFFFFFFFFFFFFFF1F
:10C13000FFFFFFFFFFFFFFFFFFFFFFFFFFFFFFFF0F
:10C14000FFFFFFFFFFFFFFFFFFFFFFFFFFFFFFFFFF
:10C15000FFFFFFFFFFFFFFFFFFFFFFFFFFFFFFFFEF
:10C16000FFFFFFFFFFFFFFFFFFFFFFFFFFFFFFFFDF
:10C17000FFFFFFFFFFFFFFFFFFFFFFFFFFFFFFFFCF
:10C18000FFFFFFFFFFFFFFFFFFFFFFFFFFFFFFFFBF
:10C19000FFFFFFFFFFFFFFFFFFFFFFFFFFFFFFFFAF
:10C1A000FFFFFFFFFFFFFFFFFFFFFFFFFFFFFFFF9F
:10C1B000FFFFFFFFFFFFFFFFFFFFFFFFFFFFFFFF8F
:10C1C000FFFFFFFFFFFFFFFFFFFFFFFFFFFFFFFF7F
:10C1D000FFFFFFFFFFFFFFFFFFFFFFFFFFFFFFFF6F
:10C1E000FFFFFFFFFFFFFFFFFFFFFFFFFFFFFFFF5F
:10C1F000FFFFFFFFFFFFFFFFFFFFFFFFFFFFFFFF4F
:10C20000B018002015E600001920010075E60000B6
:10C2100075E6000075E6000075E6000075E60000B2
:10C2200000000000000000000000000029E4000001
:10C2300075E6000000000000D1E30000E71D0100EA
:10C24000D5E50000D5E50000D5E50000D5E5000006
:10C25000D5E50000D5E50000D5E50000D5E50000F6
:10C26000D5E50000D5E50000D5E50000D5E50000E6
:10C27000D5E50000D5E50000D5E50000D5E50000D6
:10C28000D5E50000D5E50000D5E50000D5E50000C6
:10C29000D5E50000D5E50000D5E50000D5E50000B6
:10C2A000D5E50000D5E50000D5E50000D5E50000A6
:10C2B000D5E50000D5E50000D5E50000D5E5000096
:10C2C000D5E50000D5E50000D5E50000D5E5000086
:10C2D000D5E50000D5E50000D5E50000D5E5000076
:10C2E000D5E50000D5E50000D5E50000D5E5000066
:10C2F000D5E50000D5E50000D5E50000D5E5000056
:10C30000D5E50000D5E50000D5E50000D5E5000045
:10C31000D5E50000D5E50000D5E50000D5E5000035
:10C32000D5E50000D5E50000D5E50000D5E5000025
:10C33000D5E50000D5E50000D5E50000D5E5000015
:10C34000D5E5000000000000000000000000000033
:10C3500000000000000000000000000000000000DD
:10C3600000000000000000000000000000000000CD
:10C3700000000000000000000000000000000000BD
:10C3800000000000000000000000000000000000AD
:10C39000000000000000000000000000000000009D
:10C3A000000000000000000000000000000000008D
:10C3B000000000000000000000000000000000007D
:10C3C000000000000000000000000000000000006D
:10C3D000000000000000000000000000000000005D
:10C3E000000000000000000000000000000000004D
:10C3F000000000000000000000000000000000003D
:10C40000DEE61E284CBBCE8F025B00003C00000025
:10C4100000BE00000100000000C2000000C20000D9
:10C42000FFFF02910000000000000000000000007B
:10C4300000000000000000000000000053B94AB9ED
:10C44000002908BF00281CBF4FF0FF314FF0FF301C
:10C4500000F06CB9ADF1080C6DE904CE00F006F8FF
:10C46000DDF804E0DDE9022304B070472DE9F04770
:10C47000089D04468846002B7DD18A4217463FD945
:10C48000B2FA82F242B1C2F120009140974024FA00
:10C4900000F0944040EA01084FEA174C230C1FFAC1
:10C4A00087FEB8FBFCF60CFB168106FB0EF043EA98
:10C4B0000143984205D9FB1802D2984200F2248128
:10C4C000013E191AA3B2B1FBFCF00CFB101100FBEA
:10C4D0000EFE43EA0144A64505D93C1902D2A64501
:10C4E00000F20F81013840EA0640A4EB0E0400265A
:10C4F0001DB1D4400023C5E900433146BDE8F087B3
:10C5000002B9FFDEB2FA82F2002A50D1CB1B4FEA09
:10C51000174E1FFA87F80126210CB3FBFEFC0EFB19
:10C520001C300B4608FB0CF941EA004189450AD949
:10C5300079182CBF01230023894502D9002B00F074
:10C54000D9800CF1FF3CA1EB0901A3B2B1FBFEF0D5
:10C550000EFB101108FB00F843EA0144A04505D981
:10C560003C1902D2A04500F2C9800138A4EB0804AE
:10C5700040EA0C40BCE78B4209D9002D00F0B180A5
:10C580000026C5E9000130463146BDE8F087B3FA20
:10C5900083F6002E46D18B42C0F0A680824240F244
:10C5A000A3803046002DA8D0C5E90048A5E79740F4
:10C5B000C2F1200301FA02F04FEA174ED94024FAE3
:10C5C00003F31FFA87F894400343B1FBFEF01E0CFF
:10C5D0000EFB101100FB08FC46EA01418C4509D90D
:10C5E00079182CBF012600268C4502D9002E00F0B8
:10C5F00093800138A1EB0C019BB2B1FBFEF60EFB60
:10C60000161106FB08FC43EA01418C4505D979184F
:10C6100002D28C4500F28780013EA1EB0C0346EA72
:10C62000004679E7C6F1200703FA06F402FA06FC91
:10C6300001FA06FEFA4020FA07F8F94000FA06F37C
:10C64000224348EA0E044FEA12484FEA144E1FFAFA
:10C6500082F9B1FBF8FA08FB1A110AFB09F04EEA5D
:10C66000014E70450AD912EB0E0E2CBF012100219C
:10C67000704501D9002952D00AF1FF3AAEEB000E05
:10C68000A4B2BEFBF8F008FB10EE00FB09F944EA87
:10C690000E4EF14505D912EB0E0E01D2F14538D8F8
:10C6A000013840EA0A40AEEB090EA0FB0C89CE45EA
:10C6B00041464C4602D306D1434504D20138B8EB7B
:10C6C0000C0169EB020415B35A1A6EEB040EF2402A
:10C6D0000EFA07F72EFA06F300261743C5E9007392
:10C6E0000BE72E46284608E7841A61EB0301012078
:10C6F000884657E7ACF1020C394424E702383C4441
:10C7000034E702383C44EEE6023E3B44D9E62E468E
:10C71000F3E602389644C4E7023839446AE7AAF1DE
:10C72000020A9644AAE7023E394476E7704700BF02
:10C730002DE9E04F2746A046A146A246A346A446BF
:10C740002DED108B4FF0000545EC185B45EC195AA8
:10C7500045EC1A5A45EC1B5A45EC1C5A45EC1D5A3F
:10C7600045EC1E5A45EC1F5AF1EE105A4FF6607612
:10C77000C0F6FF763540E1EE105A84F30088254676
:10C780002646A447BDEC108BBDE8E08F0B68013353
:10C790000B60014B1B6818470000002007B50B46D3
:10C7A000002102460191034801A900F0EDF803B011
:10C7B0005DF804FB8DC700002DE9F74FB0F8189025
:10C7C000044619F0080893460ED001290CBF49F021
:10C7D000100949F02009A0F818908BF31188BFF3D5
:10C7E0006F8F03B0BDE8F08FDFF898A109F007095B
:10C7F000022907D1204605F032F80028EDD00128A3
:10C80000238B4DD16769218B002F15DA256821F024
:10C810000701C4E9008841F0010121830026218B32
:10C8200001F007024A4502D0A368002B59D10DB987
:10C83000002E71D0002355E001F007035A1F012A92
:10C840001FD821F00701062B256889B2C4E90088AA
:10C850000CD1002D2B4638BF00232BB1628B1B68F7
:10C8600001326283002BF8D141F00201204621837E
:10C8700004F0F5FF0028D1D0238B43F0200323835D
:10C88000CCE7042B0AD121F0070189B2204621838D
:10C8900004F0E5FF10B141F0200121830025BDE740
:10C8A000032809D1226923F00703166843F0060321
:10C8B000002523832F46B2E7042806D1226923F0FE
:10C8C0000703566843F00403F2E7052806D12269FE
:10C8D00023F00703966843F00503E9E700252E4699
:10C8E000E8E7012341F0080121838BF31188BFF3AE
:10C8F0006F8F03BB002D34D116B151462046B0478F
:10C900004FF02003EFF3118B83F31188BFF36F8F88
:10C91000238B23F008032383238BDA062AD50121F6
:10C9200023F010032383B4F8189009F007090029B5
:10C930007FF45EAF51E7A1680029DBD00B68002BC4
:10C9400038BF0023994620463B46D1F804B00192F7
:10C95000D847019AB9F1000FCCD04946D9F8003038
:10C96000EDE729463B46204601922D6804F093FFEF
:10C97000019ABFE713F020011EBF23F0200302211C
:10C980002383D0E7C31801002DE9F04F8846914674
:10C990001C460025A5B0039099F8000010B9284660
:10C9A00000F018BE09F101032528099307D041467C
:10C9B000039B98470028C0F20D86013545E21822F6
:10C9C000002116A805F0C9FB99F80130252B79D074
:10C9D000002216469646174694460998014610F8D6
:10C9E000013B2B2B00F09E8000F29580202B00F065
:10C9F0009B80232B00F09B80BCF1000F05D09DF89D
:10CA0000600040F004008DF860002FB19DF86000D8
:10CA100040F008008DF86000BEF1000F05D09DF8D1
:10CA2000600040F010008DF860002EB19DF86000AD
:10CA300040F020008DF860002AB19DF8602042F09F
:10CA400040028DF860209DF8602002F044004428E8
:10CA500003D16FF386128DF860209DF860202A2B99
:10CA600042F080028DF860207CD19DF861204B1C43
:10CA700042F001028DF861201A782E2A0CBF0121A4
:10CA800000219DF8612061F341028DF8612075D18C
:10CA90005A782A2A6BD000210A260133184610F84A
:10CAA000012BA2F13007092F40F2AA809DF86020E7
:10CAB0001A91C2F3400040EAD17161F341028DF84E
:10CAC00060205BE009F1020209928DF863309DF865
:10CAD0006130DE0740F16F8154F8042B002A089280
:10CAE00008DA9DF8602042F004028DF86020089A70
:10CAF00052420892580740F1668154F8047B002F97
:10CB000080F265819DF861306FF341038DF86130EB
:10CB10004FF0FF375BE12D2B0BD0302B7FF46CAF48
:10CB200001225BE7012759E74FF0010E56E7012686
:10CB300054E74FF0010C51E733460CFB0202303A48
:10CB40001E4616F8010BA0F13007092FF4D99942BF
:10CB500092D09DF860101992D20F62F341018DF8C6
:10CB6000601089E70B4600224FF00A0CE8E79DF8B9
:10CB70006120023342F004028DF86120194611F859
:10CB8000012B6C2A5CD040D8682A46D06A2A61D032
:10CB90004C2A67D019460B4613F8012B782A0993C3
:10CBA0008DF8632000F2DF80572A68D8412A04D02C
:10CBB000A2F14503022B00F2D68004219DF86230D9
:10CBC00002F0DF02A2F1410A61F30203DAF100028E
:10CBD0009DF8611042EB0A0262F3C7110A068DF854
:10CBE00062308DF86110CBB200F1E38003F078027F
:10CBF000182A40F0B5806FF3C6038DF861309CE0D1
:10CC000006FB01210346303948E7742A26D07A2AE8
:10CC1000C0D106229DF861300DE05A78682A9DF84F
:10CC2000612006D1012161F3C6028DF86120991CB3
:10CC3000B1E71346022262F3C6038DF86130AAE71A
:10CC40005A786C2A9DF8612001D10421EBE7134644
:10CC50000322F0E705229DF86130ECE707229DF8FA
:10CC60006130E8E7BDF8603023F4F04323F00203BD
:10CC700043F4804343F00203ADF860308BE7A2F148
:10CC80005803202B6FD801A151F823F03FCD0000AD
:10CC900067CD000067CD000067CD000067CD0000C4
:10CCA00067CD000067CD000067CD000067CD0000B4
:10CCB000BBCB000067CD00003FCD000011CD0000D0
:10CCC000BBCB0000BBCB0000BBCB000067CD00009E
:10CCD00011CD000067CD000067CD000067CD0000DA
:10CCE00067CD000075CD00003FCD000095CD000060
:10CCF00067CD000067CD000095CD000067CD000036
:10CD00003FCD000067CD000067CD00003FCD0000A3
:10CD100001219DF8623061F302038DF862309DF8C5
:10CD2000613003F07803402B02BF9DF8601041F0A2
:10CD300001018DF86010632A05D0002306E002216E
:10CD40009DF86230E7E7003B18BF01239DF86020A3
:10CD5000C2F340010B4363F341028DF86020B6E655
:10CD600013F0380FE9D09DF8603043F001038DF8DF
:10CD70006030E2E703229DF8623062F302038DF82F
:10CD800062309DF8613003F07803A3F140077B42E5
:10CD90007B41DBE703229DF8623062F302038DF8EA
:10CDA00062309DF8613013F0780F14BF0123002327
:10CDB000CCE70123CAE79DF96020002AACBF4FF001
:10CDC000FF32199A95E699077FF5A2AE1A9F0023C4
:10CDD000CDE919339DF8623003F00703042B09D124
:10CDE0009DF861309A0705D49DF96130002BB4BFDE
:10CDF0000D2706279DF862309DF8611003F00703A8
:10CE0000012BC1F3C30136D1CB1E042B20D8DFE8A0
:10CE100003F00307071F1F0054F8042BD31704E087
:10CE2000073424F00704F4E80223CDE916239DF823
:10CE30006060B30755D04A464146099B039804F009
:10CE400021FF0028C0F2C6830544DDF82490A3E545
:10CE500054F8042B01294FEAE273CDE9162305D1DA
:10CE60009DF85830169300231793E0E70229DED18E
:10CE7000BDF95820D2E7022B23D1CB1E042B13D8A7
:10CE8000DFE803F0030A0A12120000232268201DC3
:10CE9000169217930446CAE7073424F00700F0E817
:10CEA0000223CDE91623F5E754F8043B0129169334
:10CEB0004FF000031793D3D00229B8D1BDF85830F2
:10CEC000D0E7042B07D1073424F00704F4E8022349
:10CED000CDE91623ABE7032B04BF54F8043B1693AC
:10CEE000A5E79DF86390B9F1780FAED8B9F1570F67
:10CEF00000F2A780B9F1250F00F0EE80B9F1240F00
:10CF0000A3D9B9F1410F03D0A9F14503022B9CD855
:10CF1000DDE91623002A73F10001C0F2D581310743
:10CF200000F1D48116F0100618BF2026C3F30A5B67
:10CF3000C3F3130306920793DDE90623CDE9122319
:10CF4000BBF1000F40F0C481DDE90632134314BF8A
:10CF50004FF0010C4FF0000C58460799B9F1460FFD
:10CF60004FEAC123069908BF4FF06609CA0243EA97
:10CF700051534BEA02010C91C11719430D91DDE9A0
:10CF80000C010143CDE9122300F01582BCF1000F22
:10CF900040F0D581129B05210493139BABF2FE3B1D
:10CFA00043F000430593DDE90423CDE91223002378
:10CFB0001A461BF1020FC0F2CB811BB1DDE904015F
:10CFC000CDE91201DDE91231BBF1000F00F3DB8185
:10CFD0001399129BCBF104000BF11C0B01FA0BFB14
:10CFE000A0F1200CC34021FA0CFC43EA0B0343EAF6
:10CFF0000C03C140CDE9123109F0DF03472B40F0AB
:10D00000E181D01C02DB974280F2D881A9F10209AC
:10D01000002F5FFA89F900DD013F9DF86030990625
:10D0200000F1D081002FD4BF00230123B9F1660F96
:10D030000E9340F0C981BB1840F1C7814FF0000A40
:10D04000C7E1A9F15803202B3FF6FFAE01A252F829
:10D0500023F000BF69D200004BCE00004BCE000091
:10D060004BCE00004BCE00004BCE00004BCE00005C
:10D070004BCE00004BCE000011CF00004BCE000085
:10D0800005D1000009D2000011CF000011CF00002F
:10D0900011CF00004BCE000009D200004BCE0000A3
:10D0A0004BCE00004BCE00004BCE00009FD20000C4
:10D0B00069D200006DD200004BCE00004BCE0000C4
:10D0C000DFD000004BCE000069D200004BCE000044
:10D0D0004BCE000069D200004146484668E4002F6C
:10D0E000DDF858900ADB3946484604F0CFFF0026A9
:10D0F00009EB000AB9F1000F0CD1A6E6484604F08E
:10D10000BEFFF4E70026169B0DF1750A8DF874300A
:10D110000DF17409AAEB090206B101329DF8620013
:10D12000C30640F14C820232199940060A44089B1A
:10D1300044BF1A995218002B25DD9B1A9DF86020D8
:10D140005107C2F3800B00F14C82570640F1458233
:10D15000002E00F04482089341463046039B9847D6
:10D160000028C0F237825E463027089B01350893BD
:10D1700003EB050B089BABEB0305002B03F1FF331F
:10D18000089300F320823EB141463046039B984706
:10D190000028C0F21F8201359DF86220560640F13A
:10D1A0007E829DF96120002AC0F21D82A5EB09054F
:10D1B00099F800004F46A0F13002092A05EB090B4F
:10D1C00009F1010940F23F829DF86220199E900604
:10D1D00008D406EB0B09002EA9EB060B06F1FF366F
:10D1E00000F3388238782E280BD14146039B9847AC
:10D1F0000028C0F2EF81002E0BF1010B00F3328208
:10D200000137ABEB070B38E230072BD416F01006D2
:10D2100018BF2026DDE91623002A73F1000105DA84
:10D220002D26524263EB4303CDE91623DDE91601B7
:10D230000DF18D03009318AA1DAB04F0D8FC8146B4
:10D24000002F0DF18D030BDB9DF86010A3EB09029D
:10D250006FF3861197428DF8601001D9BF1A1997A4
:10D260009A4647E72B26D5E70026DFE716980028E1
:10D2700000F09F810DF18D03009300211DAB18AAD2
:10D2800004F0B5FCBDF86230814603F0EF0343F4CF
:10D29000F04343F010030026ADF86230D0E7169B50
:10D2A00007293FF6D2ADDFE801F00D04060D0808AE
:10D2B0000D0D1D70C9E51D80C7E52846E917C3E9B6
:10D2C0000001C2E51D60C0E52D262FE62B262DE6C8
:10D2D00040F2FF739B452DD1DDE906231343A9F1ED
:10D2E000410918D1B9F1190F95BF44F6496346F6C3
:10D2F0006963ADF87430ADF8743094BF462366238B
:10D300008DF876309DF860300DF1770A6FF3861353
:10D310008DF86030FCE6B9F1190F95BF44F24E1359
:10D3200046F26E13ADF87430ADF8743094BF4E23EE
:10D330006E23E5E74FF0000C0EE60BF1FF3B921871
:10D340005B41002A73F10001F7DACDE9122321E6EF
:10D35000049B05985B0843EAC0734008B0F1333F73
:10D36000DC46CDE904300BF1010BF1D2A3FB01AB9C
:10D370004843CDE904AB059B0CF1020BC3180593A0
:10D38000013A012315E6023341F1000112A8CDE96B
:10D3900012310E9204F0F5FBDDE912010E9A0BF149
:10D3A000FF3B013200184941002871F100030BF1E5
:10D3B000FF3BF7DA04E60022934609E64FF06609E0
:10D3C000BF1A2AE6002331E67B1C102BA8BF1023CE
:10D3D0009A461021002011914FF00061CDE914010F
:10D3E000DDE914100AF1FF3ABAF1FF3F1FD1129B99
:10D3F000CB180A93139B6FF0704140EB03034FF07F
:10D40000FF300B93DDE90AAB594508BF50451AD3ED
:10D4100050465946CDE91201B9F1660F53D1002AA1
:10D4200020DC30230DF1750A8DF874302BE04908AB
:10D4300041EAC0714008CDE9141014A80F9204F01D
:10D44000A0FB0F9ACCE70A9B0F920B9A5B0843EA6A
:10D45000C273510812A8CDE9123104F092FB0F9A61
:10D460000132D9E70DF1740A1199002909DD11A9DA
:10D4700012A80F9204F0A4FB0F9A0AF8010B013ACC
:10D48000F2D1199200229DF86010880601D4002F75
:10D490003FDD53462E2103F8011B92B1002F76DDAC
:10D4A0005142B942A8BF394600291991A7EB01079B
:10D4B000D4BF002101219DF8620061F345108DF871
:10D4C00062009A4620E011A912A80F9204F078FB9E
:10D4D0000F9A9DF86030302818BF02F1FF3299068C
:10D4E0008DF8740001D4002F53DD2E238DF8753094
:10D4F0000DF17603E5E711A912A80F9204F060FB85
:10D500000F9A0AF8010B013F002F02DD1199002943
:10D51000F1DC0E9B002B3FD11A9709F0DF01452962
:10D5200023D1002AB4BF2D212B215046B8BF52422F
:10D53000632A00F8029B8AF801100ADD642792FB37
:10D54000F7F107FB112201F1300C0AF103008AF810
:10D5500002C00A2792FBF7F1824607FB112201F174
:10D56000300C30320AF802CB4270199A002A1EDCC5
:10D570001A9A002AD4BF002201229DF8621062F399
:10D58000861100228DF862108AF80020C0E59A46C4
:10D59000BFE70DF1750ABCE700211A9150461AF851
:10D5A000011D3029FAD02E2918BF8246B5E7012285
:10D5B000E3E7DFF83CA10646AAF10509AAE507075B
:10D5C00048BF0132B0E541463846039B98470028E2
:10D5D000BFF6D0AD25B0BDE8F08F2027C7E53027D6
:10D5E000C5E50893CFE5A5EB090B4E460BEB090506
:10D5F00019F8010B702820D11A9A02EB0509A9EB42
:10D600000502002A43DC534632464146039804F0A3
:10D6100039FB0028DEDB089B2844034405469A4674
:10D62000AAEB0503002B7FF710AC41462020039B9B
:10D6300098470028CEDB0135F2E74146039B984727
:10D640000028D2DAC6E74146039B98470028BFF678
:10D65000AFADBFE741463020039B98470028BFF697
:10D66000BAADB7E741463020039B9847013EBFE57E
:10D670004146039B98470028ACDB3E460BEB070571
:10D6800017F8010BA0F13002092AF1D9B4E741469D
:10D690003020039B984700289CDB0135AFE7D1067B
:10D6A00001D4120706D541463020039B9847002835
:10D6B00090DB01359DF86220D30607D541469DF8E1
:10D6C0006300039B9847002884DB0135199E2E4494
:10D6D000721B002A02DC53464A4696E74146302038
:10D6E000039B98470028FFF675AF0135F0E700BFB0
:10D6F0004A2A01004FF02002EFF3118382F31188D0
:10D70000BFF36F8F0121044AC2F8401583F31188DB
:10D71000BFF36F8F002070470090035020B1034B80
:10D72000800143F001031847704700BF90270100B4
:10D7300007B501904FF02002EFF3118382F31188B7
:10D74000BFF36F8F04F051FB019801F0B5F8034867
:10D7500004F078F800F0ECFEFCE700BF4B2A010073
:10D760000E4A70B5841A05460C200E464021A310BF
:10D770000B4C5C43E4B200FB0420084404F0A7FA1D
:10D78000011E05DB074B03EBC404636898470021C7
:10D7900028463346BDE87040184700BF700200209D
:10D7A000B76DDBB6AC2701002DE9F0410C25104E1A
:10D7B0008046841BA3100F4C0F465C43E4B26543C4
:10D7C00005F140004021304404F09AFA011E09DBC3
:10D7D000094A7319C3E90E27084B53F83430BDE8E2
:10D7E000F041184740463B46BDE8F041184700BFAE
:10D7F00070020020B76DDBB6631D0100AC2701008D
:10D8000070B5002201210446052000F03BFE0520F2
:10D8100000F01AFE0F4801F0CBFC0F4B984215D1D7
:10D8200004F0E7FCE6680D49304604F068F800288B
:10D830000BDB01253564E468084904F11C0004F0A1
:10D840005EF8002801DB0020E56470BD6FF0040085
:10D85000FBE700BF9DD800000000AD0BBC27010016
:10D8600073B50C23014600264B430A48C4184033C5
:10D87000D4E90E521844A663019204F05FFA35B160
:10D880002B46019A044802B0BDE87040184702B028
:10D8900070BD00BF70020020C000002010B1012840
:10D8A00004D07047034B1B6C5B0701D1FFF7D8BF57
:10D8B000704700BF7002002008B54FF02003EFF35F
:10D8C000118183F31188BFF36F8F124A136843F0FD
:10D8D000020013F0010310600CD04FF05022D2F878
:10D8E0000C34D2F80C2413F0010303D00A4804F0DE
:10D8F00025FA012381F31188BFF36F8F23B1BDE8AF
:10D9000008400020FFF7ACBF0120BDE8084001F04F
:10D910005FBC00BFC0020020B0020020074BD3E86C
:10D92000EF2F22F00201C3E8E01F0028F7D1D30750
:10D9300002D4012001F07EBC704700BFC00200206D
:10D940001FB500220123CDE902236B46084ACDF81A
:10D9500000D0CDF804D004F02BFA002805DB4FF4FA
:10D9600080420023684602F0BFFD05B05DF804FB6D
:10D97000831D01002DE9F843012206463949D1E80B
:10D98000EF3FC1E8E02F0028F9D133B936493748D5
:10D990004B60CB608A6003F0C5FF731E012B32D849
:10D9A000012E07D14FF05023D3F81C3403F00303AA
:10D9B000022B28D004F044FD044618B92C4B1B78E8
:10D9C000002B47D14FF02003EFF3118583F311882B
:10D9D000BFF36F8F0124274FDFF89C80DFF89C9006
:10D9E0004FF05022D2F81834D2F81824D2030CD5B4
:10D9F00003F00303022B01D0012E06D124B385F3DB
:10DA00001188BFF36F8FBDE8F883C4B1284600F0DA
:10DA10009DFD4FF05022D2F81835DBB2012BDFD13B
:10DA200039680029DCD00021396039680221C2F848
:10DA300018152022C8F88021C9F80030D0E700214D
:10DA4000212002F009FDE4E74FF050230222C3F841
:10DA50000423D8E74FF0502302220546C3F80823D9
:10DA6000B9E700BFC4020020600200208C02002041
:10DA7000A90800200451005000E100E008500050C7
:10DA8000044A1368C91A21F07F400344136002F06E
:10DA9000EFBE00BFD40200202DE9F0474FF48037DD
:10DAA0004FF00009860000F1500406F15026A40052
:10DAB00006F58036A4B204F15024D6F84035DFF8DC
:10DAC0006C8021F07F4504F580348740D8F804A5A8
:10DAD000A3EB0A0323F07F432AF07F42012BC6F811
:10DAE000402502D1132004F0B1FC0AF10202AB1A66
:10DAF00023F07F43B3F5000F88BF1546C4F80090AC
:10DB0000236825F07F43C8F84473C6F84035D8F839
:10DB100004359A4506D0EB1A023B23F07F43B3F558
:10DB2000000F01D8BDE8F0872B46CFE70050015029
:10DB3000F8B5002427460F4E0F4B104A18461D68B3
:10DB400004B1F8BDD2F80413C903FAD5316800292D
:10DB5000F7D0346031684FF48031C2F848130124A3
:10DB6000D2F8401525B100205A681F60A847E3E7A6
:10DB70000560E6E740510150C80200200050015006
:10DB800038B500244FF480334FF400120D4D0121BD
:10DB9000C5F80845C5F804330B4B1520C3F88021A0
:10DBA000224600F06FFC152000F04EFC0123074ACE
:10DBB00002201360064A2B601360FFF7DBFE20464D
:10DBC00038BD00BF0050015000E100E00850015096
:10DBD000D0020020134BB0F1FF3F08BF18460138B8
:10DBE00000281CDD9842A8BF18460F4BD3F8042527
:10DBF0000E4B1968521A12F4000F18BF002022F0C1
:10DC00007F4301330A4A03440A48106000205060F1
:10DC1000044A934294BFC9188918FFF73DBF0020FA
:10DC2000E3E700BFFFFF7F0000500150D402002057
:10DC3000C802002081DA00004FF02002EFF31183C8
:10DC400082F31188BFF36F8F064AD2F80405064AA3
:10DC50001268801A20F07F4083F31188BFF36F8F22
:10DC6000704700BF00500150D4020020034610B599
:10DC700088B08DF807300DF1070302930123094A9C
:10DC8000CDE9051310680393002207238DF81020B7
:10DC90008DF81C30836802225C6802A94623A047E5
:10DCA00008B010BDD802002070B586B00E460DF148
:10DCB000070105461446FFF7D9FFC8B99DF807309C
:10DCC0008DF8085023EA06010A4B44EA010218685D
:10DCD00002AB039302238DF807208DF809200493EB
:10DCE0008DF81430836801225C6803A94623A0479D
:10DCF00006B070BDD802002008B501F0F9FD044B54
:10DD0000002818600CBF6FF01200002008BD00BF93
:10DD1000D8020020F7B500281C4614BF4FF400536A
:10DD20004FF400438A4241D90D46214F00283AD092
:10DD300005F5E07647F826406E1CB24231D15A43D1
:10DD40001C484B4300922A4603F07CFD1A4B14F00A
:10DD5000100F1A491A4808BF194603F073FD14F052
:10DD6000040F14BF72212D21164803F06BFD14F02F
:10DD7000020F14BF77212D21124803F063FD14F028
:10DD8000010F0CBF2D2178210E4803F05BFD6C21A3
:10DD90000C4803F057FD0C4803B0BDE8F04003F019
:10DDA00051BD3546C2E705F5C076C3E703B0F0BD07
:10DDB00000300050932A0100872A01007E2A0100CA
:10DDC000122C0100AD2A0100E72D010008B543B275
:10DDD000002B0CDB012200F01F018A405B09104977
:10DDE000203341F82320BFF34F8FBFF36F8F8300A1
:10DDF00003F1A04303F540533128D3F8002806D09F
:10DE0000002A07DA02F00302023A012A02D8054A80
:10DE1000C3F80028012104F0C7F8002008BD00BFA6
:10DE200000E100E00001008030B54FF4C13485B05E
:10DE30002E4D4FF4C1312E4803F004FD21682D48CA
:10DE400003F000FD29682C4803F0FCFC102200219F
:10DE5000684604F082F9236868460093029400F053
:10DE60000BFF012000F038FF002000F021FF002010
:10DE700000F046FF0121002000F060FF00F054FF99
:10DE80002C681E4803F0DEFC0820FFF79FFF24F0FB
:10DE90000104BFF34F8FBFF36F8F64086400204607
:10DEA000214622462346B7EE000AF7EE000AB7EEF7
:10DEB000001AF7EE001AB7EE002AF7EE002AB7EEC6
:10DEC000003AF7EE003AB7EE004AF7EE004AB7EE36
:10DED000005AF7EE005AB7EE006AF7EE006AB7EEA6
:10DEE000007AF7EE007AFEF723FC00BF04820100FF
:10DEF000B02A0100C72A0100DC2A0100FA2A010029
:10DF00002DE9F8433B4803F09DFC002140F2171334
:10DF100008460322FFF7FEFE40F2071320220321EA
:10DF20000020FFF7F7FE344803F08CFC334B344AF3
:10DF3000C3F3C431C3F30E03C3F50043C3F3431368
:10DF4000C2F80015C2F80435D2F80015D2F804253D
:10DF50002C48520103F076FC274803F073FC03F0D1
:10DF600073FF014610B1284803F06CFC00242748D9
:10DF700003F068FC40F21713082200210120FFF78C
:10DF8000C9FE1F4D40F20713202208210120FFF790
:10DF9000C1FE194803F056FCC5F880441C4803F044
:10DFA00051FC1C4FC5F8C044DFF87C801A4DDFF8E7
:10DFB0007C906E792146002E14BF3B46434648466E
:10DFC0002A6803F03FFC66B91448013403F03AFCB8
:10DFD0001A2C05F10805ECD10748BDE8F84303F019
:10DFE00031BC2879FFF7F2FE08B10D48EDE70D4886
:10DFF000EBE700BF302B0100E72D0100E07F0100BF
:10E0000000300050542B01009A2B0100CA2B010054
:10E01000EC2B0100252B0100C8270100152C010065
:10E020001C2C0100242C01008B2A0100082C01006B
:10E030002DE9F0430746002685B0DFF83490DFF87D
:10E04000348001AD59F8044B98E807003C4485E85A
:10E0500007000C222946204604F02DF800B91CB90F
:10E060000136052EEED10024204605B0BDE8F08330
:10E07000982801006027010070B50C461546064639
:10E08000B0BB6FF01500BDE8704071467246734634
:10E09000B7EE000AF7EE000AB7EE001AF7EE001A24
:10E0A000B7EE002AF7EE002AB7EE003AF7EE003A94
:10E0B000B7EE004AF7EE004AB7EE005AF7EE005A04
:10E0C000B7EE006AF7EE006AB7EE007AF7EE007A74
:10E0D0008EF3008C10B4F1EE10CA4FF66074C0F6E7
:10E0E000FF740CEA040CE1EE10CA10BCF44674474D
:10E0F000002AC6D003F0BEFF0128C2D0B4F5404FBD
:10E1000017D32B19B3F5424F06D90B4A94420AD9BB
:10E1100002F61D22934209D82A462146304603F0D2
:10E12000F1FF0020AFE7054A944202D9044A934226
:10E13000F2D94FF0FF30A6E70302FF002F01FF00E6
:10E140003801FF0070B5054610460E46144603F030
:10E1500091FF012837D16FF01503BDE870401846D4
:10E16000714672467346B7EE000AF7EE000AB7EE44
:10E17000001AF7EE001AB7EE002AF7EE002AB7EE03
:10E18000003AF7EE003AB7EE004AF7EE004AB7EE73
:10E19000005AF7EE005AB7EE006AF7EE006AB7EEE3
:10E1A000007AF7EE007A8EF3008C10B4F1EE10CA0C
:10E1B0004FF66074C0F6FF740CEA040CE1EE10CA6E
:10E1C00010BCF44674472846FFF732FF0546304638
:10E1D000FFF72EFFCDB12A6A0E4B9A4215D148B1F6
:10E1E0000123016A0B4A914202D13BB92370B4E783
:10E1F000002BB0D0012323700023AEE76B69426986
:10E20000934234BF00230123F5E70028A3D0002365
:10E21000E7E700BFFFFF0291014802F0D9BD00BF50
:10E22000AC28010008B5B0B14368042B0DD1002221
:10E230000368D3E8EF1F012903D1C3E8E02F0028CA
:10E24000F7D1074808BF104608BD3BB1006801F090
:10E2500047FD0020F8E76FF4E040F5E70148F3E7F9
:10E26000E98FFFFFEA8FFFFF10B5044618B90D4B89
:10E270000D485B689847616808290DD031F00403A8
:10E280000AD011F0020108D02146084801F086FCAE
:10E29000002323600023636010BD1422206803F074
:10E2A0005CFFF7E774000020252D0100DC02002050
:10E2B00010B5044618B9164B16485B689847636852
:10E2C000042B23D0082B21D0CBB92368BBB94FF046
:10E2D000FF324FF0FF3321460F4801F02DFC08B903
:10E2E00023681BB90A4B0D485B689847142200212C
:10E2F000206803F032FF636843F002036360206824
:10E3000003F0EBFF636843F00103636010BD00BFDF
:10E3100074000020252D0100DC0200204B2D01009F
:10E3200008B5E8B14368042B0CD101220368D3E897
:10E33000EF1F002903D1C3E8E02F0028F7D10BD14C
:10E34000002008BD53B100684FF0FF324FF0FF339B
:10E3500001F04EFC0028F3D00348F2E70348F0E751
:10E360006FF4E040EDE700BFE98FFFFFEA8FFFFFAA
:10E3700008B5064940231422054803F093FFBDE881
:10E3800008400449044802F075BD00BFF8020020AF
:10E39000DC020020C4280100B4280100094A0A490F
:10E3A000936809689867D96708494B6843F08053B8
:10E3B0004B60002383F31188BFF36F8F9368D86F8E
:10E3C000704700BF480800204C29010000ED00E024
:10E3D00013498A684FF038001044EFF3098C80E845
:10E3E000F01F202080F31188BFF36F8F0D4F4FF087
:10E3F00000668A6A8A603E60906F0023936780F3AC
:10E40000118802F1380090E8F01F8CF3098802F1BE
:10E41000000004B503F0F6FDBDE8044070470000BD
:10E420004808002004ED00E01EF0040F0CBFEFF3DD
:10E430000880EFF30980816911F8021C0229FFD0DE
:10E4400001B503F0E5FD01BD43B2002B08DB01225D
:10E4500000F01F0002FA00F0024A5B0942F82300B4
:10E46000704700BF00E100E0054B420953F822204D
:10E47000012300F01F0003FA00F01040704700BFB6
:10E4800000E100E043B2002B01F10101ACBF03F158
:10E490006043064B4FEA4111C9B2ABBF03F561437C
:10E4A00000F00F0083F800131954704714ED00E0DA
:10E4B00042F8203C009B0B4942F81C3C019B21F098
:10E4C000010142F8183C029B42F8081C42F8143C37
:10E4D0004FF0807342F8043C0023203A8265836742
:10E4E000704700BFB719010008B504460E4615462F
:10E4F0000023E1EE103A00F055FA094B9C60A36E40
:10E5000083F30B88284686F30988002163B681F3DC
:10E510001188BFF36F8F0022002303F04CFA00BF75
:10E5200048080020014910220A60704710ED00E001
:10E5300072B6404080F31188BFF36F8FBFF34F8FE7
:10E5400030BF62B6BFF36F8F704700BF72B64940ED
:10E5500081F3118820BF80F3118862B6704700BF35
:10E5600030BFFFF7FDBF00BF174A08B5174B22F0B9
:10E570007F029A60BFF34F8FBFF36F8FD3F888206D
:10E5800022F47002C3F88820D3F8882042F4A00255
:10E59000C3F888200E4A536823F040435360BFF30A
:10E5A0004F8FBFF36F8F0023E1EE103AEFF3148328
:10E5B00023F0040383F3148801F0F2F902F060F809
:10E5C00000F0C2F901F010FA00C2000000ED00E016
:10E5D00030EF00E001B572B60B4A506A00281EBF4A
:10E5E0000021516203F05CFE62B6EFF30580A0F1FA
:10E5F00010004FEAC0000549014409C99847BDE829
:10E600000140034908470000480800204C2501004C
:10E610009DE80000002080F31488BFF36F8F002076
:10E6200080F30A8880F30B8803F046FB00200E4934
:10E630000860BFF34F8F0D4880F3088800F05EF943
:10E64000202080F311880A484FF40061401880F3BD
:10E650000988EFF314800221084380F31488BFF384
:10E660006F8FFFF781FF000094ED00E0B0180020ED
:10E67000F0190020EFF30880EFF3098101B572462D
:10E6800000F074F801BD00BF0E4B9A6A9A6A9A6A4C
:10E69000920708D55A6B9A6A120604D518B19A6A7D
:10E6A00022F080029A620020064B9A6A9A6A9A6A5D
:10E6B000D20658BF9A6A9A6A42F0FF029A620870BC
:10E6C000704700BF00ED00E00D4B9A6A9A6A9A6AA3
:10E6D000920508D59A6B9A6A120404D518B19A6A01
:10E6E00022F400429A620020054B9A6A9A6AD20587
:10E6F00058BF9A6A9A6A42F47F429A6208707047D9
:10E7000000ED00E0094B9A6A9A6A986A9A6A9A6AD6
:10E710009A6A9A6A9A6A10F480106FEA02426FEA63
:10E72000124218BF02209A62704700BF00ED00E05D
:10E730000D4B9A695A695A69D0070FD45A699107E3
:10E740000CD45A69520709D45A69100706D45A6979
:10E75000D10603D45A69920658BF5A695A6942F0E1
:10E76000FF025A61704700BFD0ED00E0F0B5414BA9
:10E7700000255B688BB0C3F3080385F31188BFF3F2
:10E780006F8F02F07F44B4F17F4F1ED112F001046D
:10E790001AD0560602F0080467D482F00402C2F3CD
:10E7A000800564B1EFF389860022033B8DF80720D2
:10E7B000042B4BD8DFE803F00B4C50414800EFF33B
:10E7C0008886F1E70E46EFE725462E46ECE7294B13
:10E7D000DA6A92073AD4DC6A14F0804408D028330D
:10E7E0001B78EBB101200DF10701FFF74DFF044647
:10E7F0009DF8073093B92022314602A803F082FC2D
:10E80000099B6DB3C3F3080222B96FEA53236FEA81
:10E8100043230993204602A903F0F8FB0BB0F0BD97
:10E82000154B1B782BB101200DF10701FFF74CFFB1
:10E83000DDE7124B1F88BFB217B1FFF763FFD6E7C2
:10E840000F4B5C69002CD3D0FFF772FF0024CFE799
:10E8500000200DF10701C8E700200DF10701E5E7F1
:10E8600023F4FF7323F00103D3E7002CAAD106465B
:10E87000012599E700ED00E029ED00E02AED00E038
:10E88000D0ED00E0044B5A6942F010025A615A6917
:10E8900042F480625A61704700ED00E0044B9968D1
:10E8A000986A884203D003494FF080520A6070474B
:10E8B0004808002004ED00E0BFF34F8F0549064BE8
:10E8C000CA6802F4E0621343CB60BFF34F8F00BF0E
:10E8D000FDE700BF00ED00E00400FA050023184644
:10E8E000054A1168C1F307218B4200D1704793603C
:10E8F00010610133F8E700BF90ED00E010B572B68B
:10E90000002484F31388FFF7E9FF0E4A23461146DB
:10E910004FF0FF3403F120000133102B42F8204068
:10E92000F8D100234FF0FF3003F160020133102BC8
:10E9300041F82200F8D162B6BFF34F8FBFF36F8F5B
:10E9400010BD00BF00E100E0002320210348C218F1
:10E950000133412B82F80013F9D1704700E100E048
:10E9600008B50E4B9B68834207D1EFF3058393B143
:10E970000B4A536843F08053536001F0BFFB4FF0E4
:10E980002003EFF3118083F31188BFF36F8FBDE88D
:10E99000084003F0A9BC01F05FFE00BF480800205A
:10E9A00000ED00E01FB5094C094A23460121094842
:10E9B00000F002F900230393074B0121E41A01A898
:10E9C0000193029400F002F904B010BD0000012090
:10E9D00000000020D82801005801002010B50B6865
:10E9E0000C7A23F01F0204F01F031A43CB6864095A
:10E9F00023F01F03044943EA440343F00103886002
:10EA0000CA600B6110BD00BF90ED00E02DE9F04F32
:10EA10008846144606464FF000094A4D85B0C14568
:10EA200005DA7768BFB31F2F05D86FF015042046AD
:10EA300005B0BDE8F08FFB06F7D1D6F800A01AF0BC
:10EA40001F0FF2D1504603F00BFB834607EB0A0081
:10EA5000013803F005FB8345E7D11BF1160FE4D025
:10EA6000631E5B45E1DBC5F808B0E968C5F808B08E
:10EA70002F6921F01F01D6E900321A44994247F06C
:10EA80001F0702F1FF3A1CD1574508D131465FFA02
:10EA90008BF003F0C8FA09F101090C36BFE73146E3
:10EAA000C5F808B0EB6822F01F0203F01F031A43F9
:10EAB000EA60E0B203F0B7FA10F1160FB5D0441CCB
:10EAC000E9E7013B5745E0B223F01F03C5F808B062
:10EAD00006D12A69314602F01F0213432B61E9E790
:10EAE000296901F01F010B432B61314603F09BFAAA
:10EAF00010F1160F99D0C5F808B0EA689DF80830F3
:10EB0000013F62F304038DF808302B699DF808205B
:10EB10005B0863F347128DF80820D6E900321344EE
:10EB2000009323F01F033B44441CA3EB0A0AE0B20A
:10EB30002AF01F030F2803933FF677AF6946FFF7CC
:10EB40004DFFBCE790ED00E00522034B5A60BFF398
:10EB50004F8FBFF36F8F704790ED00E0BFF35F8F73
:10EB60000022014B5A60704790ED00E038B50E4C22
:10EB70002568102D14D8FFF7F1FF00200B4B0C4A2D
:10EB80001A63854205D10B4B1D70FFF7DDFF002096
:10EB900038BD616801EB0011FFF720FF0130F0E79D
:10EBA0004FF0FF30F4E700BFE428010090ED00E0F3
:10EBB000AAFF4400A808002010B5034C2278FFF7F4
:10EBC00025FF207010BD00BFA80800202DE9F74FD9
:10EBD000264D8A4606464FF00008AB46244FD045E6
:10EBE0001BDAD6F80490B9F1000F39D03168084625
:10EBF000019103F035FA0199044609EB010001384F
:10EC000003F02EFA84424FF014021A4B08D06FF032
:10EC1000150302FB08F84BF8083003B0BDE8F08F8D
:10EC200014F1160F2C60F8D01978A142F5DD02FB23
:10EC300008B0BC60BC60FC6800F10801007B64F3B4
:10EC40000400087138690C79400860F347140C71AE
:10EC5000F96821F01F016960396921F01F012961FC
:10EC600008F1010814350C36B9E700BFF807002099
:10EC700090ED00E0A808002082680C4B9A600368C1
:10EC800083F38888436883F38988027B02F001015B
:10EC9000EFF3948323F00303920748BF43F002038A
:10ECA00009B143F0010383F39488704700ED02E05B
:10ECB000084AD36848B123F400531B041B0C43F0EB
:10ECC000BF6343F40033D36070479BB243F40053F7
:10ECD000F5E700BF00ED00E0084AD36840B19BB201
:10ECE00043F4804343F0BF6343F40033D360704781
:10ECF00023F480431B041B0CF4E700BF00ED00E08D
:10ED0000084AD36840B19BB243F0080343F0BF63A5
:10ED100043F40033D360704723F008031B041B0C3B
:10ED2000F4E700BF00ED00E0034AD2F88C3043F472
:10ED30004063C2F88C30704700ED00E0084B1A6861
:10ED400018B142F001021A60704722F001021A6005
:10ED50001A6811B142F00202F5E722F00202F2E76E
:10ED6000D0ED00E008B51248FEF7C6FFF0B903F099
:10ED700055F8D8B903F05EF8C0B9012003F05FF888
:10ED8000A0B9012003F04FF880B9072003F034F850
:10ED900060B91F2003F02AF840B9072003F037F8C4
:10EDA00020B9BDE80840012003F02CB808BD00BF21
:10EDB000872D010010B50446002201210A20FFF72B
:10EDC00061FB6068E368064A00F1080100F0A8FAF8
:10EDD000044B984214BF6FF00F00002010BD00BF1D
:10EDE000E9ED00000000AD0B0378012B08D0022BE9
:10EDF00008D04BB9054B0B6201F1100001F054BB78
:10EE0000034BF8E7034BF6E7034BF4E70000AD0BC9
:10EE10000100AE0B0200AE0B0100AD0B2DE9F04F6F
:10EE20001D46C46889B0238D064689469246002156
:10EE3000142203A8D4F82C80009303F08EF98DF8E7
:10EE40000D504FF0FF324FF0FF33204601F04CFBE6
:10EE5000F068103000270022002301F045FB7068A5
:10EE600000F0A4FA4D463C46DFF814B1574501D3F3
:10EE700000242EE0297A0B0777D4009B6BB17B1C12
:10EE800053450AD2880708D42B7D81EA030202F099
:10EE9000010203F00403134325D0002C3CD10024CD
:10EEA0002B6806936B6804932B7A706803F0010259
:10EEB00013F0020F8DF80C2003A90CBF20220022B2
:10EEC00000F0A0FA584529D02C4B984253D06FF04F
:10EED0000404706800F07AFAF06801F0E5FA204660
:10EEE00009B0BDE8F08F01236A68009802EB040CBA
:10EEF00084453DD8C90706D4296808EB040001936E
:10EF000003F000F9019B6A681444C3B9002CC6D011
:10EF1000CDF818800494C7E70023E5E7F0681030C7
:10EF20004FF48042002301F0DFFA0028CFD1F368CC
:10EF30001B6A5B45CBD12B7ADB0703D40024013756
:10EF40000C3593E7069B9845F8D10C2303FB0793F8
:10EF50005A680C3B9442F1D3A41AD86808EB040118
:10EF6000019303F0CFF8019BF2E76FF02204B0E7C2
:10EF70006FF01B04ADE76FF00F04AAE70B00AD0BB9
:10EF80000000AD0B2DE9F0430025214C214E54F833
:10EF9000048CDFF8889085B0A84503D8002005B020
:10EFA000BDE8F083636A96E807001F6801AB83E859
:10EFB00007000C221946384603F07DF890B98FB14E
:10EFC000636A21691B681A6991420BD19A69A16928
:10EFD000914207D8E169914204D962695B6932EADA
:10EFE00003030AD0276A67B10B4802F02BFC4040AC
:10EFF00080F311884FF0040002DFE36801351C4400
:10F00000CAE7484602F01EFC636A1F60F5E700BFCE
:10F010003CC400006C2701008D2D0100B62D0100BD
:10F02000054B1868043B1B68092B03D1431E58424B
:10F0300058417047002070473401FF004F4A08B51F
:10F04000136843F0020313604D4B1B68092B01BF8B
:10F050004FF050230022C3F81421C3F81821FFF702
:10F06000DFFF30B10123474A1360A2F63822C2F80D
:10F070007835434B1B68092B07D1434B1B68012B89
:10F080001EBF0122414BC3F87825FFF7C9FF10B11D
:10F090000E223F4B1A603A4B1B68092B04D1002209
:10F0A0003C4B1A6001225A600022D30003F57F0313
:10F0B000D3F80013013108D0D3F800130132D3F88C
:10F0C0000433B2F5807F0B60EFD1334BDA69D1079F
:10F0D0003BD5324B1946D3F80024012AFBD1C3F8A3
:10F0E0000425D1F80034012BFBD12B4BDA69D20770
:10F0F00008D5DA69294922F00102DA61D1F8002441
:10F10000012AFBD11A6A01320AD11A6A22F0FF02DF
:10F1100042F020021A62214AD2F80034012BFBD1BE
:10F1200000221E4BC3F80425D3F80024012AFBD18A
:10F13000BFF34F8F1A491B4BCA6802F4E0621343B6
:10F14000CB60BFF34F8F00BFFDE71B6A0133C0D018
:10F15000134BD3F88C2042F44062C3F88C20D3F8D0
:10F16000882042F47002C3F88820BFF34F8FBFF3AA
:10F170006F8F0D4B0D4A1A6008BD00BFD0ED00E047
:10F180003001FF00384A00503401FF0000400050B9
:10F19000E4AE03500C4700500080FF000090035085
:10F1A00000ED00E00400FA05540000200090D003B8
:10F1B000044B1A7922B9012218601A71024870476B
:10F1C000024870470C0800200000AD0B0C00AD0B8E
:10F1D00010B1012820D070474FF05022D2F81834D7
:10F1E000D2F81814C90311D503F00303022B0DD173
:10F1F000C2F8183500220D4B1A601B6802224FF02E
:10F200005023C3F8042301229A6070474FF0502323
:10F210000122C3F81825EDE70022054B1A601B6890
:10F220004FF05023C3F80403186070470451005096
:10F230000051005038B510B1012818D038BD4FF03A
:10F2400050230222012142F210751C46C3F8082304
:10F25000154A10601268154A1160D4F81834DB039F
:10F26000ECD5012002F0C3FF013DF6D1E6E74FF0F7
:10F270005024002242F210750D4BC4F808031A60A6
:10F280001B680C4B1860D4F80C34D4F80C2403F031
:10F290000103D203D2D5002BD0D0012002F0A7FF6A
:10F2A000013DF0D1CAE700BF045100500C5000509E
:10F2B0000051005004500050164B10B51A6852B15E
:10F2C000002018601B6801224FF05023C3F8082368
:10F2D000114B1B689847114B1A688AB100221A60BB
:10F2E0001B684FF05023D3F81824D3F8181402F0F9
:10F2F0000302012A4FF0020103D1C3F818159A60E6
:10F3000010BDC3F80813044B0120BDE810401B6872
:10F31000184700BF005100500C0800200451005055
:10F320004FF0340CF8B506791C4D0CFB06FC05EBD0
:10F330000C0494F82D707FBB40F20C6EA7606360E4
:10F3400084F82F704B7B84F830700F6884F832306B
:10F3500045F80C2007F01F03DFF84CC080334CF851
:10F3600023E04C68006804F01F0380334CF823E06E
:10F370008B68C0F80875C0F80C45C0F824351AB180
:10F3800040F30730FFF760F8342303FB06550123F1
:10F39000034885F82D30F8BD0248FCE7140800202A
:10F3A0000000AD0B0500AD0B00258450062102685E
:10F3B0000379C2F800153421034A01FB032302221A
:10F3C00083F82D20704700BF1408002002680379DD
:10F3D00034200A4900FB0313002009499860C2F851
:10F3E0000813D2F8001221F4BC51C2F80012C2F87E
:10F3F0000005012283F82D20704700BF140800206B
:10F4000002029C012DE9F0473426002390F804E025
:10F41000AE4F046806FB0E7686F82E30CB680D469C
:10F4200003F06043B3F1005F944603D0A84E30462A
:10F43000BDE8F087A74BC4F8083396F82F3003F0E7
:10F44000FF0A23B1B368A44EC4F80433EFE712F007
:10F45000140F0CBF01230023894686F82F3006F1D4
:10F460000C08B9E80F00A8E80F00D9F80030C6F87A
:10F4700020C0C8F80030CCF3001386F830306B7829
:10F48000C4F88835C4F804A1D4F80431C4F824A120
:10F49000D4F82431C4F860A1D4F86031C4F848A18C
:10F4A000D4F848311CF0010318BF0123C4F85035CB
:10F4B0001CF0020318BF0123C4F840352B78032B3E
:10F4C00000F2B280DFE803F0819D66022A6902F053
:10F4D0006043B3F1005FA9D14FF48073E968C4F8C9
:10F4E00000326B68C4F84415C4F848350023C4F8EA
:10F4F0005031D4F8501101212162A160D4F850118B
:10F500000029FBD0C4F85031D4F85031AB68C4F8AE
:10F510004425C4F8483534234FF4802203FB0E738E
:10F520009A6008236D4E1CF0080F04D12A78032A34
:10F530001CBF0122E250342303FB0EF3FA18FB58E0
:10F54000002B74D10125D4F84821D4F804110029E6
:10F5500040F08780003A18BF0122D4F82411002916
:10F5600000F08580C4F82431D4F82411D4F8600167
:10F57000D4F8001210B111F4007F04D12562656146
:10F580000028E0D00022C90571D5C4F84831D4F86C
:10F590004821D8E76B68EA68C4F84425C4F84835C0
:10F5A0002B6903F06042B2F1005F7FF43FAFAA68BD
:10F5B000C4F834354FF48453C4F83825C4F8003205
:10F5C0003423022203FB0E7312E06B68EA681CF01E
:10F5D000200FC4F84425C4F848354FF034030BD04D
:10F5E0004FF48072C4F800224FF4802203FB0E73A4
:10F5F0009A600123236294E74FF40072C4F800225A
:10F60000DFE76B68EA68C4F83425C4F838354FF48E
:10F610008053C4F800323423022203FB0E739A6035
:10F620000123236200237DE708232D4E7BE71CF096
:10F63000040F1CBF002393601CF0400F06D134233D
:10F6400003FB0E739A6842F002029A60342303FBB4
:10F650000E77BB6843F40073BB60BB68C4F8043327
:10F66000E5E6C4F80431D4F80421012275E7002A44
:10F670003FF469AF3421002001FB0E72D4F8C4348A
:10F68000C4F8C43482F82F008BB1164A13F0010F6E
:10F69000154E18BF164613F0020F02F1010218BFF3
:10F6A000164613F0040F114B18BF1E46BFE61CF0A0
:10F6B000400F7FF4BCAE20460EFB017102F0A4FDAA
:10F6C000094B002808BF1E46B1E600BF1408002001
:10F6D0000A00AD0B02029C010B00AD0B0000AD0B4C
:10F6E0000400AD0B0000AE0B0100AD0B0200AE0B31
:10F6F000F0B55B4B5B4CD3F824211D4687B0FAB1C3
:10F700000022C3F82421D3F82421D3F80421BAB964
:10F71000A268C3F808230222A260A268C3F80423E7
:10F72000D3F860211AB1D3F800329E0503D4012228
:10F730004B4B1A625A61012384F82E3007B0F0BD9A
:10F74000D5F80431002B54D00023C5F80431D5F886
:10F750000431236A5D060AD494F82E303BB941493E
:10F760003F4802F051FD80F0010084F82E00236A2A
:10F7700013F0040722D13C4E01AD0FCE0FC5336804
:10F7800094F830C02B60364BC3F86071D3F8602119
:10F79000C3F85C71D3F85C21BCF1000F02D094F87F
:10F7A0002E205AB10022C3F80022A2602F4AC3F8CB
:10F7B00008234FF480622E4BC3F88021284AD2F8E8
:10F7C000C4349807C2F8C4343CD501238DF8003006
:10F7D00094F830300BB984F82F30236A5B0703D5D7
:10F7E00094F82E30002BA9D0D4E900316846984710
:10F7F000A4E7C5F84831D5F84831237B83B91A4FBF
:10F8000001AE0FCF0FC63B68336094F83030002B49
:10F81000D4D1C5F80032A360144BC5F80833C8E74B
:10F820004FF40073C5F8003240F20223A36003F1E5
:10F83000CE73C5F80833A368C5F804330123AB6061
:10F840002B627BE7590701D50223BFE7DA0701D511
:10F850000323BBE794F82E30002BB7D00423B5E781
:10F8600000A00050140800202008002002029C0183
:10F8700000E100E0F8B5104B104F53F82050013074
:10F8800053F82060AE4200D8F8BDD5E900342046D8
:10F89000984770B16CB10123E41B094A2411610936
:10F8A00052F8210004F01F0403FA04F4044342F860
:10F8B00021400835E6E700BF38290100C0000020DC
:10F8C00000010020084BC01A0011084B420953F8F0
:10F8D0002220012300F01F0003FA00F010420CBFA9
:10F8E00018460020704700BFC00000200001002023
:10F8F000114970B505460E46104C8C4204D10F4C90
:10F90000B4420AD1002414E02046FFF7DBFF10B117
:10F910002368AB420DD01034EFE72046FFF7D2FF4B
:10F9200008B91034ECE72846216802F0B8FB00283B
:10F93000F7D1204670BD00BF00010020C0000020AC
:10F94000F8B505460027154E4FF02002EFF311835E
:10F9500082F31188BFF36F8F286988B12F6183F319
:10F960001188BFF36F8F00F0C9FB4FF02003EFF356
:10F97000118083F31188BFF36F8F02F0B5FCE3E7CA
:10F9800002F07FFD012104460228D8BF084602F09C
:10F9900088FD7462FEF7CCFDD6E700BF4808002062
:10F9A0000248034A0021121A02F0D7BB5801002076
:10F9B000AC080020012208B5094B02201A70FFF79D
:10F9C00059FF02F047FD0320FFF754FF00F0E6FD6A
:10F9D00001F012FF034A137B23F00103137308BDE8
:10F9E000A9080020D80100202DE98048374BA7B096
:10F9F00003F5006989F3088883F30A880024E0236B
:10FA0000334D4FF0010B85F82230EC772C766C7675
:10FA1000AC76EC766B6A2F4E43F4E0236B626B6A34
:10FA2000DFF8CCA043F400236B62AC63FEF72AFF3F
:10FA3000FEF778FD4FF0FF33AB62EB6240F201134B
:10FA4000254DADF8243006ABAB602046CDE920440F
:10FA5000FFF710FF0120FFF70DFF00F0A3FC1F4B85
:10FA6000AE624FF480521E49059330465346CDE9AD
:10FA7000034BCDE90144009400F060FD737B8046A8
:10FA800023F004033046737302F05AFC0F23154F22
:10FA90004FF4A072CDE902431349144B3846CDE927
:10FAA00004B4CDE9005400F049FD7B7B524623F0BD
:10FAB00004037B7305F11C0341463046C5E9073357
:10FAC000EF602C76C5F80490FEF70EFDF0190020CB
:10FAD00000ED00E0D801002048080020F42D0100CE
:10FAE000B008002058010020B018002041F90000A3
:10FAF000B5F9000070B50E4B0E4CA34201D30020A7
:10FB000070BDD3E9030141EA000212F003020BD1F8
:10FB10009D685A61AA4201D11C33EEE75E69013249
:10FB20000E6059610144F5E76FF01500E8E700BF8A
:10FB30000401002004010020D3B50C4616461F46E0
:10FB40004FF02003EFF3118183F31188BFF36F8F20
:10FB500043695BB123601B6843618369013383613F
:10FB6000002081F31188BFF36F8F11E056EA07027E
:10FB700003D16FF00B002360F3E70246CDE9006785
:10FB8000044800F07DFB18B9034B9B685B69236058
:10FB900002B0D0BDAA08002048080020F8B50446ED
:10FBA0000D464FF02003EFF3118683F31188BFF366
:10FBB0006F8F47696FB902F01EFC50B12A68C767A2
:10FBC000426102F0BDFB3146BDE8F840074800F055
:10FBD0000FB92B6862691A602B686361A369013BE6
:10FBE000A36186F31188BFF36F8FF8BDAA080020C8
:10FBF0002DE9F341044616461F464FF02003EFF36C
:10FC0000118883F31188BFF36F8FC368324A6BB1D9
:10FC100080689168884219D056EA070318D188F3A2
:10FC20001188BFF36F8F6FF00F000CE0916891F9AE
:10FC30000E100133E36093682161A36088F311889B
:10FC4000BFF36F8F002002B0BDE8F0812169F0E7BB
:10FC500090F90E3091F90E109942A8BF194621EA89
:10FC6000E17199422CDA00F059FB054622464146E3
:10FC7000CDE90067194800F003FB0028E3D04FF0FE
:10FC80002003EFF3118683F31188BFF36F8F23688E
:10FC90002169A34207D033B193F90E309942A8BF2E
:10FCA000194621EAE171A06890F90E30994209D114
:10FCB0006DB13146094800F09BF86FF00A00C2E7C9
:10FCC0000025D3E700F02AFB0028F2D1F0E786F305
:10FCD0001188BFF36F8FF0E748080020AA080020C2
:10FCE00038B583680446002B36D01E4A926893428A
:10FCF00035D1DA7B013ADA73C368012B05D0013BB9
:10FD0000C36000F0D9F8002038BD4FF02003EFF3B6
:10FD1000118583F31188BFF36F8F0169806890F9B3
:10FD20000E30994201D000F0F9FA204602F063FB50
:10FD3000A06058B190F90E2022610022C26702F043
:10FD4000FFFA2946084800F053F8DAE7E06085F347
:10FD50001188BFF36F8FD4E76FF01500D4E74FF031
:10FD6000FF30D1E748080020AA08002010B5084C51
:10FD700023685BB1FDF760FF2268064910444861C3
:10FD8000BDE810400021104602F08BBB10BD00BF43
:10FD90008408002048080020F8B50C464FF02003E6
:10FDA000EFF3118583F31188BFF36F8F4FF4004198
:10FDB00040F2E73600270022E1FB0067094B30469E
:10FDC0005A6139464FF47A720023FCF737FB064B31
:10FDD0001860064B1C60FFF7C9FF85F31188BFF35D
:10FDE0006F8FF8BD4808002084080020800800209C
:10FDF00049B9EFF3058030B9054B9A6A9B689A427E
:10FE000001D0FEF7CBBA81F31188BFF36F8F704733
:10FE1000480800204FF02003EFF3118183F311888D
:10FE2000BFF36F8F044B9A68D37B013BD37381F38D
:10FE30001188BFF36F8F704748080020094B03F10A
:10FE40002C02824205D19B688B4202D14B7BDB06A0
:10FE500006D1D1E9003213605A600023C1E90033B2
:10FE6000704700BF4808002038B5124C014623698E
:10FE7000A2680BB1E5680CE004F12C0002F056FA20
:10FE80000546537B980644BF43F008035373002D87
:10FE9000F0D049B9537BDB0606D1AB6923B9D389CE
:10FEA0007F2B01D9A26238BD954201D0FFF75EFFDA
:10FEB000A562F8E74808002010B54FF02003EFF3E3
:10FEC000118483F31188BFF36F8F084B00209A6869
:10FED000D37B0133D373FFF7C7FF84F31188BFF3DC
:10FEE0006F8FBDE8104002F00BBA00BF4808002039
:10FEF00070B490F90D20437B002A2CDBDB062AD15D
:10FF0000836943BB154A114651F82C4F8C4218BFE8
:10FF10002346002B38BF0023146BB3B190F90E6059
:10FF200093F90E50AE4203DBA3420ED01B68F4E7F8
:10FF30005A68C0E9003210605860437B63F07F0369
:10FF4000437370BC0020FFF78FBFC0E90014136B30
:10FF500018601063F1E770BC704700BF48080020CC
:10FF600010B54FF02002EFF3118482F31188BFF334
:10FF70006F8F427B510704D484F31188BFF36F8FD6
:10FF800010BD22F004024273FFF7B2FF2146BDE824
:10FF900010400148FFF72CBFAA08002070B590F967
:10FFA0000D300146002B02DA1748FFF747FF174ACA
:10FFB000104650F82C3F146B834208BF0023002BDF
:10FFC00038BF0023D3B191F90E6093F90E50AE42C1
:10FFD00003DBA34212D01B68F4E75868C1E9003084
:10FFE000016059604B7B906863F07F034B73431A49
:10FFF00058425841BDE87040FFF736BFC1E90004E0
:020000040001F9
:10000000136B19601163EDE77408002048080020A5
:10001000014670B54FF02003EFF3118483F311888C
:10002000BFF36F8F164B174A98681568A8421D4694
:1000300006D1FFF79BFE84F31188BFF36F8F70BD6D
:1000400000261660104A1268BAB1C2897F2A14D8F5
:10005000427BD20611D10D4A90F90E601268964289
:100060000BDB0B4A904208D05A698A4202DCFFF748
:1000700095FFDEE7521A5A61DDE700236B61DAE78C
:10008000480800207C080020840800208008002008
:100090005801002070B50446183002F0DCF94FF02A
:1000A0002003EFF3118683F31188BFF36F8F94F968
:1000B0000D30002B07DA21460E48FFF7BFFE637BA9
:1000C00003F07F0363730C4D637BA86843F0100358
:1000D0006373031B58425841FFF7C6FE86F311882D
:1000E000BFF36F8FAB68A34203D1BDE8704002F04D
:1000F00007B970BD74080020480800202DE9F041C0
:1001000004464FF02003EFF3118283F31188BFF30D
:100110006F8F437B13F0280F05D082F31188BFF354
:100120006F8FBDE8F08143F02003437382F31188A1
:10013000BFF36F8F183002F08EF94FF02003EFF30A
:10014000118683F31188BFF36F8F637BD80616D1B6
:10015000A269A2B9190607D521462648FFF76EFE07
:10016000637B03F07F036373234B9868021B504249
:100170005041FFF779FE002704F130081DE09B078E
:10018000F9D52146A068FFF759FE637B23F00203EF
:1001900063730023A360EEE705F1180002F05BF93A
:1001A000A8682946FFF74AFE6B7B284623F0020326
:1001B0006B73AF60EF67FFF79BFE256B454501D082
:1001C000002DE9D10C4B9A680C4B9A4202D10120C8
:1001D000FFF74AFE637B43F008036373236E86F3E5
:1001E0001188BFF36F8F002B9BD02046BDE8F041F4
:1001F000184700BF7408002048080020580100205C
:1002000008B590F90D300146002B06DA0748FFF7D4
:1002100015FE4B7B03F07F034B73054B9868431A25
:1002200058425841BDE80840FFF71EBE7408002040
:10023000480800202DE9F041064614461D464FF0BF
:100240002003EFF3118783F31188BFF36F8F02F060
:10025000A7F887F31188BFF36F8F6B1C08BFB4F149
:10026000FF3F08D022462B4606F118000349BDE89F
:10027000F04100F06FBABDE8F08100BF61230100DA
:1002800010B50C46064B11469868064B1860DDE920
:100290000223FFF7CFFF2046BDE81040FEF77EB8EF
:1002A000480800207C080020F7B50546019102F0BF
:1002B00013F904464FF02002EFF3118782F31188FF
:1002C000BFF36F8F124E134AB0681060FFF798FFAC
:1002D000B06811492A46019B183000F03BFAB26819
:1002E0003846537B43F010035373FEF757F86019F9
:1002F000044602F0F1F80025241A65F10005002CEF
:1003000075F10003B8BF0024204603B0F0BD00BF64
:10031000480800207C080020612301002DE9F041FD
:1003200004464FF02003EFF3118883F31188BFF3E5
:100330006F8F437B4EB2DB062ED1856965BB184FAC
:10034000214607F12C00FFF779FDFB6A3A6B8342E7
:1003500018BF1D46002D38BF0025A673B5B195F90D
:100360000E10B14203DCAA4210D02D68F6E76A688D
:10037000C4E9005214606C600120FFF775FD012094
:1003800088F31188BFF36F8FBDE8F081C4E90002E4
:100390003B6B1C603C63EFE70020A673F0E700BFF7
:1003A000480800200021044B084603F12C02C3E951
:1003B0000B22FFF7F1BC00BF48080020F8B5244C21
:1003C000244BA2689A4230D04FF02003EFF31185FE
:1003D00083F31188BFF36F8FA16804F12C00FFF73E
:1003E0002DFDE36AA268834208BF0023002B38BFBB
:1003F0000023216B2BB392F90E7093F90E60B74274
:1004000003DB8B421DD01B68F4E75968C2E9003159
:100410000A605A60537B012063F07F035373FFF738
:1004200023FD85F31188BFF36F8F4FF02003EFF3A7
:10043000118083F31188BFF36F8FBDE8F840FDF79B
:10044000ADBFC2E90001236B1A602263E2E700BF7F
:100450004808002058010020B1F1FF3F08BFB0F16B
:10046000FF3F08B502460B4606D10B4B9868FFF7D5
:1004700011FE4FF0FF3008BD13430AD1FFF79EFF76
:1004800000204FF47A7380FB0323D00B40EA4340F3
:10049000F1E7FFF709FFF4E748080020014B9868EF
:1004A000704700BF4808002038B504464FF02003CD
:1004B000EFF3118583F31188BFF36F8F01F09BFF7A
:1004C00048B10022C26701F03BFF2946BDE8384031
:1004D0000448FFF78DBCD4E902329A4218BF0133B9
:1004E000A360F2E7AA08002037B514461D464FF076
:1004F0002003EFF3118183F31188BFF36F8F8368BB
:1005000043B1013B836081F31188BFF36F8F0020FB
:1005100003B030BD54EA050306D181F31188BFF35F
:100520006F8F6FF00F00F3E70246CDE900450248F8
:10053000FFF7A6FEECE700BFAA0800202DE9B041B6
:1005400000F1300585B0C0E90C550E9D04460573D9
:10055000042545730D9D07328573002522F007029F
:10056000C0E91A1201EB02080C9AC0E90655C573DE
:10057000056702920B9A01920A9A00924246FDF791
:1005800097FF054BC4E917559B6803B15B6F404665
:10059000636705B0BDE8B081480800202DE9F04749
:1005A0002A4E2B4DB04686B0B54205F1300410D32B
:1005B000FFF730FC4FF4004940F2E7360027244CA7
:1005C000DFF890A0444521D306B0BDE8F047FFF71F
:1005D00073BC54F8043C059354F8103C049354F84D
:1005E000143C039354F8183C029354F81C3C0193B8
:1005F00054F8203C009354E90A2354E90C01FFF716
:100600009DFF54F8303CDD652546CDE7636A5A1CF2
:100610000DD03046394623EAE373C9FB0301B942E2
:1006200008BFB042256804D12846FFF799FC303452
:10063000C8E74FF47A720023FBF700FF02460B462F
:1006400005F11800514600F085F8F0E7040100209C
:10065000040100206123010008B54FF02003EFF3EF
:10066000118483F31188BFF36F8F044B986818616E
:10067000FFF710FD2046FDF791FE00BF480800205F
:1006800008B50648064A0749121A01F03BFDBDE8C5
:100690000840054A0549064801F034BD0000002025
:1006A00054010020002E010000000000002E010077
:1006B00000000020034B1B680BB9FDF7BDBA0020FA
:1006C000704700BF8808002030B5036868B10A4A47
:1006D0005268904209D043B1D3E90421D0E90445DE
:1006E000121945EB0101C3E90421426813605A6005
:1006F0000023C0E9003330BD58000020134B10B573
:100700001C689C4208BF0024FFF7D4FFCCB1D4E999
:100710000423121A63EBE073012A73F1000113DB67
:1007200010466FF0004219460023824273EB010429
:1007300000DA1046064B5B6913B19842A8BF184611
:1007400010BD6FF00040F5E70020F3E758000020EF
:10075000480800202DE9F74F019119464B1C08BFAE
:10076000B2F1FF3F824670D06FF001034FF0FF3BC4
:10077000541C41F10005B3EB04086BEB0509B8F11B
:10078000000F79F100030FDBFFF794FF6FF0010317
:10079000344AD2E9001C5B1A6BEB0C021E1B62EBA5
:1007A0000507341A67EBE075019BCAF808304FF073
:1007B0002003EFF3118683F31188BFF36F8FFFF7E8
:1007C00079FF012C75F10003BCBF01240025264BE5
:1007D00024181A6845EBE0759A42CAE9044501D02D
:1007E0005F6852B95A68CAF80030CAF804205A68DB
:1007F000C2F800A0C3F804A014E0D2E90489DAE941
:100800000445444575EB090122DAB8EB040069EBB5
:100810000501C2E904015168CAE90021C1F800A03C
:10082000C2F804A01A689A420BD0924509D1FFF78A
:1008300065FF18B10D4B5B69834202D00021FDF7C3
:10084000C9F986F31188BFF36F8F03B0BDE8F08F4D
:10085000B4EB080065EB0901BA42CAE90401C1D052
:100860001268BEE758020020580000204808002007
:100870002DE9F74F0646FFF7CBFB4FF02003EFF3D0
:10088000118483F31188BFF36F8FDFF8B0A02A4D76
:100890005146DFF8ACB02E60D5F800C0DBF80000A0
:1008A0006246DAE90089D3175845CDE900230DD017
:1008B00060B1D0E90467B445BB411DDA009BB6EBDB
:1008C000030C019B67EB0306C0E904C60026009BEE
:1008D0002E6013EB0802019B43EB0903C1E90023DF
:1008E000FFF70CFF3146FDF775F984F31188BFF36C
:1008F0006F8F03B0BDE8F08F0022002318EB0608CD
:1009000049EBE679C0E90423ACEB0606CAE90089A5
:100910002E60FFF7D9FE84F31188BFF36F8F8368D1
:1009200098474FF02003EFF3118483F31188BFF34E
:100930006F8F0249B0E700BF8808002058020020EE
:100940005800002010B54FF02003EFF3118483F31B
:100950001188BFF36F8FFDF76FF9064BD3E90023C2
:10096000121843F1000384F31188BFF36F8F104610
:10097000194610BD5802002038B5064C064DAC4251
:1009800001D3002038BD2046D4E9011201F0A8FDB2
:100990001434F4E7040100200401002001F09BBBA3
:1009A0000A46002101F0D9BB10B5114800F048F803
:1009B00000B110BD0F4800F043F80028F9D10E4CEB
:1009C000204600F03DF80028F3D10C4B0C481C6089
:1009D00000F036F801460028EBD100F02DF804466F
:1009E00008B1204610BD00F051F82046FAE700BFDC
:1009F0006C000020600000206800002070000020D3
:100A00006400002008B5084800F024F8074800F00A
:100A100021F8074800F01EF8064800F01BF8BDE872
:100A2000084000F00BB800BF6C0000206000002000
:100A3000680000206400002000207047704700BF5D
:100A400008B5034B02681B6810689847002008BD72
:100A50008400002008B5034B02685B681068984763
:100A6000002008BD84000020024B02689B681068CB
:100A7000184700BF8400002008B5034B0268DB68FC
:100A800010689847002008BD8400002070B5094C0C
:100A9000094D2069AB68984718B1084B08485B6856
:100AA00098470021074AEB6811602069BDE8704053
:100AB000184700BF9400002084000020740000202C
:100AC000502901008C08002070B51A4D1A4E0446BA
:100AD000B26828699047F0B95CB1184C2368ABB193
:100AE000012B1AD0013B23602869F3689847002046
:100AF00070BD124C216839B90120114B114AC3F85D
:100B000000051368002BFCD101312160F3682869CE
:100B10009847002070BD0C4870BD0A4A1368002B2E
:100B2000FCD1074A6FF07E40C2F8003500F020F893
:100B30002368D7E794000020840000208C08002060
:100B40000000845010198450E98FFFFF0020704787
:100B500000207047430503D54FF0FF32024B1A6067
:100B6000024B1860704700BF08118450081A845067
:100B7000014B1860704700BF041A845008B100F0A0
:100B800003B84FF4750070470246074803681342E4
:100B9000FCD021B1054B06481B680B600360054B78
:100BA00000201A60704700BF001A8450041184505E
:100BB00008118450081A845000F09EB838B131B141
:100BC000002201440346013081421A70FAD1704775
:100BD0002DE9F041ADF51A7D0E460592002114462F
:100BE00012A84FF408721D4601F0B7FA002128221E
:100BF00008A8069101F0B1FA002E3CD0002D3AD0A1
:100C0000002C38D0042106A8FFF7CAFE08A8282126
:100C1000FFF7C6FE08A800F031F878B14FF0FF37B3
:100C20004FF4087112A8FFF7C9FF042106A8FFF7C7
:100C3000C5FF38460DF51A7DBDE8F08112AB0DF108
:100C40001C080246CDE90153039005AB08A9CDF875
:100C5000008006A800F02AFD0028DFD12B68A342FF
:100C6000DCD3D8F800100746224630460831FFF79B
:100C700095FE2C60D4E74FF0FF37DAE71C2330B540
:100C800083B001A90446019300F0E4F9054638B9A0
:100C9000019B1C2B07D0164D20461C21FFF780FE20
:100CA000284603B030BD0121D4E90032003B18BF13
:100CB0000123E1610AB143F00203A26832B9E2689C
:100CC00042B9C4E908328BB90A4DE5E7E26843F05E
:100CD00004033AB10022284643F00803C4E908326D
:100CE00003B030BD1546C4E90832D9E71546D7E749
:100CF000370CF0000E0CF00010B50C4C236813B14B
:100D00000B4B1B682BB900F065F930B90122084B79
:100D10001A6001230020236010BD0138062801D984
:100D2000044810BD044B53F8200010BD900800206B
:100D300094080020FE8FFFFF7029010010B50A4CB7
:100D400023681BB101230020236010BD00F0AEF822
:100D50000028F7D00138062803D8044B53F82000A8
:100D600010BD034810BD00BF90080020702901008D
:100D7000FE8FFFFFBFF34F8F0549064BCA6802F491
:100D8000E0621343CB60BFF34F8F00BFFDE700BFAE
:100D900000ED00E00400FA054FF0FE33002130B40E
:100DA000064A074D074C2B6013602360064A074C28
:100DB000EB606368C2F8001530BC18470414845017
:100DC00000148450081484500000845074000020E3
:100DD000024BD0E90012C3E90012704774000020F2
:100DE00048B143682BB1BFF35F8F002303601846FF
:100DF0007047024870476FF4E0407047EA8FFFFF8A
:100E000010B5044628B1636813B100232360636002
:100E100010BD024B02485B689847F4E7740000205D
:100E20008C29010010B5044630B1002263682260AD
:100E300043F00103636010BD0148FFF7ADFFF4E725
:100E4000B429010080B1436863B10122D0E8EF3FCB
:100E5000C0E8E12F0029F9D1012BF7D0BFF35F8F54
:100E600000207047024870476FF4E040704700BFB1
:100E7000EA8FFFFF70B40B4B0668C268D0E90154DB
:100E8000C3E90242C3E90065D1E903020E68064BDB
:100E9000D1E90154C3E90065C3E902401A6170BC9D
:100EA000704700BF840000209400002010B5FFF7B9
:100EB0004DFE20B10324FFF7A5FD204610BDFFF72E
:100EC00073FD90B9FFF700FE90B90F4B1B681B0E26
:100ED000F02B08D10D4A0E4B12689A420AD0072413
:100EE000FFF736FEE7E70624FAE70424204610BDA4
:100EF0000024F5E70120FFF7E7FD04460028F7D1BD
:100F0000044B1860D9E700BF28198450241A845074
:100F10000000E0200C1A845030B5ADF5157D4FF47B
:100F2000087200210CA801F018F90021282202A85B
:100F3000019101F012F902A8FFF7A0FE20B10524EB
:100F400020460DF5157D30BD1D4D4FF0FF31286851
:100F5000FFF78AFD0446E8B90020FFF7B5FD58BB4E
:100F60000CAA02A901A800F0EDFB04460120FFF73E
:100F7000ABFDE8B92868FFF77FFD28B9002CDED16A
:100F800020460DF5157D30BD0E48FFF705FF002CFE
:100F9000F6D0D4E70C48FFF7FFFE012CDCD128681F
:100FA000FFF76AFD0028CAD00648FFF7F5FEC6E73E
:100FB0000648FFF7F1FEDDE70548FFF7EDFECFE756
:100FC00070000020F0290100D8290100282A010022
:100FD000082A010008B5FFF7B9FD18B1FFF712FDA7
:100FE000032008BDFFF7E0FCC0B9FFF76DFDB8B9FD
:100FF000144B1B681B0EF02B0AD1134A134B1268BB
:101000009A4217D0FFF7A4FDFFF7FCFC072008BDAC
:10101000FFF79EFDFFF7F6FC062008BD042008BD83
:10102000FFF796FDFFF7EEFCFFF776FF002818BFED
:10103000052008BD0120FFF747FD0028F0D1044B33
:101040001860F1E728198450241A84500000E02029
:101050000C1A8450002866D0002964D00B681C2B21
:1010600061D14FF47F033B4AD3F8101C91425CD00E
:10107000D3F8102C013258D0D3F8102C4FF47F0342
:101080000260D3F8141C344A914260D0D3F8142C77
:1010900001325CD0D3F8142C4FF47F034260D3F8B4
:1010A000182C12F5947F4FD0D3F8182C01324BD066
:1010B000D3F8182C4FF47F038260D3F81C1C274A06
:1010C00091423ED0D3F81C2C01323AD0D3F81C2CDC
:1010D0004FF47F03C260D3F8002C70322FD0D3F8C6
:1010E000002C01322BD0D3F8002C4FF47F03026187
:1010F000D3F8042CAF3220D0D3F8042C01321CD00A
:10110000D3F8042C4FF47F034261D3F8081C144A2F
:1011100091420DD0D3F8082C013209D0D3F8083C05
:101120008361002070470120704740F6FC02A5E76C
:1011300040F237338361002070475122E2E790226A
:10114000D3E742F60412C3E740F6D862B2E742F2B0
:10115000D002A1E7FCF8FFFFD020FFFF0429FFFF2A
:1011600037F3FFFF2DE9F843002877D00C4600291C
:1011700074D01D46002B71D006461AB101220023FF
:101180002A6003602B68002B64D02946204600F0BB
:1011900015FB074600285ED12146286800F0F0FACA
:1011A0000746002857D12B68082B66D0042B67D040
:1011B000A3F10208B8FA88F84FEA581801239C46B0
:1011C000314A3249136010460B60943AC0F800C0AF
:1011D000636A136011688B42F8D14FF000092C4B01
:1011E0004FF0FF30C3F80090FFF7B4FC294B2A4AB8
:1011F00048461A60FFF7BCFC284A294BC2F8008019
:10120000186840F48060FFF7B3FC0A22254B1A608F
:10121000089A2369012A616A24D0234AA2FB032386
:101220001B09012203FB01F303EB43031F49DB030B
:101230009B090B60164B38461A6033682A6823F006
:101240007F4343EA026333602A6843EA0223336040
:10125000BDE8F883164F3846BDE8F883154F384689
:10126000BDE8F8834FF47F03D3F80C2C013202D091
:10127000D3F80C3CD1E71623D3E74FF003089DE7E2
:101280004FF002089AE700BFC41184504011845007
:101290002C11845000118450FEFFFF0F0C1184505C
:1012A000041A845038118450ABAAAAAAD8118450C9
:1012B000310CF100350CF100F0B40024C9002646D1
:1012C000274601F1FF3C06E09F4215D00126654507
:1012D00018D82C461F46630950F8233004F01F012C
:1012E000CB401F2904F1010518BF03F00103002CB6
:1012F000EAD101263546ECE701369642E7D10348AC
:10130000F0BC70470020F0BC704700BF360CF10005
:1013100000285FD02DE9F0414C1EB4F5047F26D2A1
:101320002BB322B3CC00012B04F1FF3E2FD00021C0
:101330008C460F460D4603F1FF384C0950F8244007
:1013400001F01F06F4401F2E18BF04F0010421B95C
:101350000125AC4629462746EFE7AB4213D0A7420A
:1013600001D10CF1010C454504D1624502D21A4865
:10137000BDE8F0813C4601318E4505F10105EAD218
:101380000020BDE8F08100254FF0010CF3E70026B6
:10139000B446374631464B0950F8233001F01F055B
:1013A000EB401F2D18BF03F0010339B15FB99C4515
:1013B00001D0634608E06346013605E00126314668
:1013C0009C460127E7E73E46B242D0D30131A14215
:1013D000F6D1D5E700487047370CF1002DE9F04F02
:1013E0008DB0189E07460C46179D002E4CD1D1F8A3
:1013F00010B000211D60169B1960002A00F01E81AC
:101400009A4A9B4B1168626A1B689A4247D10A2923
:1014100045D1FB7804930423B8460293954BA3FB74
:101420000B234FEA930A0AEB4A0305F108020392E1
:10143000ABEB430A169BC3F800B0BBF1000F00F002
:10144000C3805D464FF00009039E00F0C7F90023FA
:101450000593B8F1000F00F0E580002C00F0E28069
:10146000049B002B00F0DC80204604A900F0A6F9C4
:10147000B8B1814B984240F0A780029000F0AEF9DD
:1014800002980DB0BDE8F08F4FF47F01D1F80C0C3D
:1014900001300CBF4FF4047BD1F80CBCA9E77748AE
:1014A000EBE72146049800F06BF90028E1D1049F96
:1014B000082F00F0B980042F00F0B880A7F10207D0
:1014C000B7FA87F77F09012319466D48036040F892
:1014D000843C6B4B66481960636A03600068834212
:1014E000F7D10023674A4FF0FF301360FFF732FB5C
:1014F000002365491846654B1960FFF739FB6449BD
:10150000644B0F6018685B4F40F48060FFF730FB5E
:101510000A210122554B604819602169636AA7FBC3
:1015200001C1090903FB01F303EB4303DB039B093F
:101530000360544B05A81A600499D8F800200B02E8
:1015400043EA016322F07F421343C8F8003000F001
:1015500007F900288DD1514BA7FB05271A681433D2
:10156000069253F8102CB9EB970F079253F80C2CF6
:10157000089253F8082C099253F8042C0A921B681D
:101580000B9302D1BAF1000F41D1182230460DEB76
:101590000201FFF703FA183D183609F10109002D81
:1015A0007FF453AFBBF5047F5DD8039D59462846B1
:1015B0006269FFF781FE00284BD00023169A136062
:1015C0002D4B98423FF459AF049D082D34D0002292
:1015D00004AB214640466D0000920495FFF7C2FD22
:1015E0002F4B984224D000287FF447AFD8F8002032
:1015F000130A03F47F03134323F07F43C8F800303A
:10160000029B013B02937FF415AF002035E7304683
:10161000524606A9FFF7C2F9A5EB0A055644BCE7F6
:101620001F4826E71F4824E703274CE702274AE71D
:10163000236A002B3FF421AF1B481EE701222146FD
:101640003846009604ABFFF78DFD00283FF4E3AE6B
:1016500013E74FF4806359462846A269FFF758FE06
:101660000028AAD1D1E7169B1D60ADE73811845040
:1016700030118450ABAAAAAA020CF100300CF10080
:10168000C41184502C118450FEFFFF0F00118450B0
:101690000C118450041A8450D811845014118450B1
:1016A000310CF100350CF100320CF1002DE9F04164
:1016B0001F4E84B004460D4630684FF0FF3190460F
:1016C0000C9FFFF7D1F9D8B90020FFF7FDF9F8B961
:1016D00000230B9A204600920293424629460A9B19
:1016E0000197FFF77BFE04460120FFF7EDF9D0B923
:1016F0003068FFF7C1F978B9204604B0BDE8F08141
:101700000C48FFF749FB0020FFF7DEF90028DFD087
:101710000948FFF741FBDBE70848FFF73DFB2046A0
:1017200004B0BDE8F0810648FFF736FBE0E700BFF4
:1017300070000020D8290100082A0100F0290100CA
:10174000282A010010B5012486B005ABCDE901249B
:101750000093002204ABFFF741FE06B010BD00BFAE
:10176000014608B54FF48060FFF708FA00230249EC
:10177000024A0B60136008BDC81184502C118450BC
:101780000138072805D8DFE800F00A0E0412040427
:10179000040609487047CB6800204B6270470B680D
:1017A00000204B6270474B6800204B6270478B688B
:1017B00000204B62704700BF310CF1000B6802E063
:1017C000082B0B6006D8026A13424FEA4303F7D096
:1017D0000020704700487047310CF1000023044995
:1017E000044A0B604FF480601360FFF7B3B900BF89
:1017F0002C118450C411845008B5FCF781FBBDE85E
:101800000840FCF711BB60B1436803F00303012BF0
:1018100003D0032B05D103681BB100238360184656
:1018200070476FF01500704700224368816003F035
:101830000303032B14BF1346036842601846704726
:10184000002070470FB407B504A951F8040B0191AB
:10185000FAF7A4FF03B05DF804EB04B07047038B04
:1018600013F0070305D10368002B0CBF00200320F1
:101870007047022B05D1438B002B14BF002004209E
:101880007047012B05D10368002B0CBF00200520F9
:1018900070470020704773B50D4606461946281D4F
:1018A00001920093FFF7C0FF044640B1DDE900322A
:1018B00029463046A44602B0BDE87040604702B0F9
:1018C00070BD10B44FF02004EFF3118284F311883F
:1018D000BFF36F8F41615DF8044B0121FAF76CBFD4
:1018E00010B50C4640B139B1081DFFF78CFF28B97F
:1018F000A36833F0030301D06FF0150010BD38B5B5
:101900000C46054658B151B10B6843B14B6833B131
:101910001C22002100F021FC00202C6138BD6FF05A
:101920001500FBE770B504460E46FFF7D9FF051E0C
:1019300031DB4FF02003EFF3118183F31188BFF304
:101940006F8F4FF6FF75638B208BAB4200F0070261
:101950002ED0022A0ED1013363831546012381F371
:101960001188BFF36F8FB3B1002331462046FFF7D4
:1019700092FF10E0830701D0062A0ED100233360C6
:10198000636893B9C4E90066154662B90A46204601
:101990000221FAF711FF284670BD052A0CBF6FF02F
:1019A00022056FF004050023D9E71E606660EBE7AF
:1019B0006FF00A05F7E7044608B5084611461A46CF
:1019C000A047FEF76BFDFCF7CBFF836800EBC1017E
:1019D000B3F5004F2CBF51F8220031F812007047C8
:1019E00000EBC1018068B0F5004F2CBF41F82230F8
:1019F00021F812307047012208B5FFF7E6FF4008D2
:101A000008BD836800EBC101B3F5004F08D34B68F4
:101A10001AB143F001034B60704723F00103FAE76A
:101A20004B881AB143F001034B80704723F0010348
:101A3000FAE753000122FFF7D3BF80680131B0F508
:101A4000004F2CBF02200120081AB0FA80F0C0F12C
:101A50001F0070472DE9F04104460D46FFF7CBFF0C
:101A6000A3680146B3F5004F01D3012835D02046C5
:101A7000FFF7E3FF04EB800216699EB9012303FA26
:101A800000F0E36829460343E360204615612B46D6
:101A90000222FFF7A5FF032229462046BDE8F041B8
:101AA000FFF79EBF022231462046FFF78EFF074612
:101AB0000346022229462046FFF792FF33460322BF
:101AC00029462046FFF78CFF032239462B46204645
:101AD000FFF786FF02223146DFE7BDE8F081B2F56D
:101AE000802FF8B52CBF082504250023551B0022A4
:101AF000CC1D24F007040460C4E9002300230D4436
:101B000025F007052D1BED0829462046A560E3605A
:101B1000FFF793FF8600411C18461B36F60804F1B8
:101B200010028B4229DB324620460021FFF781FF5D
:101B3000AF1B204601220021FFF763FF3A463146E2
:101B4000FFF777FF3346314620460022FFF748FF74
:101B5000294620460022FFF76CFF3B4629462046D7
:101B60000022FFF73DFF294620460122FFF749FFEB
:101B70003146BDE8F840FFF76DBF42F8040B013372
:101B8000CFE72DE9F048D0E900244FF03333A2FB32
:101B900003BC1BEB03064CEB03052F460026A4FBFE
:101BA00003451BEB04024CEB0501D219324646EB10
:101BB0000101631845EB0202C0E90032BDE8F0887C
:101BC0000B6870B5002B10DD013B0B600A21026829
:101BD0004468A2FB015601FB046626F07043C0E98D
:101BE0000053310F3031084670BD3021FBE72DE93D
:101BF000F74F9946D37814466F2BA3F1410206465E
:101C00000F4601922DD028D8582B14BF0A25102535
:101C1000AA464FF0000BDDF8308052465B46304656
:101C20003946FAF70BFC092AD3B21FD830335F4587
:101C3000DBB208BF564508F8013D01D3C84512D8AC
:101C400023789B0605D5082D16D1A37843F0080309
:101C5000A370404603B0BDE8F08F03F0F703702B8C
:101C6000D3E70825D4E706460F46D6E7019A192A96
:101C700094BF37335733DAE7102DEAD1A37843F016
:101C80001003E5E72DE9F8438046894616461F46CE
:101C90001546BD42A5EB060405D30FB1204608E06A
:101CA0002B78002BFAD0494615F8010BC0470028C5
:101CB000EFDABDE8F8837047FDF7C0B9CBB20C216D
:101CC000C26803FB0121086C00F0070070474FF069
:101CD0002003EFF3118283F31188BFF36F8F036842
:101CE00013F0C00301D08B4207D101230360002011
:101CF00082F31188BFF36F8F70474FF0FF30F7E723
:101D000010B54FF02003EFF3118283F31188BFF376
:101D10006F8F036803F00704012C06D101600020D7
:101D200082F31188BFF36F8F10BD03F0C0038B42A5
:101D300014BF4FF0FF306FF04400F1E74FF0200385
:101D4000EFF3118283F31188BFF36F8F036803F001
:101D5000C00343F00203036082F31188BFF36F8F67
:101D6000704710B41C24C068CBB203FB04000021F0
:101D70005DF8044B10470020FDF72ABA0020FDF75C
:101D800059BA1046FEF790BB38B50C23CCB263436A
:101D90000546C068403380211844FFF798FF0028AB
:101DA00005DB696801EBC40463689847002038BD0F
:101DB0002DE9F8430C27CDB26F43C468064607F1FE
:101DC00040008021204490469946FFF799FF002863
:101DD00007DB3C44C4E90E89736853F835309847F3
:101DE0000020BDE8F88370477047704700F01F027D
:101DF0001F210420FBF758BF00F007020721022033
:101E0000FBF752BF024601210720FBF74DBF4001FF
:101E100000F0E002E0211520FBF746BF18223F2129
:101E20002A20FBF741BF400000F0FE0202212920DA
:101E3000FBF73ABF13223F212C20FBF735BF0246A8
:101E400001212B20FBF730BF002307B501A88DF837
:101E50000430FEF7B1FE03B05DF804FB70B5064632
:101E60000C46154600F006F9012836D16FF0150032
:101E7000BDE87040714672467346B7EE000AF7EE51
:101E8000000AB7EE001AF7EE001AB7EE002AF7EED6
:101E9000002AB7EE003AF7EE003AB7EE004AF7EE46
:101EA000004AB7EE005AF7EE005AB7EE006AF7EEB6
:101EB000006AB7EE007AF7EE007A8EF3008C10B469
:101EC000F1EE10CA4FF66074C0F6FF740CEA040C11
:101ED000E1EE10CA10BCF4467447284600F0CAF878
:101EE0000128C3D0902CC1D12B4622463146002078
:101EF000FEF76EFEBCE738B505460C46B1BB6FF089
:101F00001500BDE83840714672467346B7EE000AC8
:101F1000F7EE000AB7EE001AF7EE001AB7EE002A45
:101F2000F7EE002AB7EE003AF7EE003AB7EE004AB5
:101F3000F7EE004AB7EE005AF7EE005AB7EE006A25
:101F4000F7EE006AB7EE007AF7EE007A8EF3008CB7
:101F500010B4F1EE10CA4FF66074C0F6FF740CEACC
:101F6000040CE1EE10CA10BCF446744700F082F88D
:101F70000128C4D1204600F07DF80128BFD02846B2
:101F8000FCF756F8014628B13C22204600F0BAF88A
:101F90000020B6E76FF00D00B3E70020FBF7C8BBE9
:101FA0000021012000F032B843B2C9B9002B15DB83
:101FB00001215B099B0003F1604303F56143D3F802
:101FC000802200F01F00814022EA0102C3F8802233
:101FD000D3F88012C14001F00101C9B20846704730
:101FE000002B0DDB01225B099B0003F1604303F52D
:101FF0006143D3F8801200F01F0082400A43E5E7F6
:102000000021EBE7836E83F30B88704700F02CB957
:102010000146006800F028B908B5FCF7A1FABDE850
:102020000840FCF73BBC7FB50A898E7A0B684D6887
:1020300002F01F0242EA461200938DF8082023F0B6
:102040001F036A1E134423F01F030F28039304D8B1
:102050006946FCF7C3FC04B070BD6FF01500FAE7E9
:1020600040E800F0C3B210F4803F14BF18466FF090
:102070001500704740E800F0C0F3805070470346F9
:1020800000201A5C02B970470130FAE703460020CD
:102090001A5C0AB1884200D170470130F8E7013874
:1020A000013910F8013F11F8012F934201D1002BA3
:1020B000F7D1981A704710B55AB10139841810F841
:1020C000012B11F8013FA04201D09A42F7D0D01A5B
:1020D00010BD1046FCE7431A934210B500EB020313
:1020E00008D3024601399A420BD011F8014F02F889
:1020F000014BF8E70A4412F8014D8A4203F8014DFA
:10210000F9D110BDF0B581EA0004A50703460BD054
:10211000013B0A4491421BD1F0BD002AFCD011F8CA
:10212000014B013A03F8014B9C07F6D122F003045E
:102130001D1F96080F19B94205D16FF003052344FE
:1021400005FB0622E4E751F804CB45F804CFF2E79B
:1021500011F8014B03F8014FDCE7034670B5C9B233
:102160009C0711D141EA012422F0030644EA044508
:102170001E449408B3420DD16FF0030505FB042201
:102180001A44934209D170BD002AFCD003F8011B08
:10219000013AE5E743F8045BECE703F8011BF0E7DD
:1021A000CA07436805D4C1F34202012A04D0022AB7
:1021B0000BD06FF0150070474FF0CC721B68C3F85E
:1021C0002425C3680020596270474FF0C8621B681D
:1021D000F5E7002008B5FCF76FFB08B5FCF71CF825
:1021E000FCF7C6F8BDE80840FEF7A8BD004700F0C0
:1021F0002DB908B50520FCF737F920B9BDE808402E
:102200000520FCF721B908BD0B7B032B2AD8DFE89A
:1022100003F022261A028B685A0304D5D0F84C35F5
:102220000A699A4207D18B685B031BD4D0F84C35FE
:102230004A699A4216D000230622C0F80035C0F839
:10224000002518467047D0F84C350A699A42F2D1F9
:10225000D0F83C35ECE7D0F84C350A69E9E7D0F81E
:102260003C35FAE70120704773B5054601914FF000
:102270002003EFF3118683F31188BFF36F8FFEF70E
:102280000DF9019904462846FFF7A3FF86F311884C
:10229000BFF36F8F204602B0BDE87040FCF760BB13
:1022A000FFF7A2BD30B50024846141EA020414F0B6
:1022B0000304C0E9023201610CD14461A34203D19D
:1022C000C0E90000002030BD456901340D60416166
:1022D0001144F3E76FF01500F5E70023C0E90000B3
:1022E000C0E9023318467047034620B9EFF3058270
:1022F0000AB9FCF753B883F31188BFF36F8F7047A7
:102300004FF02003EFF3118083F31188BFF36F8F39
:10231000FFF7EABF014608B58068FDF78FFD4B7BEC
:1023200023F002034B7300238B6008BD03689842BF
:1023300004D0002B38BF0023184670470020704798
:1023400010B54FF02003EFF3118483F31188BFF32E
:102350006F8FFDF7CDFD84F31188BFF36F8F10BD34
:1023600037B504464FF02003EFF3118583F311884E
:10237000BFF36F8F54F8103C18381BB10190FFF772
:10238000C9FF019814F80B3C23F0140304F80B3C2C
:10239000FDF7AEFD85F31188BFF36F8F03B030BD3D
:1023A00038B504460D46FDF72BFF637B43F002036F
:1023B0006373C5B12B68A5609D4208BF0023002B45
:1023C00038BF002383B194F90E1093F90E20914287
:1023D00004DB6A689A4207D01B68F3E75A68C4E9CD
:1023E000003214605C6038BD6B68256063606B68A8
:1023F0001C606C60F7E738B54FF02003EFF31182F3
:1024000083F31188BFF36F8FFFF790FF044682F3C9
:102410001188BFF36F8F88B14FF02003EFF3118560
:1024200083F31188BFF36F8FFFF774FF85F3118873
:10243000BFF36F8F04F1180000F00DF8204638BD8F
:10244000EFF30580003818BF0120704708B1FBF793
:1024500065B97047704710B54FF02002EFF3118453
:1024600082F31188BFF36F8F03683BB1FEF72CF93D
:10247000002084F31188BFF36F8F10BD6FF015003B
:10248000F7E710B54FF02003EFF3118483F31188C1
:10249000BFF36F8FFEF732F984F31188BFF36F8FAC
:1024A00010BD37B5044601914FF02003EFF31185BD
:1024B00083F31188BFF36F8FFEF720F9012805DD44
:1024C000A042019902DD2046FBF784FB85F31188C9
:1024D000BFF36F8F03B030BD08B5FEF733FA08BD08
:1024E00010B400F10C04C0E903445DF8044BFFF79D
:1024F000F6BA7047789FFF7F01000000F5D6000014
:1025000000000000F5FA0000000000007909010059
:10251000000000006DEB00000000000001D800008A
:10252000C000002081DB0000D0000020DB21010082
:10253000E0000020B5ED0000F000002085EF000075
:102540000000000065ED0000000000000000000039
:10255000A11F010000000000A11F010000000000F9
:10256000A11F010000000000A11F010000000000E9
:10257000A11F0100B9F20000ED21010000000000E0
:10258000A11F010000000000A11F010000000000C9
:10259000A11F010000000000A11F0100F1F60000D2
:1025A000ED21010000000000A11F0100000000005B
:1025B000A11F010000000000A11F01000000000099
:1025C000A11F010000000000A11F01000000000089
:1025D000A11F010000000000A11F01000000000079
:1025E000A11F010000000000A11F01000000000069
:1025F000A11F01000000000031DB0000000000000E
:10260000A11F010000000000A11F01000000000048
:10261000A11F010000000000A11F01000000000038
:10262000A11F010000000000A11F01000000000028
:10263000A11F010000000000A11F01000000000018
:10264000A11F010000000000A11F01000000000008
:10265000A11F010000000000A11F010000000000F8
:10266000A11F010000000000A11F010000000000E8
:10267000A11F010000000000A11F010000000000D8
:10268000A11F010000000000A11F010000000000C8
:10269000A11F010000000000A11F010000000000B8
:1026A000A11F010000000000A11F010000000000A8
:1026B000A11F010000000000A11F01000000000098
:1026C000A11F010000000000A11F01000000000088
:1026D000A11F010000000000A11F01000000000078
:1026E000A11F010000000000A11F01000000000068
:1026F000A11F010000000000A11F01000000000058
:10270000A11F010000000000A11F01000000000047
:10271000A11F010000000000A11F01000000000037
:10272000A11F010000000000A11F01000000000027
:10273000A11F010000000000A11F01000000000017
:10274000A11F010000000000A11F01000000000007
:10275000A11F0100FFFFFFFFFFFFFFFFFFFFFFFFC4
:10276000DEE61E284CBBCE8F025B0000DEE61E2894
:10277000EAAC45B8025B0000DEE61E284CBBCE8FFB
:10278000025B0000000000000000000000000000EC
:102790000338FDD87047000041D90000891D0100B1
:1027A000B11D010000000000BD1C0100B9D80000EF
:1027B0001DD90000771D01007D1D0100A9D7000073
:1027C00061D7000000000000292C01004201000038
:1027D000302C0100050100003A2C0100140100001A
:1027E000432C0100150100004C2C010039010000B0
:1027F000552C010009010000602C01000A000000B6
:102800006B2C01000A010000752C01000B01000077
:102810007F2C01000F0100008A2C01001001000034
:10282000952C010011010000A02C01000E010000F8
:10283000AA2C010021010000B32C0100220100009C
:10284000BC2C010023010000C52C01002401000064
:10285000CE2C010018010000D62C01002A01000036
:10286000DE2C01003A010000E62C01002C010000E2
:10287000EE2C01001C010000F72C01001D010000DE
:10288000002D0100170100000A2D010004010000C5
:10289000192D0100310100000000000000020000BD
:1028A000000400000008000000100000000000000C
:1028B0009B1F0100B1E2000069E2000021E300007B
:1028C00025E200001C00002004000020140000206D
:1028D000000000000C0000200000002000000000AC
:1028E0000600010002000000EC28010000000000CA
:1028F000782D010006000000E0FF0F00000000201E
:10290000802D010021000000E0FF0020A121010036
:102910001DEE0000000000000000000000000000AC
:1029200000A00050000000000C0000000B000000A0
:102930000000400600000000FC24010024250100E6
:102940002C250100442501004C250100F5FFFFFF67
:10295000436F756C64206E6F74206C6F636B2070B6
:102960006F7765722073617665206D757465780088
:10297000FF8FFFFFFF8FFFFFFE8FFFFFFE8FFFFF29
:10298000FD8FFFFFFC8FFFFFFC8FFFFF6D757465F0
:10299000785F667265652063616C6C656420776939
:1029A0007468204E554C4C20706172616D65746581
:1029B0007200000043616E277420696E697469615A
:1029C0006C697A65206D757465782C207761732049
:1029D0004E554C4C0D0A00004661696C20746F2006
:1029E00061637175697265206D757465780A0000A0
:1029F0004661696C20746F2072656C656173652037
:102A00006D757465780A00004661696C20746F20EA
:102A1000696E63726561736520504D20636F756EDA
:102A20007465720A000000004661696C20746F20B2
:102A3000646563726561736520504D20636F756EC8
:102A40007465720A00286E696C29004661696C65BC
:102A50006420746F207265626F6F743A20737069BE
:102A60006E6E696E6720656E646C6573736C792E2B
:102A70002E2E0A007379735F636C6F636B0053656E
:102A8000637572650909004E6F6E2D53656375722B
:102A900065090025303275202530327520307825C3
:102AA00030357820307825303578200900256300CE
:102AB00053504D3A204E5320696D61676520617413
:102AC00020307825780A0053504D3A204E53204D3F
:102AD000535020617420307825780A0053504D3AC5
:102AE000204E5320726573657420766563746F722F
:102AF00020617420307825780A0053504D3A2070B8
:102B000072657061726520746F206A756D702074D3
:102B10006F204E6F6E2D53656375726520696D6110
:102B200067652E0A004E6F6E2D53656375726500E2
:102B3000466C61736820726567696F6E730909443A
:102B40006F6D61696E09095065726D697373696FA4
:102B50006E730A004E6F6E2D736563757265206328
:102B6000616C6C61626C6520726567696F6E2030A4
:102B700020706C6163656420696E20666C617368A7
:102B800020726567696F6E202564207769746820FC
:102B900073697A652025642E0A00436F756C642082
:102BA0006E6F7420696E697469616C697A652073EF
:102BB0006563757265207365727669636573202835
:102BC000657272202564292E0A005352414D2072ED
:102BD0006567696F6E0909446F6D61696E09095017
:102BE00065726D697373696F6E730A0050657269FF
:102BF00070686572616C0909446F6D61696E0909DD
:102C00005374617475730A002530327520252D3296
:102C1000317325730009534B49500A00094552523C
:102C20004F520A00094F4B0A004E52465F50300087
:102C30004E52465F434C4F434B004E52465F5254F8
:102C40004330004E52465F52544331004E52465F6D
:102C50004E564D43004E52465F5541525445310049
:102C60004E52465F554152544532004E52465F54D3
:102C700057494D32004E52465F5350494D33004E36
:102C800052465F54494D455230004E52465F5449BA
:102C90004D455231004E52465F54494D4552320027
:102CA0004E52465F5341414443004E52465F505797
:102CB0004D30004E52465F50574D31004E52465FE8
:102CC00050574D32004E52465F50574D33004E52D2
:102CD000465F574454004E52465F495043004E529F
:102CE000465F564D43004E52465F465055004E5289
:102CF000465F45475531004E52465F4547553200C5
:102D00004E52465F4450504943004E52465F524532
:102D100047554C41544F5253004E52465F4750491D
:102D20004F544531006D757465785F696E69742024
:102D300063616C6C65642077697468204E554C4CF7
:102D400020706172616D6574657200436F756C64AB
:102D5000206E6F7420616C6C6F63617465206D759B
:102D6000746578206265666F726520696E69746942
:102D7000616C697A696E6700464C4153485F300068
:102D80005352414D5F30004932435F320045525249
:102D90004F523A2043616E6E6F742066756C66699F
:102DA0006C6C204558545F415049207265717565BF
:102DB00073742E0D0A005741524E494E473A204F28
:102DC0007074696F6E616C204558545F41504920A2
:102DD00072657175657374206E6F742066756C66AC
:102DE000696C6C65642E0D0A0048575F4343335885
:102DF000585F30006D61696E0000000000C0000087
:102E00004118010004010020010000001801002009
:102E1000010000002C010020010000004001002002
:102E20000100000024000020240000200100000018
:102E300001000000340000203400002000000000E9
:102E40000100000000000000000000000000000081
:102E5000000000000090D00358000020580000201F
:102E600098000020A40000209C0000209400002076
:102E70006800002000000000750D01009808002087
:102E800001000000250E0100010E0100450E0100A9
:102E9000E10D0100B80000207C000020B0000020FF
:102EA00000000000A80000209C0800200100000095
:102EB000A008002001000000A4080020010000007C
:102EC000342C0100AC27010098270100700200207B
:102ED000742A010000000000000000000000000053
:102EE000E92D0100000000000000000000000000CB
:102EF000872D0100202901000C2901002400002059
:102F00000000000004010020040100200000000077
:102F1000000000000F000000180100201801002030
:102F200000000000000000000F0000002C01002045
:102F30002C01002000000000000000000F00000035
:102F400040010020400100200000000000000000BF
:102F50000F000000FFFFFFFFFFFFFFFFFFFFFFFF6E
:102F60000000000000000000000000000000000061
:102F70000000000000000000000000000000000051
:102F80000000000000000000000000000000000041
:102F90000000000000000000000000000000000031
:107FE0007FE97FE9F9F787BF7FE97FE9F9F736BFD6
:107FF0007FE97FE9F6F7A6B87FE97FE9F6F73CB8B5
:10800000FFFFFFFFFFFFFFFFFFFFFFFFFFFFFFFF80
:10801000FFFFFFFFFFFFFFFFFFFFFFFFFFFFFFFF70
:10802000FFFFFFFFFFFFFFFFFFFFFFFFFFFFFFFF60
:10803000FFFFFFFFFFFFFFFFFFFFFFFFFFFFFFFF50
:10804000FFFFFFFFFFFFFFFFFFFFFFFFFFFFFFFF40
:10805000FFFFFFFFFFFFFFFFFFFFFFFFFFFFFFFF30
:10806000FFFFFFFFFFFFFFFFFFFFFFFFFFFFFFFF20
:10807000FFFFFFFFFFFFFFFFFFFFFFFFFFFFFFFF10
:10808000FFFFFFFFFFFFFFFFFFFFFFFFFFFFFFFF00
:10809000FFFFFFFFFFFFFFFFFFFFFFFFFFFFFFFFF0
:1080A000FFFFFFFFFFFFFFFFFFFFFFFFFFFFFFFFE0
:1080B000FFFFFFFFFFFFFFFFFFFFFFFFFFFFFFFFD0
:1080C000FFFFFFFFFFFFFFFFFFFFFFFFFFFFFFFFC0
:1080D000FFFFFFFFFFFFFFFFFFFFFFFFFFFFFFFFB0
:1080E000FFFFFFFFFFFFFFFFFFFFFFFFFFFFFFFFA0
:1080F000FFFFFFFFFFFFFFFFFFFFFFFFFFFFFFFF90
:10810000FFFFFFFFFFFFFFFFFFFFFFFFFFFFFFFF7F
:10811000FFFFFFFFFFFFFFFFFFFFFFFFFFFFFFFF6F
:10812000FFFFFFFFFFFFFFFFFFFFFFFFFFFFFFFF5F
:10813000FFFFFFFFFFFFFFFFFFFFFFFFFFFFFFFF4F
:10814000FFFFFFFFFFFFFFFFFFFFFFFFFFFFFFFF3F
:10815000FFFFFFFFFFFFFFFFFFFFFFFFFFFFFFFF2F
:10816000FFFFFFFFFFFFFFFFFFFFFFFFFFFFFFFF1F
:10817000FFFFFFFFFFFFFFFFFFFFFFFFFFFFFFFF0F
:10818000FFFFFFFFFFFFFFFFFFFFFFFFFFFFFFFFFF
:10819000FFFFFFFFFFFFFFFFFFFFFFFFFFFFFFFFEF
:1081A000FFFFFFFFFFFFFFFFFFFFFFFFFFFFFFFFDF
:1081B000FFFFFFFFFFFFFFFFFFFFFFFFFFFFFFFFCF
:1081C000FFFFFFFFFFFFFFFFFFFFFFFFFFFFFFFFBF
:1081D000FFFFFFFFFFFFFFFFFFFFFFFFFFFFFFFFAF
:1081E000FFFFFFFFFFFFFFFFFFFFFFFFFFFFFFFF9F
:1081F000FFFFFFFFFFFFFFFFFFFFFFFFFFFFFFFF8F
:10820000D081022079440200A3B90300D9440200BE
:10821000D9440200D9440200D9440200D9440200E2
:1082200000000000000000000000000055410200B6
:10823000D944020000000000A1400200B53902004C
:108240003944020039440200394402003944020032
:108250003944020039440200394402003944020022
:108260003944020039440200394402003944020012
:108270003944020039440200394402003944020002
:1082800039440200394402003944020039440200F2
:1082900039440200394402003944020039440200E2
:1082A00039440200394402003944020039440200D2
:1082B000858702009BCD0300394402003944020047
:1082C00039440200394402003944020039440200B2
:1082D00039440200394402003944020039440200A2
:1082E0003944020039440200394402003944020092
:1082F0003944020039440200394402003944020082
:108300003944020039440200394402003944020071
:108310003944020039440200394402003944020061
:108320003944020039440200394402003944020051
:108330003944020039440200394402003944020041
:1083400039440200000000000000000000000000AE
:10835000000000000000000000000000000000001D
:10836000000000000000000000000000000000000D
:1083700000000000000000000000000000000000FD
:1083800000000000000000000000000000000000ED
:1083900000000000000000000000000000000000DD
:1083A00000000000000000000000000000000000CD
:1083B00000000000000000000000000000000000BD
:1083C00000000000000000000000000000000000AD
:1083D000000000000000000000000000000000009D
:1083E000000000000000000000000000000000008D
:1083F000000000000000000000000000000000007D
:10840000DEE61E284CBBCE8F025B00003C00000065
:10841000482B0300010000000082010000820100DF
:10842000FFFF0291000000000000000000000000BB
:10843000000000000000000000000000FFFFFFFF40
:1084400081F0004102E000BF83F0004330B54FEA05
:1084500041044FEA430594EA050F08BF90EA020F72
:108460001FBF54EA000C55EA020C7FEA645C7FEA05
:10847000655C00F0E2804FEA5454D4EB5555B8BF28
:108480006D420CDD2C4480EA020281EA030382EA99
:10849000000083EA010180EA020281EA0303362D2B
:1084A00088BF30BD11F0004F4FEA01314FF4801CFE
:1084B0004CEA113102D0404261EB410113F0004F10
:1084C0004FEA03334CEA133302D0524263EB4303C7
:1084D00094EA050F00F0A780A4F10104D5F1200E65
:1084E0000DDB02FA0EFC22FA05F2801841F10001C0
:1084F00003FA0EF2801843FA05F359410EE0A5F194
:1085000020050EF1200E012A03FA0EFC28BF4CF0C4
:10851000020C43FA05F3C01851EBE37101F000457A
:1085200007D54FF0000EDCF1000C7EEB00006EEB87
:108530000101B1F5801F1BD3B1F5001F0CD3490811
:108540005FEA30004FEA3C0C04F101044FEA445268
:1085500012F5800F80F09A80BCF1004F08BF5FEAEF
:10856000500C50F1000041EB045141EA050130BDCF
:108570005FEA4C0C404141EB0101013C28BFB1F5E1
:10858000801FE9D291F0000F04BF01460020B1FA2C
:1085900081F308BF2033A3F10B03B3F120020CDAFF
:1085A0000C3208DD02F1140CC2F10C0201FA0CF0DD
:1085B00021FA02F10CE002F11402D8BFC2F1200C42
:1085C00001FA02F120FA0CFCDCBF41EA0C019040F8
:1085D000E41AA2BF01EB0451294330BD6FEA040441
:1085E0001F3C1CDA0C340EDC04F11404C4F120022C
:1085F00020FA04F001FA02F340EA030021FA04F33E
:1086000045EA030130BDC4F10C04C4F1200220FA94
:1086100002F001FA04F340EA0300294630BD21FAD2
:1086200004F0294630BD94F0000F83F4801306BF98
:1086300081F480110134013D4EE77FEA645C18BF8C
:108640007FEA655C29D094EA050F08BF90EA020F23
:1086500005D054EA000C04BF1946104630BD91EA1B
:10866000030F1EBF0021002030BD5FEA545C05D11E
:108670004000494128BF41F0004130BD14F580045D
:108680003CBF01F5801130BD01F0004545F0FE41D1
:1086900041F470014FF0000030BD7FEA645C1ABF06
:1086A000194610467FEA655C1CBF0B46024650EA3D
:1086B000013406BF52EA033591EA030F41F4002169
:1086C00030BD00BF90F0000F04BF0021704730B5EF
:1086D0004FF4806404F132044FF000054FF00001C4
:1086E00050E700BF90F0000F04BF0021704730B585
:1086F0004FF4806404F1320410F0004548BF40425A
:108700004FF000013EE700BF42004FEAE2014FEAAE
:1087100031014FEA02701FBF12F07F4393F07F4F89
:1087200081F06051704732F07F4208BF704793F08C
:108730007F4F04BF41F40021704730B54FF460749F
:1087400001F0004521F000411CE700BF50EA0102A2
:1087500008BF704730B54FF000050AE050EA01024B
:1087600008BF704730B511F0004502D5404261EBBB
:1087700041014FF4806404F132045FEA915C3FF4FC
:10878000D8AE4FF003025FEADC0C18BF03325FEA99
:10879000DC0C18BF033202EBDC02C2F1200300FA4A
:1087A00003FC20FA02F001FA03FE40EA0E0021FA6F
:1087B00002F11444BDE600BF70B54FF0FF0C4CF45D
:1087C000E06C1CEA11541DBF1CEA135594EA0C0F0F
:1087D00095EA0C0F00F0DEF82C4481EA030621EA4A
:1087E0004C5123EA4C5350EA013518BF52EA033585
:1087F00041F4801143F4801338D0A0FB02CE4FF037
:108800000005E1FB02E506F00042E0FB03E54FF066
:108810000006E1FB03569CF0000F18BF4EF0010E5E
:10882000A4F1FF04B6F5007F64F5407404D25FEA5A
:108830004E0E6D4146EB060642EAC62141EA55510D
:108840004FEAC52040EA5E504FEACE2EB4F1FD0C4F
:1088500088BFBCF5E06F1ED8BEF1004F08BF5FEACD
:10886000500E50F1000041EB045170BD06F000467F
:1088700046EA010140EA020081EA0301B4EB5C042C
:10888000C2BFD4EB0C0541EA045170BD41F4801124
:108890004FF0000E013C00F3AB8014F1360FDEBF49
:1088A000002001F0004170BDC4F10004203C35DA25
:1088B0000C341BDC04F11404C4F1200500FA05F3A8
:1088C00020FA04F001FA05F240EA020001F0004249
:1088D00021F0004110EBD37021FA04F642EB0601BF
:1088E0005EEA430E08BF20EAD37070BDC4F10C04E9
:1088F000C4F1200500FA04F320FA05F001FA04F2AD
:1089000040EA020001F0004110EBD37041F1000198
:108910005EEA430E08BF20EAD37070BDC4F12005A3
:1089200000FA05F24EEA020E20FA04F301FA05F20B
:1089300043EA020321FA04F001F0004121FA04F2B3
:1089400020EA020000EBD3705EEA430E08BF20EA83
:10895000D37070BD94F0000F0FD101F000464000BD
:1089600041EB010111F4801F08BF013CF7D041EA3F
:10897000060195F0000F18BF704703F00046520043
:1089800043EB030313F4801F08BF013DF7D043EA14
:108990000603704794EA0C0F0CEA135518BF95EACA
:1089A0000C0F0CD050EA410618BF52EA4306D1D151
:1089B00081EA030101F000414FF0000070BD50EA70
:1089C000410606BF1046194652EA430619D094EAFA
:1089D0000C0F02D150EA013613D195EA0C0F05D1E4
:1089E00052EA03361CBF104619460AD181EA030138
:1089F00001F0004141F0FE4141F470014FF00000F0
:108A000070BD41F0FE4141F4780170BD70B54FF08A
:108A1000FF0C4CF4E06C1CEA11541DBF1CEA13550A
:108A200094EA0C0F95EA0C0F00F0A7F8A4EB0504EC
:108A300081EA030E52EA03354FEA013100F08880E3
:108A40004FEA03334FF0805545EA131343EA1263AC
:108A50004FEA022245EA111545EA10654FEA002661
:108A60000EF000419D4208BF964244F1FD0404F51A
:108A7000407402D25B084FEA3202B61A65EB030576
:108A80005B084FEA32024FF480104FF4002CB6EB33
:108A9000020E75EB030E22BFB61A754640EA0C00B3
:108AA0005B084FEA3202B6EB020E75EB030E22BFF3
:108AB000B61A754640EA5C005B084FEA3202B6EB34
:108AC000020E75EB030E22BFB61A754640EA9C00F3
:108AD0005B084FEA3202B6EB020E75EB030E22BFC3
:108AE000B61A754640EADC0055EA060E18D04FEA81
:108AF000051545EA16754FEA06164FEAC30343EA21
:108B000052734FEAC2025FEA1C1CC0D111F4801FED
:108B10000BD141EA00014FF000004FF0004CB6E7E6
:108B200011F4801F04BF01430020B4F1FD0C88BF85
:108B3000BCF5E06F3FF6AFAEB5EB030C04BFB6EB90
:108B4000020C5FEA500C50F1000041EB045170BD83
:108B50000EF0004E4EEA113114EB5C04C2BFD4EBB0
:108B60000C0541EA045170BD41F480114FF0000E34
:108B7000013C90E645EA060E8DE60CEA135594EAB0
:108B80000C0F08BF95EA0C0F3FF43BAF94EA0C0FB3
:108B90000AD150EA01347FF434AF95EA0C0F7FF428
:108BA00025AF104619462CE795EA0C0F06D152EA7C
:108BB00003353FF4FDAE1046194622E750EA410660
:108BC00018BF52EA43067FF4C5AE50EA41047FF471
:108BD0000DAF52EA43057FF4EBAE12E74FF0FF3CD6
:108BE00006E000BF4FF0010C02E000BF4FF0010CA7
:108BF0004DF804CD4FEA410C7FEA6C5C4FEA430C20
:108C000018BF7FEA6C5C1BD001B050EA410C0CBF6E
:108C100052EA430C91EA030F02BF90EA020F0020D0
:108C2000704710F1000F91EA030F58BF994208BF37
:108C300090422CBFD8176FEAE37040F001007047F4
:108C40004FEA410C7FEA6C5C02D150EA013C07D14B
:108C50004FEA430C7FEA6C5CD6D152EA033CD3D096
:108C60005DF8040B704700BF8446104662468C4690
:108C70001946634600E000BF01B5FFF7B7FF0028C3
:108C800048BF10F1000F01BD4DF808EDFFF7F4FFEC
:108C90000CBF012000205DF808FB00BF4DF808ED77
:108CA000FFF7EAFF34BF012000205DF808FB00BF9A
:108CB0004DF808EDFFF7E0FF94BF012000205DF8BC
:108CC00008FB00BF4DF808EDFFF7CEFF94BF012071
:108CD00000205DF808FB00BF4DF808EDFFF7C4FF6A
:108CE00034BF012000205DF808FB00BF4FEA4102BD
:108CF00012F5001215D211D56FF47873B3EB6252EE
:108D000012D94FEAC12343F0004343EA505311F014
:108D1000004F23FA02F018BF404270474FF00000A6
:108D2000704750EA013005D111F0004008BF6FF0E4
:108D3000004070474FF00000704700BF4A0011D25A
:108D400012F5001211D20DD56FF47873B3EB6252A5
:108D50000ED44FEAC12343F0004343EA505323FAB1
:108D600002F070474FF00000704750EA013002D126
:108D70004FF0FF3070474FF0000070474FEA41025C
:108D8000B2F1E04324BFB3F5001CDCF1FE5C0DD969
:108D900001F0004C4FEAC0024CEA5070B2F1004FB3
:108DA00040EB830008BF20F00100704711F0804FB6
:108DB00021D113F13872BCBF01F00040704741F47B
:108DC00080114FEA5252C2F11802C2F1200C10FA7F
:108DD0000CF320FA02F018BF40F001004FEAC12363
:108DE0004FEAD32303FA0CFC40EA0C0023FA02F307
:108DF0004FEA4303CCE77FEA625307D150EA0133DD
:108E00001EBF4FF0FE4040F44000704701F00040AC
:108E100040F0FE4040F40000704700BF7BB972B9DB
:108E20000029BEBF00204FF0004106E008BF002827
:108E30001CBF6FF000414FF0FF3000F0EDB9ADF115
:108E4000080C6DE904CE002909DB002B1ADB00F0C9
:108E500083F8DDF804E0DDE9022304B07047404206
:108E600061EB4101002B1BDB00F076F8DDF804E03C
:108E7000DDE9022304B0404261EB4101524263EB61
:108E800043037047524263EB430300F065F8DDF89B
:108E900004E0DDE9022304B0404261EB4101704788
:108EA000524263EB430300F057F8DDF804E0DDE9DC
:108EB000022304B0524263EB4303704753B94AB9EB
:108EC000002908BF00281CBF4FF0FF314FF0FF30D2
:108ED00000F0A2B9ADF1080C6DE904CE00F03CF849
:108EE000DDF804E0DDE9022304B0704738B5002264
:108EF000002304460D46FFF7D1FE28B92046294637
:108F0000BDE8384000F00AB8204605F1004100F005
:108F100005F8404261EB410138BD00BFD0B50022E9
:108F20000B4B06460F46FFF747FCFFF707FF0446CB
:108F3000FFF7C8FB0022074BFFF73EFC02460B463B
:108F400030463946FFF780FAFFF7F8FE2146D0BDDC
:108F50000000F03D0000F0412DE9F047089D044677
:108F60008846002B7DD18A4217463FD9B2FA82F259
:108F700042B1C2F120009140974024FA00F09440A1
:108F800040EA01084FEA174C230C1FFA87FEB8FB92
:108F9000FCF60CFB168106FB0EF043EA01439842F7
:108FA00005D9FB1802D2984200F22481013E191A19
:108FB000A3B2B1FBFCF00CFB101100FB0EFE43EA68
:108FC0000144A64505D93C1902D2A64500F20F81FD
:108FD000013840EA0640A4EB0E0400261DB1D4403F
:108FE0000023C5E900433146BDE8F08702B9FFDE42
:108FF000B2FA82F2002A50D1CB1B4FEA174E1FFA69
:1090000087F80126210CB3FBFEFC0EFB1C300B463F
:1090100008FB0CF941EA004189450AD979182CBFAF
:1090200001230023894502D9002B00F0D9800CF1DF
:10903000FF3CA1EB0901A3B2B1FBFEF00EFB101146
:1090400008FB00F843EA0144A04505D93C1902D2C7
:10905000A04500F2C9800138A4EB080440EA0C40A6
:10906000BCE78B4209D9002D00F0B1800026C5E98C
:10907000000130463146BDE8F087B3FA83F6002E92
:1090800046D18B42C0F0A680824240F2A380304697
:10909000002DA8D0C5E90048A5E79740C2F12003FC
:1090A00001FA02F04FEA174ED94024FA03F31FFAEF
:1090B00087F894400343B1FBFEF01E0C0EFB101129
:1090C00000FB08FC46EA01418C4509D979182CBF00
:1090D000012600268C4502D9002E00F0938001382D
:1090E000A1EB0C019BB2B1FBFEF60EFB161106FBC9
:1090F00008FC43EA01418C4505D9791802D28C4518
:1091000000F28780013EA1EB0C0346EA004679E7B6
:10911000C6F1200703FA06F402FA06FC01FA06FE7D
:10912000FA4020FA07F8F94000FA06F3224348EA29
:109130000E044FEA12484FEA144E1FFA82F9B1FBAF
:10914000F8FA08FB1A110AFB09F04EEA014E7045C5
:109150000AD912EB0E0E2CBF01210021704501D956
:10916000002952D00AF1FF3AAEEB000EA4B2BEFBCA
:10917000F8F008FB10EE00FB09F944EA0E4EF14549
:1091800005D912EB0E0E01D2F14538D8013840EA6C
:109190000A40AEEB090EA0FB0C89CE4541464C4679
:1091A00002D306D1434504D20138B8EB0C0169EB78
:1091B000020415B35A1A6EEB040EF2400EFA07F7CA
:1091C0002EFA06F300261743C5E900730BE72E4677
:1091D000284608E7841A61EB03010120884657E717
:1091E000ACF1020C394424E702383C4434E702383D
:1091F0003C44EEE6023E3B44D9E62E46F3E6023816
:109200009644C4E7023839446AE7AAF1020A964450
:10921000AAE7023E394476E7704700BF4FEA410CA7
:109220007FEA6C5C02D150EA013C0AD14FEA430C60
:109230007FEA6C5C02D152EA033C02D14FF000009D
:1092400070474FF00100704710F8012B11F8013BF7
:10925000012A28BF9A42F7D0D01A7047034613F864
:10926000012B002AFBD1181A0138704700000000BA
:10927000F0B50B880546042B8FB040F0AA805A4BFE
:109280001A781AB901221A700FB0F0BD836838211C
:10929000DB68984700280ADA5448554B5549C01AEC
:1092A000C008800140F0010021F0E1FCECE76A46D3
:1092B0000021284621F0DBF90121044602AA2846B4
:1092C00021F0D5F904AA04440221284621F0CFF95F
:1092D00022180AD0464B45484749C01AC0088001A9
:1092E00040F0010021F0C3FCCEE70198FFF7FAF946
:1092F0003BA3D3E90023FFF789FB044600980D4602
:10930000FFF7F0F902460B4620462946FFF79EF884
:1093100004460D460398CDE90845FFF7E3F930A36D
